:020000040800F2
:10000000E0510020E1010008855B0008ED370008A1
:10001000AD5A0008E10300086D6F00080000000001
:10002000000000000000000000000000490100087E
:10003000CD050008000000008D010008E166000801
:10004000FB010008FB010008FB010008C162000879
:10005000FB010008FB010008FB010008FB01000890
:10006000FB010008FB010008FB010008FB01000880
:100070002105000831050008410500085105000868
:100080006105000871050008FB0100084D6F0008BC
:100090005D6F0008E5030008F5030008FB01000898
:1000A000FB0100089D670008FB010008FB01000838
:1000B000AD670008BD670008FB010008FB010008F0
:1000C000FB010008FB010008FB010008FB01000820
:1000D000FB010008A96E0008B96E0008C96E00088F
:1000E000FB010008FB010008FB010008FB01000800
:1000F000FB010008FB010008FB010008FB010008F0
:10010000FB010008FB010008FB010008FB010008DF
:10011000ED68000879690008FB010008FB01000890
:10012000FB010008FB01000881050008910500089B
:10013000DFF810D000F0CAF800480047C59D00085D
:10014000AFF30080E0510020224B19680868B0E846
:10015000F00F80F30988BFF36F8F4FF0000080F33A
:1001600011884EF00D0E7047000000000648006830
:10017000006880F3088862B661B6BFF34F8FBFF3A3
:100180006F8F00DF00BF00BF08ED00E0EFF30980D4
:10019000BFF36F8F0F4B1A6820E9F00F106008B59E
:1001A0004FF0500080F31188BFF34F8FBFF36F8F74
:1001B0000BF072F84FF0000080F31188BDE80840A2
:1001C00019680868B0E8F00F80F30988BFF36F8FF3
:1001D000704700BF34070020EFF305807047000030
:1001E0000648804706480047FEE7FEE7FEE7FEE7D1
:1001F000FEE7FEE7FEE7FEE7FEE7FEE79B67000897
:1002000031010008202A04DB203A21FA02F0002103
:10021000704721FA02F3D040C2F120029140084316
:100220001946704740EA01039B0703D009E008C95B
:10023000121F08C0042AFAD203E011F8013B00F8AB
:10024000013B521EF9D27047D2B201E000F8012BF7
:10025000491EFBD270470022F6E710B513460A4646
:1002600004461946FFF7F0FF204610BD30B505469D
:100270002A460B4612F8010B13F8014B08B1A042B5
:10028000F8D01CB1002802D06D1CF1E7284630BD23
:10029000421C10F8011B0029FBD1801A704730B5B1
:1002A0000B46014600202022012409E021FA02F534
:1002B0009D4205D303FA02F5491B04FA02F52844CE
:1002C000151EA2F10102F1DC30BD0000064C074D05
:1002D00006E0E06840F0010394E807009847103416
:1002E000AC42F6D3FFF728FF10F0000830F000080A
:1002F00070B58D1810F8014B14F0030201D110F8FD
:10030000012B231106D110F8013B03E010F8016B1B
:1003100001F8016B521EF9D1ABB110F8012B04F0BA
:100320000C048A1A0C2C03D0A2EB84129B1C08E04C
:1003300010F8014BA2EB0422F8E712F8014B01F888
:10034000014B5B1EF9D5A942D4D3002070BD2DE925
:10035000F04104460D46164604F1B00800270AE0B5
:100360004146284606F00AFF2146284600F04AF892
:10037000A84610351037B742F2D31022414604F197
:10038000B000FFF74FFFBDE8F08170B504460E46A0
:1003900015463146204604F0DFF81022294604F1C4
:1003A000B000FFF73FFF70BD70B504460B4600205C
:1003B00013E000210DE0250105EB80050D44555D9E
:1003C00003EB8006765C754003EB800675544D1C8C
:1003D000E9B20429EFDB451CE8B20428E9DB70BD73
:1003E00000BFFEE710B5024800F03CFA10BD000067
:1003F000D422002010B5024800F034FA10BD0000ED
:10040000D422002070B505460E4600243246294607
:100410000020FFF7C9FF012400BF284606F046F977
:10042000284605F0EBFF0A2C00D10AE0284605F02B
:100430003FFB324629462046FFF7B6FF601CC4B298
:10044000EBE700BF324629460A20FFF7ADFF70BD3B
:1004500010B50020214948618860C8604862886101
:10046000C86148638862C86248648863C863086179
:100470000862086308641A4807F052F8194807F040
:100480004FF8194807F04CF8184807F049F8184891
:1004900007F046F8174807F043F8174807F040F808
:1004A000164807F03DF8164807F03AF8154807F0E7
:1004B00037F8154807F034F8144807F031F80020F1
:1004C00013490870134908701349087013490870DC
:1004D0004FF480300149486010BD000098070020AB
:1004E0000000070800100708002007080030070870
:1004F0000060070800680708007707080078070809
:10050000003807080040070800480708005007089F
:10051000F6000020F7000020F8000020F90000207D
:1005200010B5024800F01EFD10BD0000802F002015
:1005300010B5024800F016FD10BD00003C2F002051
:1005400010B5024800F00EFD10BD0000702E002016
:1005500010B5024800F006FD10BD00002C2E002052
:1005600010B5024800F0FEFC10BD0000B42E0020C3
:1005700010B5024800F0F6FC10BD0000F82E002077
:1005800010B5024800F0EEFC10BD0000A42D0020C4
:1005900010B5024800F0E6FC10BD0000E82D002078
:1005A00030B590F840500124AC40C56B6C600468D5
:1005B00063604468102C04D10468A2600468E160A0
:1005C00003E00468A1600468E26030BD7047000089
:1005D00010B504464FF6FF7322460249024803F065
:1005E0009BF810BD80140020602D002072B600BF63
:1005F000FEE700000021074AD1610749096941F07F
:100600000401054A11611146096941F04001116177
:1006100070470000D0400020002002400021074A1F
:10062000D1610749096941F00201054A116111468A
:100630004861096941F0400111617047D0400020D4
:10064000002002400022054BDA61054A126942F09F
:100650000102034B1A61018070470000D040002066
:100660000020024000201E49C96801F0100139B184
:100670001C49C96941F002011A4AD16140F01000D9
:100680001749C96801F0040139B11649C96941F037
:100690000101144AD16140F004001149C96901F017
:1006A000010169B10F49C96941F004010D4AD161E5
:1006B00000BF0B49C96921F00101094AD16100BF9E
:1006C00000BF40F20111884206D10549C96921F0F5
:1006D0000101034AD16101E00149C86000BF7047D0
:1006E00000200240D040002070B5044601F038F9E7
:1006F000054609E0601C38B124B101F031F9401B16
:10070000A04201D9032070BD1248C06800F001006A
:100710000028EFD10F48C06800F0200020B100BFD2
:1007200020200C49C86000BF0A48C06800F01000D3
:1007300048B90848C06900F0010020B90548C06800
:1007400000F0040018B1FFF78DFF0120DBE7002067
:10075000D9E7000000200240F0B504460A462168AF
:1007600094F82050012D01D0022D74D1D1F800024F
:1007700040F00100C1F80002107D00F01F060120CA
:1007800000FA06F3D1F81C029843C1F81C02D069A4
:10079000C8B9D1F80C029843C1F80C02908880B215
:1007A000968940EA064601F51070576940F83760AF
:1007B000108880B2168940EA064601F51070576924
:1007C00000EBC7004660D069012819D1D1F80C02AE
:1007D0001843C1F80C02908880B2168840EA064699
:1007E00001F51070576940F83760908980B216891A
:1007F00040EA064601F51070576900EBC7004660F5
:10080000906928B9D1F804029843C1F8040204E0C1
:10081000D1F804021843C1F80402106928B9D1F8CC
:1008200014029843C1F8140204E0D1F814021843EA
:10083000C1F81402106A012804D1D1F81C0218432F
:10084000C1F81C02D1F8000220F00100C1F800023A
:100850000020F0BDFFE7606A40F480206062012064
:10086000F7E770472DE9F05F0446002520684669E8
:100870002068D0F80490206887682068D0F80CA021
:100880002068D0F810B02068D0F8188006F0010079
:10089000002855D007F00100C0B101202168886010
:1008A00007F0020018B1204600F057FA0EE007F0FA
:1008B000040010B145F4006508E007F0080010B12D
:1008C00045F4805502E0204600F046FA07F48070B7
:1008D000C8B14FF480702168886007F4007018B1C7
:1008E000204600F03CFA0EE007F4806010B145F4B9
:1008F000005508E007F4006010B145F4804502E0BF
:10090000204600F02BFA07F48030C8B14FF4803055
:100910002168886007F4003018B1204600F021FA01
:100920000EE007F4802010B145F4004508E007F41C
:10093000002010B145F4803502E0204600F010FAA6
:1009400006F0080038B10AF0100020B145F4007537
:1009500010202168C86006F0040040B10AF00800C9
:1009600028B108202168C860204600F0C1F906F0CF
:10097000020038B12068C06800F0030010B12046C2
:1009800000F0B7F906F0400038B10BF0100020B1CC
:1009900045F4806510202168086106F0200040B110
:1009A0000BF0080028B1082021680861204600F0FB
:1009B000A1F906F0100038B12068006900F00300CA
:1009C00010B1204600F097F906F4003040B109F06C
:1009D000100028B1102021684860204600F08CF9F2
:1009E00006F4803040B109F0080028B108202168E1
:1009F0004860204600F0B6F906F4004088B309F0DC
:100A0000040078B306F4807020B108F0010008B14A
:100A100045F0010506F4007020B108F0020008B1AD
:100A200045F0020506F4806020B108F0040008B12A
:100A300045F0040506F40060A0B108F0700088B12C
:100A400008F07000402817D006DC10280BD02028B2
:100A50000CD0302819D10CE0502810D0602814D1C7
:100A600010E01DE019E045F008050FE045F0100525
:100A70000CE045F0200509E045F0400506E045F0B2
:100A8000800503E045F4807500E000BF00BF2068EA
:100A9000806920F070002168886104202168486026
:100AA0002DB1606A284360622046FFF7DAFEBDE898
:100AB000F09F70B504460CB9012070BD94F8200079
:100AC00010B9204600F0B0F82068006840F001003E
:100AD0002168086000F044FF05460DE000F040FF8B
:100AE000401B0A2808D9606A40F400306062052083
:100AF00084F820000120E0E72068406800F0010051
:100B00000028EBD02068006820F00200216808600F
:100B100000F026FF05460DE000F022FF401B0A28EA
:100B200008D9606A40F400306062052084F8200033
:100B30000120C2E72068406800F002000028EBD1E5
:100B4000207E012806D12068006840F080002168DE
:100B5000086005E02068006820F0800021680860D7
:100B6000607E012806D12068006840F040002168BE
:100B7000086005E02068006820F0400021680860F7
:100B8000A07E012806D12068006840F0200021687E
:100B9000086005E02068006820F0200021680860F7
:100BA000E07E012806D12068006820F0100021684E
:100BB000086005E02068006840F0100021680860C7
:100BC000207F012806D12068006840F008002168D5
:100BD000086005E02068006820F0080021680860CF
:100BE000607F012806D12068006840F00400216879
:100BF000086005E02068006820F0040021680860B3
:100C0000D4E9020108432169084361690843616826
:100C1000491E08432168C86100206062012084F8F1
:100C20002000002049E7000010B586B004460020EF
:100C300002900390049005902A49206888424ED182
:100C400000BF2948C06940F000702749C8610846C4
:100C5000C06900F00070019000BF00BF00BF0846EF
:100C6000806940F0040088610846806900F0040053
:100C7000019000BF00BFC8140290002003900490B0
:100C800002A91A4800F0B4FC4FF4805002900220F0
:100C900003900320059002A9144800F0A9FC00224B
:100CA0000521132000F012FF132000F0FFFE0022A8
:100CB0000521142000F00AFF142000F0F7FE0022A6
:100CC0000521152000F002FF152000F0EFFE0022A4
:100CD0000521162000F0FAFE162000F0E7FE06B00F
:100CE00010BD0000006400400010024000080140F8
:100CF0007047704770477047704770B5044694F866
:100D00002000012822D1022084F8200020680068F9
:100D100020F001002168086000F022FE05460DE089
:100D200000F01EFE401B0A2808D9606A40F400301B
:100D30006062052084F82000012070BD20684068B2
:100D400000F001000028EBD16062F6E7606A40F431
:100D5000002060620120F0E77047704770477047DD
:100D60007047704770470146002291F82100022821
:100D700008D00420886300BF002081F8200000BF55
:100D8000012070470868006820F00E000B681860AA
:100D90000868006820F001000B68186091F8403086
:100DA00001209840CB6B5860012081F8210000BFE2
:100DB000002081F8200000BF1046E2E770B504462D
:100DC000002594F82100022803D00420A063012507
:100DD000C1E02068006820F00E00216808602068EB
:100DE000006820F00100216808605C4920688842A2
:100DF00052D95A4978392068884201D1012047E008
:100E0000564964392068884201D1102040E0534996
:100E100050392068884201D1801539E04F493C396A
:100E20002068884201D1801432E04C49283920687A
:100E3000884202D14FF480302AE0484914392068B2
:100E4000884202D14FF4801022E044492068884251
:100E500001D140041CE042492068884201D10120B0
:100E600016E03F4914312068884201D110200FE07C
:100E70003B4928312068884201D1801508E0384973
:100E80003C312068884201D1801401E04FF4803069
:100E90003349091F086051E0304978392068884299
:100EA00001D1012047E02D4964392068884201D1F1
:100EB000102040E0294950392068884201D180152E
:100EC00039E026493C392068884201D1801432E05B
:100ED000224928392068884202D14FF480302AE024
:100EE0001E4914392068884202D14FF4801022E054
:100EF0001A492068884201D140041CE01849206842
:100F0000884201D1012016E0154914312068884239
:100F100001D110200FE0124928312068884201D108
:100F2000801508E00E493C312068884201D18014C8
:100F300001E04FF48030094980394860012084F88D
:100F4000210000BF002084F8200000BF606B10B1BA
:100F50002046616B8847284670BD00008000024033
:100F60000804024070B50446E06B05682068066816
:100F700094F84010042088402840002875D006F0DE
:100F800004000028FAD02068006800F0200028B98A
:100F90002068006820F0040021680860D5492068B6
:100FA000884254D9D34978392068884201D1042035
:100FB00049E0D04964392068884201D1402042E0AC
:100FC000CC4950392068884201D100153BE0C9491D
:100FD0003C392068884202D14FF4804033E0C54953
:100FE00028392068884202D14FF480202BE0C14983
:100FF00014392068884202D14FF4800023E0BD49B3
:101000002068884201D1C0041DE0BB4920688842A5
:1010100001D1042017E0B84914312068884201D179
:10102000402010E0B44928312068884201D10015E1
:1010300009E0B1493C312068884202D14FF4804038
:1010400001E04FF48020AC49091F086054E0A94931
:1010500078392068884201D104204AE0A5496439E2
:101060002068884202D1402043E04CE0A149503939
:101070002068884201D100153BE09E493C39206838
:10108000884202D14FF4804033E09A4928392068E1
:10109000884202D14FF480202BE096491439206811
:1010A000884202D14FF4800023E0924920688842B0
:1010B00001D1C0041DE090492068884201D104207C
:1010C00017E08D4914312068884201D1402010E09A
:1010D000894928312068884201D1001509E08649F4
:1010E0003C312068884202D14FF4804001E04FF447
:1010F0008020804980394860E06A002802D020467C
:10110000E16A8847F4E094F84010022088402840C3
:10111000002871D006F002000028FAD0206800688C
:1011200000F0200040B92068006820F00A00216823
:101130000860012084F821006E492068884254D953
:101140006C4978392068884201D1022049E0694918
:1011500064392068884201D1202042E06549503935
:101160002068884201D140153BE062493C39206843
:10117000884202D14FF4005033E05E49283920689C
:10118000884202D14FF400302BE05A4914392068CC
:10119000884202D14FF4001023E05649206888426B
:1011A00001D180041DE054492068884201D1022009
:1011B00017E0514914312068884201D1202010E005
:1011C0004D4928312068884201D1401509E04A493B
:1011D0003C312068884202D14FF4005001E04FF4C6
:1011E00000304549091F086054E0424978392068B9
:1011F000884202D102204AE057E03E496439206823
:10120000884201D1202042E03A4950392068884282
:1012100001D140153BE037493C392068884202D172
:101220004FF4005033E0334928392068884202D116
:101230004FF400302BE02F4914392068884202D146
:101240004FF4001023E02B492068884201D180042C
:101250001DE029492068884201D1022017E0264973
:1012600014312068884201D1202010E02249283121
:101270002068884201D1401509E01F493C312068AF
:10128000884202D14FF4005001E04FF40030194978
:101290008039486000BF002084F8200000BFA06AA9
:1012A00030B32046A16A884722E094F84010082015
:1012B00088402840E0B106F00800C8B12068006806
:1012C00020F00E002168086094F84010012088404A
:1012D000E16B48600120A06384F8210000BF00207A
:1012E00084F8200000BF206B10B12046216B884796
:1012F00070BD000080000240080402400146002248
:1013000009B9012070471E4B086898420BD21D4B4B
:101310000868C01A1423B0FBF3F080000864194871
:101320000838C8630AE0164B0868C01A1423B0FBDB
:10133000F3F08000086412480838C863022081F87E
:1013400021000868026843F6F0708243D1E9010386
:101350001843CB6818430B6918434B6918438B69D2
:101360001843CB6918430243086802600020886371
:10137000012081F82100002081F8200000BFC1E792
:1013800008040240080002402DE9F04104460D46E1
:1013900016461F464FF0000800BF94F820000128B1
:1013A00002D10220BDE8F081012084F8200000BFB6
:1013B00094F8210001282CD1022084F8210000207B
:1013C000A0632068006820F00100216808603B46A7
:1013D000324629462046FFF7E3F8E06A30B120683C
:1013E000006840F00E00216808600BE0206800688B
:1013F00020F00400216808602068006840F00A00BE
:10140000216808602068006840F0010021680860D9
:1014100006E000BF002084F8200000BF4FF0020863
:101420004046BFE770B5044600F09AFA06462546E6
:10143000681C10B104480078054400BF00F090FA21
:10144000801BA842FAD370BD2C0700202DE9F04183
:1014500004460E460127002500BF2648007E0128CD
:1014600002D10220BDE8F08101202249087600BFA8
:101470002068022813D14CF25030FFF735F990BBA9
:101480000120FFF7B7F84CF25030FFF72DF907466F
:101490001948006920F004001749086123E04CF264
:1014A0005030FFF721F9F0B94FF0FF303060A568F8
:1014B00012E02846FFF7B2F84CF25030FFF714F96B
:1014C00007460D48006920F002000B4908610FB182
:1014D000356007E005F50065D4E9021001EBC02096
:1014E000A842E6D800BF00BF00200249087600BF2E
:1014F0003846B7E7D040002000200240034800698A
:1015000040F080000149086100207047002002403F
:101510002DE9FE4F05468B461746984601260024C6
:101520000020029000BF2448007E012802D1022042
:10153000BDE8FE8F01202049087600BF4CF25030F4
:10154000FFF7D2F8064686BB012D02D1012002909A
:1015500006E0022D02D10220029001E00420029058
:1015600000241EE02201B946C24648465146FEF715
:1015700049FE80B20190022000FB04B00090019966
:10158000FFF760F84CF25030FFF7AEF806460B4814
:10159000006920F001000949086106B104E0601CFF
:1015A000C4B202988442DDDB00BF00BF00200249C4
:1015B000087600BF3046BBE7D04000200020024044
:1015C00000200849096901F0800151B10649054A26
:1015D0005160064951601146096901F0800101B16D
:1015E000012070470020024023016745AB89EFCD01
:1015F0002DE9F847024600239C467BE14FF00108A5
:1016000008FA03F4D1F8008008EA0400A0427DD172
:10161000DFF8F4A2D1F80480A8EB0A09D0453AD04B
:1016200014DCB8F1030F50D009DCB8F1000F31D051
:10163000B8F1010F1CD0B8F1020F49D120E0B8F188
:10164000110F18D0B8F1120F42D11EE0B9F5881F62
:1016500025D006DCB9F5803F20D0B9F5801F37D101
:101660001AE0B9F5001F18D0B9F5041F30D117E002
:10167000D1F80CC02DE0D1F80C8008F1040C28E062
:10168000D1F80C8008F1080C23E0D1F80C8008F1A7
:101690000C0C1EE000BF00BF00BF00BF00BF00BFBA
:1016A000D1F80880B8F1000F02D14FF0040C0BE024
:1016B000D1F80880B8F1010F03D14FF0080C146184
:1016C00002E04FF0080C546103E04FF0000C00E022
:1016D00000BF00BFFF2801D8904601E002F10408D6
:1016E0004646FF2802D84FEA830803E0A3F1080822
:1016F0004FEA88084746D6F800804FF00F0909FAEC
:1017000007F928EA09080CFA07F900E07AE048EA44
:101710000908C6F80080D1F8048008F08058B8F1B4
:10172000805F6FD100BFDFF8E481D8F8188048F0FF
:101730000108DFF8D891C9F81880C846D8F8188091
:1017400008F00108CDF8008000BF00BF4FEAB938AB
:101750004FEA930958F829504FEA83784FEA1879ED
:101760004FF00F0808FA09F825EA0805DFF8A0810C
:10177000424502D14FF0000824E0DFF8988142454D
:1017800002D14FF001081DE0DFF88C81424502D103
:101790004FF0020816E0DFF88481424502D14FF095
:1017A00003080FE0DFF87881424502D14FF00408CA
:1017B00008E0DFF87081424502D14FF0050801E0F2
:1017C0004FF006084FEA83794FEA197908FA09F8C9
:1017D00048EA0505DFF850814FEA930948F8295097
:1017E000D1F8048008F48038B8F5803F0BD1DFF8D9
:1017F0003C81D8F8008048EA0008DFF83091C9F849
:1018000000800AE075E0DFF82481D8F8008028EA3B
:101810000008DFF81891C9F80080D1F8048008F4B6
:101820000038B8F5003F0ED1DFF8008108F1040858
:10183000D8F8008048EA0008DFF8F09009F10409C0
:10184000C9F800800DE0DFF8E48008F10408D8F85A
:10185000008028EA0008DFF8D49009F10409C9F8EB
:101860000080D1F8048008F48018B8F5801F0ED1EC
:10187000DFF8B88008F10808D8F8008048EA0008C6
:10188000DFF8A89009F10809C9F800800DE0DFF839
:101890009C8008F10808D8F8008028EA0008DFF8E2
:1018A0008C9009F10809C9F80080D1F8048008F487
:1018B0000018B8F5001F0ED1DFF8708008F10C0891
:1018C000D8F8008048EA0008DFF8609009F10C09B8
:1018D000C9F800800DE0DFF8548008F10C08D8F852
:1018E000008028EA0008DFF8449009F10C09C9F8E3
:1018F00000805B1CD1F8008028FA03F8B8F1000FD3
:101900007FF47CAEBDE8F8870000111000100240A3
:1019100000080140000C014000100140001401408B
:1019200000180140001C0140080001400004014073
:10193000024693680B400BB1012000E00020704785
:1019400010B5C26821EA020302EA010443EA044333
:10195000036110BD0AB1016101E00B04036170472E
:101960000148006870470000240700200348006811
:10197000034909780844014908607047240700209A
:101980002C07002010B50848006840F010000649F8
:101990000860032000F0D8F80F2000F007F800F0EE
:1019A00055F8002010BD000000200240F0B587B0BF
:1019B000044600260027002500BF1F48806940F428
:1019C00000601D4988610846806900F4006000904D
:1019D00000BF00BF01A902A800F0C8FA00F0FEFA9B
:1019E00006461648B6FBF0F0471E15481549086034
:1019F00040F2E7311348C160476000210161816016
:101A0000816101F075F8054695B90E4801F0E0F8DE
:101A100005466DB9192000F049F8102C07D20022B4
:101A20002146192000F052F80748046000E0012523
:101A3000284607B0F0BD00000010024040420F00F1
:101A4000002C0140843000202807002008B500BF8A
:101A50001448806940F00100124988610846806995
:101A600000F00100009000BF00BF00BF0846C06941
:101A700040F08050C8610846C06900F08050009076
:101A800000BF00BF00220F21901E00F01FF800BF12
:101A90000549486820F0E06040F00070486000BFF1
:101AA00008BD000000100240000001400146084649
:101AB000002809DB00F01F0301229A4043099B0024
:101AC00003F1E023C3F8002100BF70472DE9F05F68
:101AD00080460D461646002705F06EFB0746394640
:101AE0002A46334601F00700C0F1070ABAF1040F95
:101AF00002D94FF0040A01E0C0F1070AD14600F113
:101B0000040ABAF1070F02D24FF0000A01E0A0F177
:101B1000030AD4464FF0010A0AFA09FAAAF1010AA7
:101B20000AEA020A0AFA0CFA4FF0010B0BFA0CFB54
:101B3000ABF1010B0BEA030B4AEA0B0421464046CA
:101B400005F042FBBDE8F09F00BF00F00702064B26
:101B500019684FF6FF031940044B0B4343EA022177
:101B6000014B196000BF70470CED00E00000FA0562
:101B7000012001490862704700000E422DE9F04340
:101B800085B0064642A30FCB01AC0FC444A0006849
:101B900000904FF00008002500270024A146042EE5
:101BA00036D004DC012E3BD0022E6BD15FE0082E34
:101BB00032D0102E66D13B484468006800F0807037
:101BC00000B301A8C4F38341475C04F4803070B1D2
:101BD00034484068C0F340401DF8008004F4803071
:101BE00040B13148B0FBF8F000FB07F502E02F48A8
:101BF00007FB00F52B48406800F48000B0F5800F2B
:101C000001D1A94603E068000321B0FBF1F93AE0F5
:101C100000F0F4F9814636E000F0F0F9814632E058
:101C20002048046A04F44070B0F5807F05D104F0C8
:101C3000020010B14FF4004918E004F44070B0F510
:101C4000007F07D11748406A00F0020010B149F642
:101C500040490BE004F44070B0F5407F06D11148D4
:101C6000006800F4003008B14FF224490BE000F0A6
:101C7000B5F90C494968C1F38131491C4900B0FBF1
:101C8000F1F900E000BF00BF484605B0BDE8F083B1
:101C900002030405060708090A0B0C0D0E0F1010AD
:101CA000010200000010024000127A0000093D000D
:101CB000F8B5044600260025207800F00100002831
:101CC0006BD000274348C06900F0805070B900BF56
:101CD0004048C06940F080503E49C8610846C0692C
:101CE00000F08050009000BF00BF01273A48006814
:101CF00000F48070B0B93848006840F4807036490C
:101D00000860FFF72DFE064606E0FFF729FE801B60
:101D1000642801D90320F8BD2F48006800F48070C2
:101D20000028F2D02B48006A00F440752DB3A0883B
:101D300000F44070A84220D02648006A20F4407584
:101D4000012026490860002008602248056205F04D
:101D5000010090B1FFF704FE064608E0FFF700FE21
:101D6000801B41F28831884201D90320D3E719480A
:101D7000006A00F002000028F0D01648006A20F443
:101D800040706168084313490862012F04D1084676
:101D9000C06920F08050C86100BF207800F00200C8
:101DA000022807D10B48406820F44040A16808434E
:101DB00008494860207800F01000102807D1054835
:101DC000406820F4800061690843024948600020AF
:101DD000A1E70000001002400070004040044242B1
:101DE00070B504460D460CB9012070BD5A48006814
:101DF00000F00700A8420ED25748006820F0070004
:101E00002843554908600846006800F00700A842CA
:101E100001D00120E9E7207800F0020002281DD15E
:101E2000207800F00400042805D14C48406840F4B4
:101E3000E0604A494860207800F00800082805D191
:101E40004648406840F46050444948604348406810
:101E500020F0F000A168084340494860207800F075
:101E6000010078B36068012806D13C48006800F49E
:101E7000003090B90120B8E76068022806D13748E1
:101E8000006800F0007040B90120AEE733480068F8
:101E900000F0020008B90120A7E73048406820F0B0
:101EA0000300616808432D494860FFF759FD064665
:101EB00009E0FFF755FD801B41F28831884202D9C5
:101EC000032092E707E02548406800F00C006168B5
:101ED000B0EB810FEDD12048006800F00700A84268
:101EE0000ED91D48006820F0070028431A490860F1
:101EF0000846006800F00700A84201D0012074E7FE
:101F0000207800F00400042807D11448406820F429
:101F1000E060E168084311494860207800F008005B
:101F2000082808D10D48406820F46050216940EA33
:101F3000C1000A49486000F061F808494968C1F3E6
:101F40000311074A515CC84006490860064800680A
:101F5000FFF72CFD002048E700200240001002405F
:101F60009BE5000830070020280700200F220260B0
:101F70000D4A526802F0030242600B4A526802F0B6
:101F8000F0028260084A526802F4E062C260064AC7
:101F9000526802F46052D2080261044A126802F0E8
:101FA00007020A6070470000001002400020024053
:101FB00001480068704700003007002000B5FFF7B7
:101FC000F7FF04494968C1F30221034A515CC84044
:101FD00000BD000000100240ABE5000800B5FFF7AF
:101FE000E7FF04494968C1F3C221034A515CC84074
:101FF00000BD000000100240ABE50008F0B585B060
:102000000FF26C0C9CE8E01001A8A0E8E0101CA501
:102010002D68009500210022002300240020194D86
:10202000696801F00C05F5B1042D02D0082D19D115
:1020300001E0154819E001ADC1F38346AC5D01F440
:10204000803555B10F4D6D68C5F340451DF805202D
:102050000D4D6543B5FBF2F302E00C4D04FB05F3B7
:10206000184602E000BF084800BF00BF05B0F0BD41
:1020700002030405060708090A0B0C0D0E0F1010C9
:10208000010200000010024000127A0000093D0029
:10209000F8B504460CB90120F8BD207800F0010025
:1020A000002878D0F848406800F00C0004280CD0D4
:1020B000F548406800F00C00082811D1F24840684B
:1020C00000F48030B0F5803F0AD1EF48006800F49A
:1020D000003000285FD0606800285CD10120DBE779
:1020E00000BF6068B0F5803F06D1E748006840F463
:1020F0008030E549086028E0606858B9E248006827
:1021000020F48030E04908600846006820F4802010
:1021100008601AE06068B0F5A02F0BD1DA480068BB
:1021200040F48020D84908600846006840F48030B8
:1021300008600AE0D448006820F48030D249086082
:102140000846006820F48020086000BF606888B1FD
:10215000FFF706FC054606E0FFF702FC401B64287B
:1021600001D9032098E7C848006800F4003000282F
:10217000F2D010E0FFF7F4FB054606E0FFF7F0FBB6
:10218000401B642801D9032086E7BF48006800F49B
:1021900000300028F2D1207800F00200022857D148
:1021A000B948406800F00C0050B1B748406800F0F2
:1021B0000C00082818D1B448406800F4803098B961
:1021C000B148006800F0020020B12069012801D068
:1021D000012061E7AC48006820F0F800616940EA3E
:1021E000C100A949086033E02069E8B10120A7498E
:1021F0000860FFF7B5FB054606E0FFF7B1FB401BA3
:10220000022801D9032047E79F48006800F0020038
:102210000028F2D09C48006820F0F800616940EA8C
:10222000C1009949086013E0002098490860FFF751
:1022300097FB054606E0FFF793FB401B022801D9F8
:10224000032029E79048006800F002000028F2D13E
:10225000207800F0080008282DD1A069B8B101202D
:102260008B490860FFF77CFB054606E0FFF778FB2B
:10227000401B022801D903200EE78348406A00F082
:1022800002000028F2D0012003F0C0FF13E000207C
:102290007F490860FFF764FB054606E0FFF760FB37
:1022A000401B022801D90320F6E67748406A00F077
:1022B00002000028F2D1207800F00400042873D135
:1022C00000277148C06900F0805070B900BF6E48A7
:1022D000C06940F080506C49C8610846C06900F090
:1022E0008050009000BF00BF01276A48006800F4DA
:1022F0008070B0B96748006840F480706549086034
:10230000FFF72EFB054606E0FFF72AFB401B64287B
:1023100001D90320C0E65F48006800F480700028FF
:10232000F2D000BFE068012806D15748006A40F0AB
:1023300001005549086227E0E06858B95248006A30
:1023400020F00100504908620846006A20F00400AD
:10235000086219E0E06805280BD14B48006A40F09C
:102360000400494908620846006A40F0010008621A
:102370000AE04548006A20F0010043490862084627
:10238000006A20F00400086200BFE068A0B1FFF717
:10239000E7FA054609E0FFF7E3FA401B41F288310E
:1023A000884202D9032077E622E03748006A00F02D
:1023B00002000028EFD012E0FFF7D2FA054608E04D
:1023C000FFF7CEFA401B41F28831884201D9032041
:1023D00062E62D48006A00F002000028F0D1012FCB
:1023E00005D12948C06920F080502749C86100BF45
:1023F000E069C8B32448406800F00C00082860D0A9
:10240000E069022848D1002020490866FFF7A8FAB1
:10241000054606E0FFF7A4FA401B022801D9032075
:102420003AE61948006800F000700028F2D1206AEE
:10243000B0F5803F07D11448406820F40030A1680F
:10244000084311494860D4E9080108430E49496826
:1024500021F4741108430C49486001200B490866B7
:10246000FFF77EFA054607E03DE0FFF779FA401BEB
:10247000022801D903200FE60348006800F000702D
:102480000028F2D02FE0000000100240000042427D
:102490008004424200700040002014490866FFF7A3
:1024A0005FFA054606E0FFF75BFA401B022801D9F8
:1024B0000320F1E50E48006800F000700028F2D11A
:1024C00011E0E069012800D1E6E50948466806F414
:1024D0008031206A814204D106F47011606A814221
:1024E00001D00120D8E50020D6E5000000004242DE
:1024F0000010024010B5034600220020024A02EB01
:1025000081021468A0B210BD006C004010B50346F3
:102510000020034800EB810094B2046010BD00006D
:10252000006C00407047704710B504462068006892
:1025300000F00100F0B12068406800F00100C8B16F
:1025400020684068C0F3800048B12046FFF7EBFFE9
:102550006FF00400216848600420607404E02046A5
:10256000FFF7E0FF012060742068406820F0010060
:102570002168486010BD000070B5044600250CB904
:10258000012070BD607C20B900202074204600F03E
:102590005BF802206074204600F068F918B104204E
:1025A00060740120EDE7204603F04FFE18B10420CF
:1025B00060740120E5E72068406820F0070021688A
:1025C0004860A06828B11F48006820F001001D493C
:1025D00008601C48001F006820F46070A168084370
:1025E0001849091F08606068401C08B1656809E067
:1025F0000120FFF7C3FA05461DB9042060740120CD
:10260000BFE76D1E2068806820F00F0040EA15408B
:10261000216888602068C06865F30F002168C86081
:10262000204603F02FFE18B1042060740120A8E7B3
:102630000021E17301216173A17301206074002006
:102640009FE70000306C004038B504460F49206811
:1026500088421AD1FFF78CFA00BF0D48C06940F0DC
:1026600000600B49C8610846C06900F00060009036
:1026700000BF00BF01200749086000220521032098
:10268000FFF724FA0320FFF711FA38BD00280040B5
:10269000001002403C0442422DE9F04704460D463A
:1026A000904600260027B14604B115B90120BDE8C7
:1026B000F08700BF207C012801D10220F7E701202C
:1026C000207400BF02206074B8F1000F06D1E978D1
:1026D000E17369786173A978A1730BE0E87803F07E
:1026E000A9FDE073687803F0A5FD6073A87803F096
:1026F000A1FDA073A27B617BE07B03F00FFE207342
:10270000207B2870204603F0EFFD06464FF4616001
:10271000B6FBF0F9B9F1180F2FD91820B9FBF0F07A
:1027200000EB4000C000C0EB4011C1EB0020A6EB65
:1027300000163146204603F04AFE38B1042060748A
:1027400000BF0020207400BF0120B0E7204603F046
:10275000BFFD0746781C80B1B7420ED20B48074434
:102760003946204603F01CFE38B10420607400BFD7
:102770000020207400BF012099E70120607400BF91
:102780000020207400BF00BF91E7000080510100CD
:102790002DE9F04704460D4690460026002704B177
:1027A00015B90120BDE8F08700BF207C012801D1C8
:1027B0000220F7E70120207400BF02206074B8F106
:1027C000000F0BD128784FF4616148436978C1EB61
:1027D000011100EB8100A978461812E0287803F077
:1027E00029FD4FF4616100FB01F9687803F022FDD7
:1027F000C0EB001009EB8009A87803F01BFD09EB82
:1028000000063146204603F0E2FD38B10420607432
:1028100000BF0020207400BF0120C3E7206840688B
:1028200020F0050021684860204603F051FD07466E
:10283000781C80B1B7420ED20B4807443946204677
:1028400003F0AEFD38B10420607400BF0020207496
:1028500000BF0120A6E70120607400BF00202074A3
:1028600000BF00BF9EE700008051010070B5044624
:1028700000250CB9012070BD2068406820F00800D8
:1028800021684860FFF76CF8054607E0FFF768F835
:10289000401BB0F57A7F01D90320ECE7206840683F
:1028A00000F008000028F1D00020E4E710B504464D
:1028B0000CB9012010BD606A38B96068B0F5827F3C
:1028C00000D105E00021E16102E0002121616161A8
:1028D0000021A16294F8510028B9002084F850002A
:1028E000204600F043F8022084F851002068006878
:1028F00020F0400021680860A08800F482702189DF
:1029000001F404410843A18901F400610843217CDA
:1029100001F002010843217D01F001010843218BF0
:1029200001F400710843217F01F0380108432021A0
:10293000095D01F080010843218D01F40051084335
:10294000216808600421A06901EA104021684860FC
:102950002068C06920F400602168C86100206065BB
:10296000012084F851000020A4E7000010B586B0D3
:102970000446002002900390049005902F4920689F
:10298000884225D100BF2E48806940F480502C49F0
:1029900088610846806900F48050019000BF00BF44
:1029A00000BF0846806940F00400886108468069DD
:1029B00000F00400019000BF00BFA02002900220A0
:1029C00003900320059002A91E48FEF711FE33E094
:1029D0001D49206888422FD100BF1948C06940F4C2
:1029E00080401749C8610846C06900F480400190E2
:1029F00000BF00BF00BF0846806940F00800886142
:102A00000846806900F00800019000BF00BF4FF445
:102A100020400290022003900320059002A90B4859
:102A2000FEF7E6FD4FF480400290002003900490F2
:102A300002A90648FEF7DCFD06B010BD00300140DB
:102A4000001002400008014000380040000C014026
:102A50007047704730B502460B4600BF92F83C0005
:102A6000012801D1022030BD012082F83C0000BFC6
:102A7000022082F83D00106844681068816824F0E4
:102A800070041868044310684460144D1068A8422C
:102A900013D0134D1068A8420FD01068B0F1804FCA
:102AA0000BD0104D1068A84207D00F4D1068A842F7
:102AB00003D00E4D1068A84205D121F0800158685E
:102AC000014310688160012082F83D0000BF0020B2
:102AD00082F83C0000BF00BFC5E70000002C0140A9
:102AE000003401400004004000080040000C004099
:102AF00010B504460CB9012010BD94F83D0028B96A
:102B0000002084F83C00204600F026F8022084F8DB
:102B10003D00211D206803F05FFE012084F846007F
:102B200000BF84F83E0001213F200155402001559F
:102B30004120015500BF00BF012084F8420043201E
:102B40000155442001554520015500BF012084F85E
:102B50003D000020D0E7000038B504462068B0F101
:102B6000804F16D100BF1848C06940F001001649D7
:102B7000C8610846C06900F00100009000BF00BFB6
:102B8000002205211C20FEF7A1FF1C20FEF78EFF6E
:102B900019E00E492068884215D100BF0A48C06973
:102BA00040F002000849C8610846C06900F0020010
:102BB000009000BF00BF002205211D20FEF786FF08
:102BC0001D20FEF773FF38BD0010024000040040D6
:102BD000014691F83D00012801D0012070470220F4
:102BE00081F83D000868C06840F001000B68D860BB
:102BF000164B0868984213D0154B086898420FD0BE
:102C00000868B0F1804F0BD0124B0868984207D08B
:102C1000114B0868984203D0104B086898420CD1B9
:102C20000868806800F00702062A0CD0086800686F
:102C300040F001000B68186005E00868006840F08B
:102C400001000B6818600020C8E70000002C01405C
:102C5000003401400004004000080040000C004027
:102C60002DE9F04104460D4600BF94F83C000128D0
:102C700002D10220BDE8F081012084F83C0000BFB1
:102C8000022084F83D002068866826F0770626F446
:102C90007F46206886602868502833D00CDC2028C6
:102CA00050D004DC00284BD0102851D149E0302806
:102CB00049D040284CD139E060282DD0702807D069
:102CC000B0F5805F03D0B0F5005F41D10DE040E08A
:102CD000D5E902136A68206803F0CCFD2068866895
:102CE00046F077062068866033E0D5E902136A680B
:102CF000206803F0BFFD2068806840F480402168B0
:102D0000886026E0EA686968206803F0C7FD502102
:102D1000206803F0BAFD1CE0EA686968206803F0E7
:102D2000D0FD6021206803F0B0FD12E0EA68696818
:102D3000206803F0B3FD4021206803F0A6FD08E001
:102D400000BF00BF00BF2968206803F09EFD00E0BF
:102D500000BF00BF012084F83D0000BF002084F8C0
:102D60003C0000BF00BF85E7704710B504462068EF
:102D70000069C0F34000D8B12068C068C0F34000CB
:102D8000B0B16FF00200216808610120207720684F
:102D9000806900F0030018B12046FFF7E5FF05E069
:102DA000204600F0ADF8204600F0ABF80020207778
:102DB00020680069C0F38000D8B12068C068C0F303
:102DC0008000B0B16FF00400216808610220207714
:102DD0002068806900F4407018B12046FFF7C4FFF6
:102DE00005E0204600F08CF8204600F08AF800202C
:102DF000207720680069C0F3C000D8B12068C0689F
:102E0000C0F3C000B0B16FF0080021680861042071
:102E100020772068C06900F0030018B12046FFF752
:102E2000A3FF05E0204600F06BF8204600F069F8AB
:102E30000020207720680069C0F30010D8B1206816
:102E4000C068C0F30010B0B16FF0100021680861D5
:102E5000082020772068C06900F4407018B120462F
:102E6000FFF782FF05E0204600F04AF8204600F018
:102E700048F8002020772068006900F0010058B170
:102E80002068C06800F0010030B16FF001002168D7
:102E90000861204600F036F820680069C0F3C010D1
:102EA00058B12068C068C0F3C01030B16FF0800026
:102EB000216808612046FFF7CBFD20680069C0F358
:102EC000801058B12068C068C0F3801030B16FF036
:102ED000400021680861204600F02EF82068006953
:102EE000C0F3401058B12068C068C0F3401030B142
:102EF0006FF02000216808612046FFF7AAFD10BD91
:102F00007047704710B5044608492068884201D1CF
:102F1000FEF72CFD00BF06480068B0F1804F03D1DA
:102F200001210448FEF70CFD00BF10BD002C01403C
:102F3000C0230020001001407047704770B5044660
:102F4000002520684069C0F3C01594F83D00212891
:102F50000ED16DB12068406920F080002168486181
:102F6000606B10B1606BFDF7FEFE204603F0EFFDD5
:102F700020684069C0F3801594F83E0022280ED1E5
:102F80006DB12068406920F0400021684861A06B65
:102F900010B1A06BFDF7E7FE204603F0ADFD002069
:102FA00070BD70472DE9F84F044620680568206819
:102FB000C668206847694FF00009CA4605F00F0946
:102FC000B9F1000F0AD105F0200038B106F0200059
:102FD00020B1204603F0C5FDBDE8F88FB9F1000F20
:102FE00071D007F0010018B906F4907000286AD07B
:102FF00005F0010030B106F4807018B1206C40F08B
:103000000100206405F0040030B107F0010018B1A0
:10301000206C40F00200206405F0020030B107F09F
:10302000010018B1206C40F00400206405F0080095
:1030300048B106F0200010B907F0010018B1206C6B
:1030400040F008002064206C68B305F0200028B12F
:1030500006F0200010B1204603F083FD206840698F
:10306000C0F3801A206C00F0080010B9BAF1000F0C
:1030700022D0204603F040FD2068406900F0400067
:10308000B0B12068406920F0400021684861A06B21
:1030900050B15648A16B4863A06BFDF78FFE10B18D
:1030A000A06B416B88470CE02046FFF77AFF08E0F1
:1030B0002046FFF776FF04E02046FFF772FF00206E
:1030C000206489E7FFE7206B012878D105F0100024
:1030D000002874D006F01000002870D000BF002037
:1030E000009020680068009020684068009000BF51
:1030F00000BF2068406900F04000C0B3A06B0068CA
:1031000040681FFA80F8B8F1000F2FD0A08D40451D
:103110002CDDA4F82E80A06B806920281FD02068A9
:10312000C06820F480702168C8602068406920F081
:103130000100216848612068406920F04000216852
:103140004861202084F83E00002020632068C06889
:1031500020F010002168C860A06BFDF704FEA08D70
:10316000E28D801A81B22046FFF7E7FE34E7FFE7E1
:10317000A08DE18D401A1FFA80F8E08DE8B1B8F11A
:10318000000F1AD02068C06820F490702168C860D1
:103190002068406920F0010021684861202084F8FF
:1031A0003E00002020632068C06820F010002168E5
:1031B000C86041462046FFF7C0FE0DE7FFE705F077
:1031C000800030B106F0800018B1204603F006FE02
:1031D00002E705F0400030B106F0400018B120468B
:1031E00003F0A5FCF8E600BFF6E600000D6A000853
:1031F00010B504460CB9012010BDA06900B100E073
:1032000000BF94F83D0028B9002084F83C00204617
:1032100000F028F8242084F83D002068C06820F4DD
:1032200000502168C860204603F00EFD2068006948
:1032300020F49040216808612068406920F02A004D
:10324000216848612068C06840F400502168C86067
:1032500000202064202084F83D0084F83E000020F7
:10326000CAE7000010B586B0044600200290039023
:1032700004900590FE49206888426AD100BFFD484D
:10328000C06940F40020FB49C8610846C06900F4E9
:103290000020019000BF00BF00BF0846806940F0D9
:1032A000100088610846806900F01000019000BF9E
:1032B00000BF08150290022003900320059002A988
:1032C000ED48FEF795F94FF400600290002003905E
:1032D000049002A9E848FEF78BF9E848E84908603D
:1032E000002048600021E64881608021C160002103
:1032F000016141618161C161FEF700F808B1FDF72C
:1033000075F900BFDE48A063446200BFDB48283087
:10331000DC490860102048600021DA488160802183
:10332000C1600021016141618161C161FDF7E6FF7A
:1033300008B1FDF75BF900BFD2486063446200BF8B
:10334000002205213420FEF7C1FB3420FEF7AEFB3E
:10335000BDE1CD492068884243D100BFC548C0695E
:1033600040F48010C349C8610846C06900F4801069
:10337000019000BF00BF00BF0846806940F0100008
:1033800088610846806900F01000019000BF00BF0E
:1033900000BF0846806940F02000886108468069C7
:1033A00000F02000019000BF00BF881402900220AE
:1033B00003900320059002A9AF48FEF719F90420F5
:1033C000029000200390049002A9B048FEF710F983
:1033D000002205213520FEF779FB3520FEF766FB3C
:1033E00075E1AB49206888426AD100BFA148806975
:1033F00040F480409F4988610846806900F480401D
:10340000019000BF00BF00BF0846806940F0040083
:1034100088610846806900F00400019000BF00BF89
:1034200048150290022003900320059002A99948B4
:10343000FEF7DEF84FF480600290002003900490C5
:1034400002A99448FEF7D4F89348944908600020F4
:1034500048600021914881608021C16000210161A4
:1034600041618161C161FDF749FF08B1FDF7BEF817
:1034700000BF8A48A063446200BF87481438884967
:103480000860102048600021854881608021C1606B
:103490000021016141618161C161FDF72FFF08B128
:1034A000FDF7A4F800BF7E486063446200BF0022BD
:1034B00005212520FEF70AFB2520FEF7F7FA06E195
:1034C0007849206888426AD100BF6A48C06940F4E0
:1034D00000306849C8610846C06900F400300190B6
:1034E00000BF00BF00BF0846806940F0040088614B
:1034F0000846806900F00400019000BF00BF04206E
:103500000290022003900320059002A96148FEF773
:103510006FF80820029000200390049002A95D48F3
:10352000FEF766F85C4814305F4908600020486088
:1035300000215D4881608021C160002101614161FD
:103540008161C161FDF7DAFE08B1FDF74FF800BFF8
:103550005548A063446200BF4F4828305349086073
:10356000102048600021514881608021C160002105
:10357000016141618161C161FDF7C0FE08B1FDF7E4
:1035800035F800BF49486063446200BF002205214E
:103590002620FEF79BFA2620FEF788FA97E044499A
:1035A000206888428BD100BF3248C06940F4802037
:1035B0003049C8610846C06900F48020019000BF0E
:1035C00000BF00BF0846806940F0080088610846D7
:1035D000806900F00800019000BF00BF081502904C
:1035E000022003900320059002A93248FEF700F85C
:1035F0004FF40060029000200390049002A92D482F
:10360000FDF7F6FF244828382B4908600020486061
:103610000021294881608021C16000210161416150
:103620008161C161FDF76AFE08B1FCF7DFFF00BFF1
:103630002148A063446200BF17483C381F49086016
:103640001020486000211D4881608021C160002158
:10365000016141618161C161FDF750FE08B1FCF774
:10366000C5FF00BF15486063446200BF002227E029
:10367000004C0040001002400010014030040240A5
:10368000A42D0020E82D002000500040001401402F
:103690000038014000080140580002402C2E002054
:1036A000702E002000440040B42E0020F82E002090
:1036B00000480040000C01403C2F0020802F0020DB
:1036C00005212720FEF702FA2720FEF7EFF906B0C2
:1036D00010BD70B504460D46164694F83E002028ED
:1036E00016D105B10EB9012070BD00BF94F83C00A1
:1036F000012801D10220F7E7012084F83C0000BF37
:103700000020206332462946204603F01BFBEBE7EE
:103710000220E9E7704770472DE9F84F04460E464E
:10372000174699464FF0000A94F83D0020285AD1D8
:1037300006B117B90120BDE8F88F00BF94F83C002E
:10374000012801D10220F6E7012084F83C0000BFE7
:1037500000202064212084F83D00FEF701F9824614
:10376000A784E784A068B0F5805F04D1206910B910
:103770000025B04602E035464FF0000800BF0020AB
:1037800084F83C0000BF1BE0534600228021204605
:10379000CDF8009003F052FB08B10320CBE745B908
:1037A000B8F80000C0F308002168486008F102087A
:1037B00003E02878216848606D1CE08C401EE0849E
:1037C000E08C0028E0D15346002240212046CDF86D
:1037D000009003F033FB08B10320ACE7202084F80D
:1037E0003D000020A7E70220A5E7704700BFFEE7E5
:1037F0000FB400B58FB06148007820B102F0C4F971
:1038000000205E4908709DF84000062856D006DC6E
:1038100006281DD2DFE800F0101D2C415051A128D0
:103820007AD004DC07284AD0A02811D163E0A2286E
:1038300071D0BB28F9D18DE05148007800905149F2
:103840000B7851490A7851490978119803F08EFE96
:103850008FE0FEF785F84E490968401A42F2107170
:10386000884202D301204B49087006F02DFB80E00E
:10387000FEF776F846490968401A42F2107188420C
:1038800002D30120434908709DF8410010B903F0AC
:103890009BFD6EE000F0F2FE6BE0FEF761F83C4944
:1038A0000968401A42F21071884202D30120394956
:1038B000087007F08DFA5CE000BF00BF00BFFEF7A4
:1038C0004FF833490968401A44F62061884208D30A
:1038D00001231A4630A132A007F0E0F901202D495A
:1038E00008703C2214A96846FCF79CFC10A80FC87D
:1038F00007F018FD3DE0FEF733F825490968401A46
:1039000042F21071884202D301202249087001F06E
:1039100041FD2EE000E00EE0FEF722F81C490968A8
:10392000401A42F21071884202D3012019490870EE
:1039300001F07CFD1DE0FEF713F815490968401AF7
:1039400042F21071884202D301201249087001F03E
:1039500007FF0EE0FEF704F80D490968401A42F22D
:103960001071884202D301200A49087003F000FB5D
:1039700000BF00BF0FB05DF814FB0000F500002091
:10398000F9000020F8000020F7000020F6000020D9
:10399000C4020020FA0000204552524F520000009D
:1039A00041542B444953434F4E4E3D300D0A0000C5
:1039B00010B508217948FDF7BBFF79490870084622
:1039C000007878490978884208D0754800787549A8
:1039D0000870FDF7C5FF74490860DCE0FDF7C0FF23
:1039E00071490968401A1E28F7D96D4800780028E7
:1039F0006FD16E48007800286CD1FDF7B1FF6C499B
:103A000008606C480078052866D006DC05281CD2C2
:103A1000DFE800F0101C29446100A0285FD004DC1E
:103A200006285AD0072810D158E0A12873D0A22820
:103A3000F9D18BE000BF00205E49087048708870A3
:103A4000C87001205C49087000BF9AE000BF0120E7
:103A5000584908704870002088700120C870564985
:103A6000087000BF8DE053484078042809D05148C1
:103A70004078401C4F49487008468078401E887046
:103A800008E04C484078042804D100204949487097
:103A90000420887001204849087072E04548407849
:103AA000032809D043484078401C424948700846E2
:103AB0008078401E887008E03E484078032804D192
:103AC00000203C4948700320887001203A49087062
:103AD00057E05CE059E000BF00BF00BF00BF3548C1
:103AE0004078012809D033484078401C314948705B
:103AF00008468078401E887008E02E4840780128EB
:103B000004D100202B4948700120887001202A49E7
:103B1000087036E0FFE7274840780E2809D025488E
:103B20004078401C2349487008468078401E8870C1
:103B300008E0204840780E2804D100201D49487034
:103B40000E20887001201C4908701AE0194840783E
:103B50000F2809D017484078401C1649487008467D
:103B60008078401E887008E0124840780F2804D101
:103B70000020104948700F20887001200E490870FD
:103B800000BF00BF012009490870012010BD0020BE
:103B900006490870FAE70020F8E70000000C014031
:103BA000A8060020A9060020AC060020A0020020E4
:103BB000C402002098070020F500002010B5102155
:103BC0007748FDF7B5FE77490870084600787649D2
:103BD0000978884208D07348007873490870FDF767
:103BE000BFFE72490860D8E0FDF7BAFE6F49096868
:103BF000401A1E28F7D96B48007800287ED16C48FF
:103C0000007800287BD1FDF7ABFE6A4908606A485E
:103C10000078052862D006DC05281CD2DFE800F019
:103C2000101C29435D00A0285BD004DC062856D078
:103C3000072810D154E0A12871D0A228F9D188E03A
:103C400000BF00205C49087048708870C87001206F
:103C50005A49087000BF96E000BF0120564908701D
:103C60000020487001208870C8705449087000BF57
:103C700089E051488078042809D04F484078401E98
:103C80004D49487008468078401C887007E04A48D3
:103C90008078042803D148494870002088700120AA
:103CA000464908706FE044488078032809D04248AC
:103CB0004078401E4049487008468078401C887013
:103CC00007E03D488078032803D13B494870002035
:103CD000887001203949087055E000BF00BF00BF5F
:103CE00000BF3548807801280CD033484078401E0A
:103CF0003149487008468078401C01E049E046E0C0
:103D0000887007E02C488078012803D12A49487040
:103D10000020887001202949087034E0FFE7264818
:103D200080780E2809D024484078401E22494870E7
:103D300008468078401C887007E01F4880780E286D
:103D400003D11D4948700020887001201B4908706C
:103D500019E0194880780F2809D017484078401E8C
:103D60001549487008468078401C887007E0124862
:103D700080780F2803D110494870002088700120F6
:103D80000E49087000BF00BF0120094908700120DA
:103D900010BD002006490870FAE70020F8E700008F
:103DA000000C0140B0060020B1060020B40600203F
:103DB000A1020020C402002098070020F500002086
:103DC00010B52021FE48FDF7B3FDFE4908700846F6
:103DD0000078FD490978884208D0FA480078FA4905
:103DE0000870FDF7BDFDF94908609FE2FDF7B8FDD9
:103DF000F6490968401A1E28F7D9F24800780028C9
:103E000076D1F3480078002873D1FDF7A9FDF14978
:103E10000860F148007805286CD006DC05281DD222
:103E2000DFE800F0101D4169E100A0287ED004DC2D
:103E300006287CD0072811D1D8E0A12878D0A22864
:103E4000F9D1FCE000BF0120E34908704870002070
:103E500088700120C870E149087000BF5CE2DE484C
:103E6000407801280FD106F03FFE00BF0220DA495A
:103E7000087004204870002088700220C87001205B
:103E8000D64908700EE006F02FFE00BF0320D2498D
:103E900008704870002088700220C8700120CF4947
:103EA000087000BF38E2CC48407870B9FCF7D0FA0F
:103EB00000BF0120C84908704870002088700120A8
:103EC000C870C649087000BF26E2C3488078C2495E
:103ED00081F8480000BFA020087001204870002031
:103EE00088700320C8700120BC49087000BF13E22D
:103EF00018E215E278E0B848407803281CD1B64AA9
:103F0000D168032390681A4606F0C8FE6420FDF7C6
:103F100089FA00BF0420B0490870012048700020D1
:103F200088700320C8700120AC4902E062E05CE0C8
:103F300084E0087000BFEFE1A7484078022818D15C
:103F4000A54AD169032390691A4606F0A7FE6420AA
:103F5000FDF768FA00BF05209F49087001204870EE
:103F6000002088700320C87001209C49087000BFA1
:103F7000D2E199484078012818D1974AD16A0323A1
:103F8000906A1A4606F08AFE6420FDF74BFA00BFDD
:103F90000620914908700120487000208870032095
:103FA000C87001208D49087000BFB5E18A4840788B
:103FB000C0B9894AD16B0323906B1A4606F06EFE96
:103FC0006420FDF72FFA00BF072083490870012005
:103FD0004870002088700320C87001207F49087055
:103FE00000BF99E100BF00BF00BF00BF04207A49B5
:103FF000C87091E17848407801280DD100BFA12018
:10400000754908700E204870002088700320C87021
:1040100001207249087010E06F48407868B900BF0D
:10402000A2206D4908700F2048700020887003207E
:10403000C87001206949087000BF6DE100BF664883
:1040400090F8480030BB64480078A22823D00024B0
:104050001EE061488078A04219D1614800EB04104D
:1040600000685D4988605E4800EB04104068C860E5
:104070005B4800EB041080680861594800EB0410AD
:104080008189584803F04AF8012057490870641C98
:104090001F2CDED323E000241FE04F4880780F3030
:1040A000A04219D14E4800EB041000684A498860CC
:1040B0004B4800EB04104068C860494800EB04100E
:1040C00080680861464800EB04108189454803F088
:1040D00025F8012044490870641C1F2CDDD33E489C
:1040E00090F8480001284BD13B480078A22823D003
:1040F00000241EE038488078A04219D1384800EBEF
:104100000410006834498861354800EB04104068A9
:10411000C861334800EB041080680862304800EB47
:1041200004108189314802F0F9FF012030490870FC
:10413000641C1F2CDED323E000241FE02648807877
:104140000F30A04219D1264800EB04100068224924
:104150008861234800EB04104068C861204800EBE8
:104160000410806808621E4800EB041081891F4813
:1041700002F0D4FF01201E490870641C1F2CDDD3FF
:10418000154890F84800022866D113480078A22804
:104190003ED0002439E010488078A04234D1104845
:1041A00000EB041000680C4988620D4800EB041015
:1041B0004068C8620A4800EB04108068086319E090
:1041C000000C0140B8060020B9060020BC06002003
:1041D000A2020020C402002098070020F500002061
:1041E000C802002000600708F600002000680708E9
:1041F000F70000204E4800EB041081894D4802F082
:104200008DFF01204C490870641C1F2CC3D323E090
:1042100000241FE0494880780F30A04219D144485B
:1042200000EB0410006845498862414800EB041027
:104230004068C8623E4800EB0410806808633C4850
:1042400000EB041081893B4802F068FF01203A49E5
:104250000870641C1F2CDDD3384890F848000328F0
:104260004BD136480078A22823D000241EE03348E2
:104270008078A04219D12E4800EB041000682F4925
:1042800088632B4800EB04104068C863284800EBA3
:10429000041080680864264800EB041081892848CF
:1042A00002F03CFF012027490870641C1F2CDED35C
:1042B00023E000241FE0214880780F30A04219D16C
:1042C0001B4800EB041000681C498863184800EB89
:1042D00004104068C863164800EB04108068086446
:1042E000134800EB04108189154802F017FF0120E4
:1042F00014490870641C1F2CDDD300BF02200F4935
:10430000087004204870002088700220C8700120C6
:104310000D49087000BF00BF00BF01200B490870A5
:10432000012010BD002009490870FAE70020F8E7D5
:10433000C802002000770708F80000209807002036
:1043400000780708F9000020F5000020A2020020F4
:1043500010B540216A48FDF7EBFA6A490870084633
:10436000007869490978884208D06648007866492B
:104370000870FDF7F5FA65490860BEE0FDF7F0FA50
:1043800062490968401A1E28F7D95E48007800285B
:104390006FD1FDF7E5FA5E4908605E4800780028B5
:1043A00068D15D480078052834D006DC05281FD286
:1043B000DFE800F010111F202F00A0285BD004DCE4
:1043C000062828D0072813D126E0A12862D0A228E9
:1043D000F9D160E000BF06F087FB00BF00204E4926
:1043E000087048708870C87001204C49087000BF80
:1043F00079E000BF06F078FB00BF01204649087055
:104400004870002088700120C8704449087000BFBF
:1044100069E000BF00BF00BF01231A4640A142A0CF
:1044200006F03CFC1E20FCF7FDFF434806F056FB5F
:1044300042490880424806F051FB42490880424800
:1044400006F04CFB41490880414806F047FB4149D2
:10445000088006F049FB00BF03202F490870487010
:10446000002088700220C87001202C49087000BF0D
:1044700039E03EE03BE000BF0220274908700420FD
:104480004870002088700220C870012023490870FD
:1044900000BF28E000BF284806F020FB274908801D
:1044A000274806F01BFB27490880274806F016FB23
:1044B00026490880264806F011FB264908801E2060
:1044C000FCF7B0FF06F010FB00BFA02012490870F7
:1044D00001204870002088700320C87001200F4917
:1044E000087000BF00BF00BF01200A49087001200A
:1044F00010BD002007490870FAE70020F8E7000027
:10450000000C0140C0060020C1060020C4060020A7
:10451000C4020020A302002098070020F50000201C
:104520004552524F5200000041542B444953434FCF
:104530004E4E3D300D0A000000000708BA02002070
:1045400000100708BC02002000200708BE0200205F
:1045500000300708C002002078B502460C46002053
:1045600020E0002505EB8005655D002606EB800652
:104570009555012505EB8005655D012606EB800656
:104580009555022505EB8005655D022606EB800644
:104590009555032505EB8005655D032606EB800632
:1045A0009555401C0428DCD304205FE0451EA9007B
:1045B000555C8DF800504D1C555D8DF801508D1CDB
:1045C000555D8DF80250CD1C555D8DF8035000F0FF
:1045D00003056DBB9DF800509DF801608DF80060EB
:1045E0009DF802608DF801609DF803608DF802600F
:1045F0008DF803509DF800501E4E755D8DF80050EB
:104600009DF80150755D8DF801509DF80250755D63
:104610008DF802509DF80350755D8DF803509DF89C
:104620000050154E06EB9006367875408DF8005018
:104630008300051FA900555C9DF800607540D554A6
:104640004D1C555D9DF8016075405E1C95558D1C97
:10465000555D9DF8026075409E1C9555CD1C555DBD
:104660009DF803607540DE1C9555401C2C289DD399
:1046700078BD000090E3000890E5000808B501202F
:10468000102350A202210090142001F058FD0120B7
:104690000E23102202210090372001F03DFC012062
:1046A0000E231122022100904B2001F035FC012045
:1046B000102345A211210090142001F040FD01209B
:1046C0000E23102211210090372001F025FC01203B
:1046D0000E231122114600904B2001F01DFC0120F9
:1046E00010233AA220210090142001F028FD01207F
:1046F0000E23102220210090372001F00DFC012014
:104700000E231122202100904B2001F005FC0120F6
:1047100010232FA22F210090142001F010FD012062
:104720000E2310222F210090372001F0F5FB0120ED
:104730000E2311222F2100904B2001F0EDFB254884
:10474000407804280BD12348807840B900201023FA
:1047500021A202210090642001F0F1FC31E01D480B
:10476000407803280CD11B488078012808D100200C
:10477000102319A211210090642001F0E0FC20E038
:104780001448407802280CD112488078022808D1B9
:104790000020102310A220210090642001F0CFFC03
:1047A0000FE00C48407801280BD10A488078032894
:1047B00007D10020102308A22F210090642001F0CF
:1047C000BEFC08BD4C2031004C2032004C20330090
:1047D0004C203400980700203C2D2D0010B50C48CB
:1047E0000078401C0A4908700AA002F0D5FC00229B
:1047F0004FF400410A48FDF7ADF84FF47A60FCF73A
:1048000011FE0120074908700749087010BD00001B
:10481000C806002042742072657365740D0A00009A
:1048200000080140CC060020D006002010B5494801
:1048300049490861FF2008764848017848A002F0FD
:10484000ABFC01F03FFE01231A464BA14CA006F041
:1048500025FA10B14EA002F09FFC514800780528BF
:1048600070D2DFE800F003041F3A55006AE001232C
:104870001A464CA14EA006F011FA78B101231A464F
:104880004EA14FA006F00AFA58B151A002F084FCE4
:1048900043480078401C4249087002E0FFF79EFF41
:1048A00050E000BF01231A464EA151A006F0F6F9D0
:1048B00078B101231A4641A150A006F0EFF958B192
:1048C00052A002F069FC36480078401C3449087058
:1048D00002E0FFF783FF35E000BF01231A4650A135
:1048E00052A006F0DBF978B101231A4633A152A099
:1048F00006F0D4F958B154A002F04EFC28480078D4
:10490000401C2749087002E0FFF768FF1AE000BF6B
:1049100001231A4651A154A006F0C0F978B1012331
:104920001A4626A154A006F0B9F958B156A002F0D3
:1049300033FC1B480078401C1949087002E0FFF75F
:104940004DFF00BF00BF00205549087001205549A8
:10495000087010BD31757464640C0020C806002016
:104960000923232330310942545F696E6974256439
:104970002E2E2E0D0A0000004552524F520000000C
:1049800041542B444953434F4E4E3D300D0A0000D5
:1049900023D2D1CEDEC9E8B1B8C1ACBDD30A000084
:1049A000CC0600202B55554944533A464646300024
:1049B00041542B55554944533F0D0A004F4B0000BD
:1049C00041542B55554944533D303030320D0A0087
:1049D000233031C9E8D6C3D6F7B7FECEF1B3C9B993
:1049E000A60A00002B555549444E3A46464631002A
:1049F00041542B555549444E3F0D0A0041542B5507
:104A00005549444E3D464630340D0A00233032C9E4
:104A1000E8D6C3B6C1B7FECEF1B3C9B9A60A000045
:104A20002B55554944573A464646320041542B557A
:104A3000554944573F0D0A0041542B555549445799
:104A40003D464646350D0A00233033C9E8D6C3D06B
:104A5000B4B7FECEF1B3C9B9A60A00002B54585022
:104A60004F5745523A30000041542B5458504F573D
:104A700045523F0D0A00000041542B5458504F57E7
:104A800045523D31300D0A00233034C9E8D6C3B752
:104A9000A2C9E4B9A6C2CAB3C9B9A60A00000000F7
:104AA00098070020F500002010B501200C4908707F
:104AB0000C480078401C0B4908700BA002F06CFBFE
:104AC000002202210D48FCF745FF41F28830FCF737
:104AD000A9FC012202210948FCF73CFF10BD00009F
:104AE000200700201D0700203447204D6F64756C9F
:104AF000655F52657365740A00000000000801409C
:104B000008B53248017832A002F046FB36A1394898
:104B1000FBF7ACFB002856D00F213648FBF79BFB78
:104B200035A002F039FB9620FCF77CFC01231A46E5
:104B300034A135A006F078F828B90120344908706E
:104B400034A002F029FB3248007818B135A002F0F9
:104B500023FB3AE001231A4637A13BA006F064F894
:104B600058B13CA002F018FB00200C2340A23221D7
:104B700000902A2001F0E3FA27E0C820FCF752FC5D
:104B800001231A463DA130A006F04EF858B13FA0CF
:104B900002F002FB00200C2341A22D2100902320D3
:104BA00001F0CDFA11E001231A4640A141A006F020
:104BB0003BF801231A463DA141A006F035F843A079
:104BC00002F0EAFA01E0FFF76FFF08BD1D070020C1
:104BD0000923232330320934475F696E69742564E1
:104BE0002E2E2E0D0A0000002B4D415452454144FB
:104BF00059000000CC380020233447C4A3BFE9C9C2
:104C0000CFB5E7004F4B000041540D0A00000000F3
:104C10001F0700203447C4A3D7E9D2ECB3A3A3A154
:104C20000D0A0000233447C4A3BFE9B3F5CABCBBD7
:104C3000AF4661696C0000002B434D452045525240
:104C40004F523A203130000041542B4350494E3FDF
:104C50000D0A0000094552524F52212D2D3ECEB46F
:104C6000BCECB2E2B5BD53494DBFA80D0A0000002F
:104C7000204E4F5F53494D20000000002B434D450F
:104C8000204552524F523A203133000009455252CA
:104C90004F52212D2D3E53494DCAA7B0DC0D0A00BD
:104CA0002053494D5F4661696C2000004552524FC8
:104CB0005200000041542B4353510D0A00000000E4
:104CC00041542B43455245473F0D0A00696E6974B4
:104CD0005F737563636573730D0A000000B58BB075
:104CE00019481A490860042048600021174881606B
:104CF000C1604FF4A02101614FF480114161002196
:104D0000017641768176C17601774177FBF7D1FE56
:104D100008B1FBF76BFC002006900790012008907B
:104D200000200190029003900490059001200990CA
:104D30000E200A9001A90548FBF70EFD0348FBF77A
:104D4000DCFF0BB000BD000000640040D422002056
:104D500008B500BF2D48406940F001002B4948616B
:104D60000846406900F00100009000BF00BF00BF8E
:104D70000846406940F0020048610846406900F07A
:104D80000200009000BF00BF002205210C20FCF7AC
:104D90009DFE0C20FCF78AFE002205210D20FCF769
:104DA00095FE0D20FCF782FE002205210E20FCF767
:104DB0008DFE0E20FCF77AFE002205210F20FCF765
:104DC00085FE0F20FCF772FE002205211020FCF763
:104DD0007DFE1020FCF76AFE002205211120FCF761
:104DE00075FE1120FCF762FE002205213A20FCF737
:104DF0006DFE3A20FCF75AFE002205213B20FCF70D
:104E000065FE3B20FCF752FE08BD0000001002408A
:104E100000B59DB01C22184916A8FBF703FA002123
:104E200016A805F09AFA154908601C2212491C318F
:104E30000FA8FBF7F7F900210FA805F08EFA10492B
:104E400008601C220C49383108A8FBF7EBF9002157
:104E500008A805F082FA0B4908601C220649543163
:104E600001A8FBF7DFF9002101A805F076FA064951
:104E700008601DB000BD000020E30008040700200A
:104E8000080700200C0700201007002000B585B09F
:104E90000020019002900390049000BF3D4880697B
:104EA00040F010003B4988610846806900F010001E
:104EB000009000BF00BF00BF0846806940F020009E
:104EC00088610846806900F02000009000BF00BFA4
:104ED00000BF0846806940F0040088610846806988
:104EE00000F00400009000BF00BF00BF08468069CA
:104EF00040F0080088610846806900F008000090D2
:104F000000BF00BF002240F211212348FCF722FD20
:104F1000012248F212012148FCF71CFD0022402129
:104F20001E48FCF717FD012280211B48FCF712FDEB
:104F300040F2912001900120029000200390022075
:104F4000049001A91448FCF753FB48F24200019079
:104F500001200290002003900220049001A90F4834
:104F6000FCF746FB102001900120029000200390E6
:104F70000320049001A90948FCF73AFB782001902E
:104F8000002002900120039001A90548FCF730FBA6
:104F900005B000BD001002400010014000080140B3
:104FA000000C01401FB500200290019000BF564840
:104FB000C06940F000605449C8610846C06900F00B
:104FC0000060009000BF00BF00BF0846C06940F00D
:104FD0008050C8610846C06900F08050009000BF52
:104FE00000BF4A484A4908604FF0FF30486000213E
:104FF00047488160FDF7C0FA08B1FBF7F7FA0121D5
:105000004348FDF777FA45F2510188424CD013200E
:105010008DF8080000208DF809008DF80A000122A3
:1050200002A93B48FDF7B4FB08B1FBF7DFFA042007
:105030008DF8040001208DF8050018208DF8060079
:1050400023208DF80700012201A93148FDF724FB38
:1050500008B1FBF7CBFA2E480068006840F0010069
:105060002B49096808600198039045F2510201211B
:105070002748FDF74BFA9DF80F2002212448FDF741
:1050800045FA9DF80D2003212148FDF73FFA9DF8D0
:105090000E2004211E48FDF739FA9DF80C20052149
:1050A0001B48FDF733FA2DE002211948FDF722FADB
:1050B000C0B28DF80F0003211548FDF71BFAC0B2EE
:1050C0008DF80D0004211248FDF714FAC0B28DF8D6
:1050D0000E0005210E48FDF70DFAC0B28DF80C0048
:1050E00003980190002201A90948FDF7D5FA08B1FB
:1050F000FBF77CFA06480068006840F001000449AC
:10510000096808601FBD0000001002400028004030
:10511000FC22002010B50F480F4908604FF4827040
:1051200048604FF400410C4881600021C16001617A
:1051300041614FF4007181610821C1610021016268
:10514000416281620A21C162FDF7B0FB08B1FBF741
:105150004DFA10BD003001401023002010B50E485C
:105160000E4908604FF48270486000210B4881604E
:10517000C160016141614FF4007181610021C16131
:105180000162416281620A21C162FDF78FFB08B1B1
:10519000FBF72CFA10BD0000003800406823002007
:1051A00000B587B000200390049005900690019010
:1051B00002904FF0804014490860092048600021A7
:1051C0001148816041F63F71C16000210161816138
:1051D000FDF78EFC08B1FBF709FA4FF480500390FD
:1051E00003A90948FDF73CFD08B1FBF7FFF90020D2
:1051F0000190029001A90448FDF72CFC08B1FBF7CF
:10520000F5F907B000BD0000C023002000B587B04D
:10521000002003900490059006900190029015489C
:105220001549086041F287304860002112488160CA
:1052300041F63F71C160002101618161FDF758FCB9
:1052400008B1FBF7D3F94FF48050039003A90A4843
:10525000FDF706FD08B1FBF7C9F9002001900290A7
:1052600001A90548FDF7F6FB08B1FBF7BFF907B048
:1052700000BD0000000400400824002010B50B48C9
:105280000B4908604FF4E130486000210848816014
:10529000C16001610C21416100218161C161FDF7A3
:1052A000A7FF08B1FBF7A2F910BD0000004C0040B9
:1052B000502C002010B50B480B4908604FF4E1302A
:1052C0004860002108488160C16001610C21416192
:1052D00000218161C161FDF78BFF08B1FBF786F901
:1052E00010BD000000500040942C002010B50B4869
:1052F0000B4908604FF4E1304860002108488160A4
:10530000C16001610C21416100218161C161FDF732
:105310006FFF08B1FBF76AF910BD000000380140CB
:10532000D82C002010B50B480B4908604FF4E13031
:105330004860002108488160C16001610C21416121
:1053400000218161C161FDF753FF08B1FBF74EF900
:1053500010BD0000004400401C2D002010B50B487B
:105360000B4908604FF4E130486000210848816033
:10537000C16001610C21416100218161C161FDF7C2
:1053800037FF08B1FBF732F910BD000000480040BC
:10539000602D002008B50020102316A201460090C1
:1053A000082000F0CCFE0120102316A2142100904A
:1053B000002000F0C4FE0120102316A2232100903B
:1053C000002000F0BCFE17484078012808D10020DA
:1053D000102315A2142100906E2000F0B0FE07E00B
:1053E0000020102310A2232100906E2000F0A7FEC1
:1053F00008BD00003E204D6163536C6963696E67B0
:10540000203C00004D41433A303030312D303030B7
:10541000460000004D41433A303031302D303031BC
:1054200046000000980700203C2D000008B5012030
:105430001023B8A200210090084600F080FE012051
:105440001023B4A20F210090002000F078FE01206C
:105450001023B0A21E210090002000F070FE012059
:105460001023ACA22D210090002000F068FEAB4874
:10547000807803284FDC01201023A94A00210090E6
:10548000202000F05CFE01201023A64A0F2100908E
:10549000202000F054FE01201023A34A1E2100907A
:1054A000202000F04CFE01201023A04A2D21009066
:1054B000202000F044FE9948807838B9002010235D
:1054C000974A01460090202000F039FE93488078EA
:1054D000012807D100201023924A0F21009020209C
:1054E00000F02DFE8D488078022807D1002010237F
:1054F0008D4A1E210090202000F021FE87488078F0
:10550000032807D100201023884A2D210090202055
:1055100000F015FEFDE081488078032854DD7F48C7
:105520008078072850DC01201023814A0021009058
:10553000202000F004FE012010237E4A0F2100905D
:10554000202000F0FCFD012010237B4A1E2100904A
:10555000202000F0F4FD01201023784A2D21009036
:10556000202000F0ECFD6D488078042807D1002051
:1055700010236F4A01460090202000F0E0FD6748AC
:105580008078052807D1002010236A4A0F21009057
:10559000202000F0D4FD61488078062807D1002043
:1055A0001023654A1E210090202000F0C8FD5B48B2
:1055B00080780728AED100201023604A2D2100906A
:1055C000202000F0BCFDA4E054488078072854DD7A
:1055D000524880780B2850DC01201023584A0021C3
:1055E0000090202000F0ABFD01201023554A0F2130
:1055F0000090202000F0A3FD01201023524A1E211C
:105600000090202000F09BFD012010234F4A2D2107
:105610000090202000F093FD40488078082807D1B2
:1056200000201023464A01460090202000F087FD0C
:105630003A488078092807D100201023414A0F21D9
:105640000090202000F07BFD344880780A2807D1A4
:10565000002010233C4A1E210090202000F06FFD06
:105660002E4880780B2854D100201023374A2D2152
:105670000090202000F063FD4BE0284880780B2844
:1056800047DD264880780E2843DC01201023304A6D
:1056900000210090202000F052FD012010232D4A0F
:1056A0000F210090202000F04AFD012010232A4AFB
:1056B0001E210090202000F042FD01201023274AE7
:1056C0002D210090202000F03AFD144880780C280D
:1056D00007D1002010231E4A01460090202000F030
:1056E0002EFD0E4880780D2807D100201023194A7E
:1056F0000F210090202000F022FD084880780E281D
:1057000007D100201023144A1E210090202000F011
:1057100016FD08BD4D41433A0000000098070020E7
:10572000FB000020080100201501002022010020BC
:105730002F0100203C0100204901002056010020DB
:1057400063010020700100207D0100208A010020FB
:1057500097010020A4010020B1010020BE0100201B
:1057600008B501201023BEA200210090084600F0D9
:10577000E6FC01201023BAA20F210090002000F0C7
:10578000DEFC01201023B6A21E210090002000F0B4
:10579000D6FC01201023B2A22D210090002000F0A1
:1057A000CEFCB148807803284FDC01201023AF4A9B
:1057B00000210090202000F0C2FC01201023AC4A00
:1057C0000F210090202000F0BAFC01201023A94AEC
:1057D0001E210090202000F0B2FC01201023A64AD8
:1057E0002D210090202000F0AAFC9F48807838B935
:1057F000002010239D4A01460090202000F09FFCCD
:1058000099488078012807D100201023984A0F2159
:105810000090202000F093FC93488078022807D164
:1058200000201023934A1E210090202000F087FCC6
:105830008D488078032807D1002010238E4A2D211F
:105840000090202000F07BFC09E187488078032845
:1058500054DD85488078072850DC01201023874AD2
:1058600000210090202000F06AFC01201023844ACF
:105870000F210090202000F062FC01201023814ABB
:105880001E210090202000F05AFC012010237E4AA7
:105890002D210090202000F052FC734880780428CD
:1058A00007D100201023754A01460090202000F007
:1058B00046FC6D488078052807D100201023704AE7
:1058C0000F210090202000F03AFC674880780628DD
:1058D00007D1002010236B4A1E210090202000F0E9
:1058E0002EFC614880780728AED100201023664A3C
:1058F0002D210090202000F022FCB0E05A48807852
:10590000072854DD584880780B2850DC01201023EC
:105910005E4A00210090202000F011FC012010239D
:105920005B4A0F210090202000F009FC0120102389
:10593000584A1E210090202000F001FC0120102375
:10594000554A2D210090202000F0F9FB4648807830
:10595000082807D1002010234C4A0146009020203F
:1059600000F0EDFB40488078092807D10020102383
:10597000474A0F210090202000F0E1FB3A48807850
:105980000A2807D100201023424A1E21009020201F
:1059900000F0D5FB344880780B2860D1002010231C
:1059A0003D4A2D210090202000F0C9FB57E02E48F1
:1059B00080780B2853DD2C4880780F284FDC01209D
:1059C0001023364A00210090202000F0B8FB01206F
:1059D0001023334A0F210090202000F0B0FB01205B
:1059E0001023304A1E210090202000F0A8FB012047
:1059F00010232D4A2D210090202000F0A0FB1A48F2
:105A000080780C2807D100201023244A01460090FA
:105A1000202000F094FB144880780D2807D1002046
:105A200010231F4A0F210090202000F088FB0E4811
:105A300080780E2807D1002010231A4A1E210090DA
:105A4000202000F07CFB084880780F2807D1002038
:105A50001023154A2D210090202000F070FB08BD76
:105A60004D41433A0000000098070020BE0100208D
:105A7000CB010020D8010020E5010020F201002028
:105A8000FF0100200C020020190200202602002045
:105A900033020020400200204D0200205A02002064
:105AA00067020020740200208102002000BFFEE790
:105AB0002DE9F0410546002460E015F8248015F832
:105AC000240005EB84014978484005EB840189787E
:105AD000484005EB8401C97880EA010615F82400E6
:105AE00005EB8401497880EA0107384605F04CFF50
:105AF000074615F8240087EA0601484005F8240007
:105B000005EB8400407805EB8401897880EA010781
:105B1000384605F039FF074605EB8400407887EAF0
:105B20000601484005EB8401487005EB840080784D
:105B300005EB8401C97880EA0107384605F024FFA7
:105B4000074605EB8400807887EA0601484005EBAC
:105B50008401887005EB8400C07880EA0807384625
:105B600005F012FF074605EB8400C07887EA0601BE
:105B7000484005EB8401C870601CC4B2042C9CDB57
:105B8000BDE8F08100BFFEE770B500240CE0002501
:105B900006E00020074901EBC5010855681CC5B2A5
:105BA000802DF6DB601CC4B2082CF0DB00F0F0F8AE
:105BB00070BD0000E407002010B504461CB90021A8
:105BC000A62000F0E1FA012C03D10021A72000F06B
:105BD000DBFA10BD10B504463CB90021C82000F026
:105BE000D3FA0021A12000F0CFFA012C07D1002127
:105BF000C02000F0C9FA0021A02000F0C5FA10BDB5
:105C0000F0B514460B46CF1701EB5777C7F3C70221
:105C1000CF1701EB5777FF10A1EBC707FEB20123A7
:105C2000B340DDB24CB1134B03EBC0039B5C2B4381
:105C3000104F07EBC007BB541AE00E4B03EBC00339
:105C40009B5CDB430B4F07EBC007BB54094B03EBDB
:105C5000C0039B5C2B43074F07EBC007BB54054BAE
:105C600003EBC0039B5CDB43024F07EBC007BB5455
:105C7000F0BD0000E40700201FB5A0200090012027
:105C80000190039069464048FBF7B2FC0122A02135
:105C90003D48FBF75FFE002210213C48FBF75AFE0F
:105CA000C820FBF7BFFB012210213848FBF752FE4A
:105CB0000021AE2000F068FA0021022000F064FA12
:105CC0000021102000F060FA0021402000F05CFA72
:105CD0000021B02000F058FA0021812000F054FA91
:105CE0000021CF2000F050FA0021A12000F04CFA52
:105CF0000021A62000F048FA0021A82000F044FA74
:105D000000213F2000F040FA0021AD2000F03CFAD5
:105D100000218B2000F038FA0021332000F034FA03
:105D20000021C82000F030FA0021D32000F02CFA26
:105D30000021084600F028FA0021D52000F024FABE
:105D40000021802000F020FA0021D92000F01CFA68
:105D500000211F2000F018FA0021DA2000F014FAC8
:105D60000021122000F010FA0021DB2000F00CFAD4
:105D70000021402000F008FAFFF706FF0021AF20C5
:105D800000F002FA1FBD00000008014000100140B1
:105D900070B500241CE004F1B001C8B2002100F08D
:105DA000F3F90021022000F0EFF90021102000F0AB
:105DB000EBF9002508E0084901EBC501085D012168
:105DC00000F0E2F9681CC5B2802DF4DB601CC4B29F
:105DD000082CE0DB70BD0000E40700202DE9FE4F39
:105DE0000746884692461C460197CDF80080082C4D
:105DF00002D14FF006091FE02046E31704EB53736E
:105E0000DB1021464FEAE47C04EB5C7C4FEAEC0CAF
:105E1000A4EBCC0CBCF1000F02D04FF0010C01E060
:105E20004FF0000C6344224604EBD27C4FEA6C0C2A
:105E300003FB0CF303F0FF09AAF12000C6B2002512
:105E40005EE0082C07D106EB46002F4901EB40002D
:105E500010F805B01DE00C2C07D106EB46002B49CD
:105E600001EB800010F805B013E0102C05D1284894
:105E700000EB061010F805B00BE0182C07D106EB6C
:105E8000C600244901EB800010F805B001E0BDE830
:105E9000FE8F002002901CE00BF0010028B141466B
:105EA00038460C9AFFF7ACFE09E00C9808B90120BF
:105EB00000E00020024641463846FFF7A1FE4FEAC7
:105EC0006B0B08F1010000F0FF080298401CC0B203
:105ED000029002980828DFDB781CC7B2082C0BD090
:105EE00004EBD4714A100199791A8A4204D1019FB6
:105EF00000980830C0B20090DDF80080681CC5B280
:105F00004D459EDB00BFC2E79CB90008C4BB00083A
:105F100038C0000828C600082DE9FC4F074688460F
:105F200016461C46BB46CDF804802046E21704EB1B
:105F30005272D2102146E31704EB5373DB10A4EB2B
:105F4000C3030BB1012300E000231A44624392B261
:105F50000092002575E0102C05D13C4800EB46105E
:105F600010F805903BE0182C07D106EBC600384925
:105F700001EBC00010F8059031E0202C05D1354828
:105F800000EBC61010F8059029E0402C05D13248EE
:105F900000EB462010F8059021E00C2C07D106EB11
:105FA00046002E4901EBC00010F8059017E00E2CBA
:105FB00007D1C6EBC6002A4901EB800010F8059016
:105FC0000DE0122C09D106EBC60000EB400025497C
:105FD00001EB400010F8059001E0BDE8FC8F4FF0A8
:105FE000000A1CE009F0010028B1414638460B9A2E
:105FF000FFF706FE09E00B9808B9012000E0002039
:10600000024641463846FFF7FBFD4FEA690908F1B1
:10601000010000F0FF080AF1010000F0FF0ABAF1E8
:10602000080FDFDB781CC7B2A7EB0B00A04204D13E
:106030005F4601980830C0B20190DDF80480681C0A
:1060400085B20098854286DB00BFC6E784D300088E
:10605000A4D80008ECD800086CD900086CDB000854
:10606000C4DD00082CE000082DE9FF4F05460E4670
:1060700017461C46DDF838904FF0000A0095B346ED
:106080002046E21704EB5272D2102146E31704EBCC
:106090005373DB10A4EBC3030BB1012300E0002317
:1060A0001A44D4B24FF0000845E0002003903BE0D2
:1060B0000D9810F80A0002900AF101001FFA80FA08
:1060C000002001901DE0029800F0010028B14A462E
:1060D00031462846FFF794FD0AE0B9F1000F01D1DF
:1060E000012000E00020024631462846FFF788FDE7
:1060F000029840100290701CC6B20198401CC0B2B9
:10610000019001980828DEDB681CC5B20098281AA7
:10611000B84204D1009D0BF1080000F0FF0B5E4671
:106120000398401CC0B203900398B842C0DB08F14A
:10613000010000F0FF08A045B7DBBDE8FF8F2DE9A7
:10614000F84106460F4614461D46DDF81C8013E054
:10615000CDF8008022782B4639463046FFF73EFEC8
:10616000082D02D1B01DC6B205E0284605EBD0715E
:1061700006EB6101CEB2641C2078202802DB207877
:106180007E28E5DDBDE8F88170B504460E462EB1E7
:10619000012240211C48FBF7DDFB04E000224021E6
:1061A0001948FBF7D7FB002210211748FBF7D2FB59
:1061B00000251BE0002220211348FBF7CBFB04F055
:1061C000800028B1012280210F48FBF7C3FB04E0C7
:1061D000002280210C48FBF7BDFB012220210A4848
:1061E000FBF7B8FB6006040E681CC5B2082DE1DBA6
:1061F000012210210448FBF7ADFB01224021024897
:10620000FBF7A8FB70BD00000008014008B5084975
:106210000968C9084FF47A72B1FBF2F14143009169
:1062200000BF00BF00994A1E00920029F9D108BDA5
:1062300030070020014600BF080900EB8000420043
:1062400001F00F001044C0B2704770B5044600253D
:10625000FBF786FB054607E0FBF782FB401BB0F52A
:106260007A7F01D9032070BD2068406800F02000CB
:106270000028F1D02068406840F010002168486094
:106280000020F0E770B5044600252068406820F043
:10629000100021684860FBF763FB054607E0FBF749
:1062A0005FFB401BB0F57A7F01D9032070BD2068E9
:1062B000406800F020000028F1D00020F6E7000040
:1062C00010B50248FCF730F910BD0000FC22002098
:1062D0000146002200230868006A82B20868406A0A
:1062E00083B243EA0240704730B5014600220023E2
:1062F000002400200D68AD69AAB20D68ED69ACB24A
:106300000D68AD69ABB29A4205D00D68ED6963F3D3
:106310001F45284601E044EA024030BDF0B504467E
:106320000B460021002504F5FA61032B1BD2C3EBB9
:10633000C30000EB03100926B0FBF6F01044001D6B
:106340004618481E06EB90066427B0FBF7F0361A95
:10635000481EBF00B0FBF7F030440726B0FBF6F74D
:1063600006FB17051AE0C3EBC30000EB0310092678
:10637000B0FBF6F01044001D084400EB91006426C9
:10638000B1FBF6F6801B4FF4C876B1FBF6F630444D
:10639000801E0726B0FBF6F706FB1705E8B2F0BD36
:1063A00070B504460D4600262046FFF74EFF08B1A3
:1063B00001260AE0280C21680862A8B22168486218
:1063C0002046FFF75FFF00B10126304670BD70B573
:1063D00004460D4600262046FFF737FF08B1012688
:1063E0000AE0280C21688861A8B22168C8612046AB
:1063F000FFF748FF00B10126304670BD4178427971
:106400004270437A4371437B437241738178827A4D
:10641000827081728179837B83718173C178C27B41
:10642000C270C37AC373C379C372C171704700BFAE
:10643000012003F081FFFBE790B000BF012003F0D3
:106440007BFF04F095FD03F0AFFD3C220749684651
:10645000F9F7E8FE054810380FC8FDF7C9F9FFF74E
:1064600097FC03F0C7FD04F0DDFFE7E7A807002075
:1064700000BF012003F060FF0E48007840B100200B
:106480000C4908704FF4E160FAF7CCFFFEF738FBD7
:10649000094800780028ECD000200749087000BFA8
:1064A0000649087048708870C87001200449087057
:1064B000DFE7000020070020FA00002098070020F6
:1064C000F500002010B5364804F008FB3549088077
:1064D000084600884FF6FF71884213D101231A46FF
:1064E00031A132A004F0DAFB002857D04AF6AA21E5
:1064F0002B4800F013FE31A000F04EFE012034497D
:1065000008704BE0274800884AF6AA21884245D106
:1065100030A000F041FE3220FAF784FF01231A4632
:1065200032A135A004F0BAFB30B936A137A000F093
:1065300033FE01202649087001231A4636A139A0EE
:1065400004F0ACFB30B93AA130A000F025FE0220E7
:106550001F49087001231A4637A13AA004F09EFB98
:1065600030B93BA129A000F017FE0320184908709C
:1065700001231A4638A13BA004F090FB38B93DA195
:1065800022A000F009FE04201149087006E03BA19A
:106590003FA000F001FE00200D49087010BD000072
:1065A00000500708CA0600204F4B000041542B52F0
:1065B000455345543D310D0A00000000232323B804
:1065C000B4CEBBC9E8B1B8B3C9B9A60D0A00000082
:1065D000CC060020232323C0B6D1C0C4A3BFE9B793
:1065E000C7CAD7B4CEC6F4B6AF0D0A002B5555496D
:1065F00044533A303030320041542B5555494453BE
:106600003F0D0A0055554944530000002573B2BBA5
:10661000B7FBBACF0A0000002B555549444E3A4605
:106620004630340041542B555549444E3F0D0A0025
:10663000555549444E0000002B55554944573A469C
:106640004646350041542B55554944573F0D0A00E5
:1066500055554944570000002B5458504F57455248
:106660003A31300041542B5458504F5745523F0D4A
:106670000A0000005458504F5745520055554944A0
:10668000CFEEBCB0B7A2C9E4B9A6C2CA00000000F0
:10669000232573B7FBBACFC9E8D6C3CFEE0A0000F3
:1066A00000BF4FF47A7003F047FEFAE710B50246D8
:1066B00000200FE0002109E002EB81031B5C074C86
:1066C000E35C02EB810423544B1CD9B20429F3DBB5
:1066D000431CD8B20428EDDB10BD000090E3000895
:1066E00010B500BF502080F31188BFF34F8FBFF368
:1066F0006F8F00BF05F016F818B14FF080500449B5
:10670000086000BF002080F3118800BF10BD0000AA
:1067100004ED00E000B595B028210BA8F9F79BFD2A
:10672000142106A8F9F797FD18216846F9F793FD9B
:1067300009200B904FF480300C9000200D90012028
:106740000F90119002201290C10313914FF4E011A9
:1067500014910BA8FBF79CFC08B1F9F747FF0F2039
:10676000069002200790002008904FF48060099066
:1067700000200A90022106A8FBF732FB08B1F9F7C6
:1067800035FF01200090400201906846FBF790FA27
:1067900008B1F9F72BFF15B000BD704710B50248DE
:1067A000FCF7E3FA10BD00008430002010B5024869
:1067B000FCF7DBFA10BD0000C023002010B54FF439
:1067C00000710348FBF7BCF80248FCF7CEFA10BD95
:1067D000001001400824002010B50268204B9842A8
:1067E0000ED0204B98420BD0B0F1804F08D01E4BFA
:1067F000984205D01D4B984202D01D4B984203D1C0
:1068000022F070024B681A43154B98420ED0154B7C
:1068100098420BD0B0F1804F08D0134B984205D06E
:10682000124B984202D0124B984203D122F440728C
:10683000CB681A4322F080034C6943EA04020260E9
:106840008B68C3620B688362054B984202D0054B8C
:10685000984201D10B6903630123436110BD00001D
:10686000002C0140003401400004004000080040BA
:10687000000C004030B50C46816821F47F4142EAAB
:10688000032525432943816030BD0A46816821F0F4
:10689000700142F0070319438160704730B50B4621
:1068A0001446026A056A25F001050562816921F036
:1068B000F00141EA041122F00A021A4381610262E6
:1068C00030BD30B50B461446056A25F0100505624B
:1068D0008169026A21F4704141EA043122F0A00288
:1068E00042EA03128161026230BD000038B5002522
:1068F0001A4800680068C0F3001555B300BF0020B7
:1069000000901648006800680090144800684068CD
:10691000009000BF00BF1148FCF710FB1048006852
:1069200044686042801E0F49087001200E490870BB
:106930000C4800780D4908700A4802780C490D4847
:10694000F9F770FC4FF400620949891E0348FCF70F
:10695000C0FE0248FCF726FB38BD0000502C00208A
:10696000A42D0020140700201E0700201C07002073
:1069700052240020CC38002010B51F4800680028A1
:1069800008DD1E4800680068C0F3001010B1002048
:1069900019490860194800680068C0F3401030B316
:1069A000164800684068C4B2154813490968445441
:1069B0001148006840F2FF71884204D20E48006816
:1069C000401C0D4908600C4800880E4908800A48A0
:1069D00001680D48F9F73FFC002004E00849095C14
:1069E000094A1154401C044909688842F6DB0348EF
:1069F000FCF7D8FA10BD000018070020942C0020E6
:106A0000800C0020CE0600208014002070B50546C2
:106A10006C6A0020E085E0842046FCF7C2FA70BD75
:106A200070B506460025746A20684069C0F3C01539
:106A300094F83D00212805D125B10020E0842046AE
:106A400000F085F820684069C0F3801594F83E0096
:106A5000222805D125B10020E085204600F04CF821
:106A6000206C40F0100020642046FCF79AFA70BDBC
:106A700070B505466C6A2868006800F02000F8B917
:106A80000020E0852068C06820F480702168C8601C
:106A90002068406920F00100216848612068406951
:106AA00020F0400021684861202084F83E00206BDF
:106AB000012805D12068C06820F010002168C86056
:106AC000206B012804D1A18D2046FCF736FA02E0A4
:106AD0002046FCF71FFE70BD70B505466C6A206B42
:106AE000012805D1A08D41082046FCF726FA02E0D6
:106AF0002046FCF710FE70BD0168C96821F4907152
:106B00000268D1600168496921F0010102685161A0
:106B1000016B012905D10168C96821F010010268E3
:106B2000D160202180F83E1000210163704710B52C
:106B300004462068C06820F040002168C86020201A
:106B400084F83D002046FCF750FE002010BD01688F
:106B5000C96821F0C0010268D160202180F83D1091
:106B60007047F8B5044694F83E00222869D1A06821
:106B7000B0F5805F0CD1206950B90025A66A206865
:106B80004068C0F308003080A06A801CA06215E055
:106B9000A56A0026A068B0F5805F03D0A06828B978
:106BA000206918B920684068287004E020684068AF
:106BB00000F07F002870A06A401CA062E08D401E9B
:106BC00080B2E085A8BB2068C06820F02000216862
:106BD000C8602068C06820F480702168C8602068A0
:106BE000406920F0010021684861202084F83E00BF
:106BF000206B01281ED1002020632068C06820F08F
:106C000010002168C8602068006800F0100010289B
:106C10000AD100BF00200090206800680090206822
:106C20004068009000BF00BFA18D2046FCF785F9A9
:106C300003E004E02046FCF76DFD0020F8BD0020D5
:106C4000FCE70220FAE7000070B5044621680969F4
:106C500021F44051E2681143226811612269A16860
:106C60001143626941EA02052168C96841F20C6278
:106C7000914329432268D1602168496921F4407118
:106C8000A2691143226851612D4A2168914202D1C3
:106C9000FBF7A4F901E0FBF791F900EBC00101EB70
:106CA000001162689200B1FBF2F100EBC00202EB4E
:106CB000001263689B00B2FBF3F26423B2FBF3F2B1
:106CC00002EBC20303EB0212A1EB8201322202EBC0
:106CD00001116422B1FBF2F101F0F00100EBC002FE
:106CE00002EB001263689B00B2FBF3F26423B2FB79
:106CF000F3F201EB021200EBC00101EB001163683B
:106D00009B00B1FBF3F100EBC00303EB00136668DB
:106D1000B600B3FBF6F36426B3FBF6F303EBC3064E
:106D200006EB0313A1EB8301322303EB0111642370
:106D3000B1FBF3F101F00F0111442268916070BDC5
:106D40000038014077B581B0044615460298A0622C
:106D5000A58500202064222084F83E001C48A16BF9
:106D600088621C48A16BC8621B48A16B08630020A5
:106D7000A16B486302AE32682368191D2B46A06BD5
:106D8000FAF702FB00BF0020009020680068009026
:106D900020684068009000BF00BF00BF002084F85A
:106DA0003C0000BF2068C06840F480702168C86063
:106DB0002068406940F0010021684861206840690E
:106DC00040F0400021684861002004B070BD000020
:106DD000716A0008D96A0008216A0008014691F822
:106DE0003D00212828D18868B0F5805F0BD1086963
:106DF00048B90A6A1088C0F308000B685860086A2E
:106E0000801C086205E00B6A581C086218780B6841
:106E10005860C88C401E80B2C88458B90868C068E1
:106E200020F080000B68D8600868C06840F040001F
:106E30000B68D860002070470220FCE72DE9F04184
:106E400004460D4617469846069E21E0701CF8B190
:106E50002EB1FAF785FDA0EB0800B04218D92068E2
:106E6000C06820F4D0702168C8602068406920F0B4
:106E7000010021684861202084F83D0084F83E002C
:106E800000BF002084F83C0000BF0320BDE8F08173
:106E9000206800682840A84201D1012000E00020BD
:106EA000B842D3D00020F1E710B50248FCF77AF8D9
:106EB00010BD0000D82C002010B50248FCF772F875
:106EC00010BD00001C2D002010B50248FCF76AF828
:106ED00010BD0000602D002070B505460E4614461A
:106EE000A2B24FF6FF7331462846FCF715FCA2B25A
:106EF0004FF6FF7331460248FCF70EFC70BD0000F0
:106F0000602D002070B505460C460DA000F044F938
:106F10002046F9F7BDF986B24FF6FF733246214697
:106F20002846FCF7F9FB2046F9F7B2F986B24FF68E
:106F3000FF73324621460448FCF7EEFB70BD0000AB
:106F40000D0A434D443A0900602D002010B5024857
:106F5000F9F788FC10BD0000D422002010B50248CB
:106F6000F9F780FC10BD0000D422002000BFFEE72E
:106F700008B566480078062875D2DFE800F0C30639
:106F80009204030500BF00BF00BF00201023604A29
:106F9000014600901D20FFF7D2F8012010235D4A22
:106FA000202100900D20FFF7CAF8012010235A4A33
:106FB000202100906420FFF7C2F85448007804288C
:106FC00018D1012010232022114600902620FEF720
:106FD000A3FF012010232122202100903A20FEF758
:106FE0009BFF012010232222202100904E20FEF73B
:106FF00093FF55E045480078032818D1012010235D
:107000001E22202100902620FEF786FF012010235B
:107010001F22202100903A20FEF77EFF012010233E
:107020000022202100904E20FEF776FF38E03748FE
:107030000078012818D11023162220210090262044
:10704000FEF76AFF012010231722202100903A202A
:10705000FEF762FF012010230022202100904E2025
:10706000FEF75AFF1CE04DE028480078052817D1AC
:10707000012010232322202100902620FEF74CFF20
:10708000012010232422202100903A20FEF744FF03
:10709000012010232522202100904E20FEF73CFFE6
:1070A00031E001200C231B4A342100901420FFF70B
:1070B00046F801200C231122342100902620FEF7EF
:1070C0002BFF01200C231222342100903320FEF7E5
:1070D00023FF01200C231322342100904020FEF7CF
:1070E0001BFF01200C231422342100904D20FEF7B9
:1070F00013FF01200C23084A342100905C20FFF785
:107100001EF800E000BF00BF08BD00008E02002096
:107110008F0200209C0200209902002070B50446D6
:107120000D46204600F0FCF9FAF74AFA0F4884426F
:1071300008D00F48844205D00E48844202D00E4841
:10714000844207D12A46002321460220FAF7E0F9BB
:10715000064607E02A46002321460120FAF7D8F91F
:10716000064600BFFAF7CAF970BD000000380708EC
:1071700000400708004807080050070810B50246FD
:10718000002005E0135C0C5C63401354431CD8B230
:107190001028F7DB10BD00000FB4054B10B503A994
:1071A000044A029800F034F810BC5DF814FB0000AB
:1071B000517500089407002002480068C0F30220BF
:1071C000704700000CED00E010B5002804DB0A0752
:1071D000130E054A135406E00A07140E034A00F082
:1071E0000F031B1FD45410BD00E400E018ED00E0B5
:1071F00002E008C8121F08C1002AFAD17047704780
:10720000002001E001C1121F002AFBD170470000DD
:107210002DE9FF4F8BB09A460F460546002606E043
:1072200025280BD052460D9990476D1C761C287866
:107230000028F5D10FB03046BDE8F08F0024A046FD
:107240000122604900E0044315F8013F203B02FAA7
:1072500003F00842F7D128782E2817D115F8010F2E
:1072600044F004042A280ED06FF02F022878A0F1F1
:10727000300109290AD808EB880102EB410100EB33
:1072800001086D1CF2E757F8048B6D1C28786928FB
:107290003ED006DC0028CDD063280BD0642804D172
:1072A00036E0732810D075284BD052460D99904780
:1072B000761C85E017F8040B8DF8000000208DF88F
:1072C0000100E946012003E057F8049B4FF0FF302E
:1072D00061074FF0000401D40AE0641C44450DDA54
:1072E0008442FADB19F804100029F6D106E0641C88
:1072F0008442FCDB19F804100029F8D1264404E08C
:1073000019F8010B52460D999047641EF8D257E0C8
:1073100001CF4FF00A0B002802DA40422D2102E093
:10732000210504D52B218DF82410012103E0E1076C
:1073300005D02021F7E70DF1200908910CE000218C
:10734000F9E701CF4FF00A0BF9E75946F8F7A7FF25
:1073500001F1300209F8012D0028F6D1ADEB09004A
:1073600000F1200B600701D44FF00108D84502DD81
:10737000A8EB0B0000E000208046002406E009A8EE
:107380005246005D0D999047641C761C0898844213
:10739000F5DB04E0302052460D999047761CB8F199
:1073A0000001A8F10108F5DC05E019F8010B5246CF
:1073B0000D999047761CBBF10001ABF1010BF4DC99
:1073C0006D1C34E70928010008B501201023232291
:1073D000192100900A20FEF79FFD0120102324228E
:1073E000192100901E20FEF797FD01201023252271
:1073F000192100903220FEF78FFD01201023262254
:10740000192100904620FEF787FD01201023272236
:10741000192100905A20FEF77FFD01201023282219
:10742000192100906E20FEF777FD08BD0FB470B5EE
:1074300086B028A00068059027A30FCB01AC0FC42D
:1074400029480078042800D10A9C2748007805289C
:1074500000D10B9C24480078062800D10C9C2248BF
:107460000078072800D10D9C200E8DF80600200C16
:107470008DF80700200A8DF80800E0B28DF80900A9
:107480000E9E300E8DF80A00300C8DF80B00300A7D
:107490008DF80C00F0B28DF80D000F9D280E8DF8C0
:1074A0000E00280C8DF80F00280A8DF81000E8B2A5
:1074B0008DF8110001200E2301AA0221009005A8D9
:1074C00003F02AFC1420F9F783F806B070BC5DF8CD
:1074D00014FB000066010000030B00000000000028
:1074E00000000000000000009807002070B5024670
:1074F0000B464FF6FF7000210FE0555C68400025F9
:1075000008E000F00104401014B14AF20106704096
:1075100080B26D1C082DF4D3491C9942EDD370BD87
:1075200030B585B0044600200190039401200490FA
:1075300000200090FAF744F8694601A8F9F786FFA1
:107540000546F9F7DBFF0A20F9F76CFF05B030BDFF
:1075500013B50C464FF6FF73012269460248FCF74B
:10756000DBF800981CBD0000602D00200FB583B033
:10757000FE48406958B101200090FC4840690C2346
:1075800002461D2102900820FEF7D9FD07E00120E8
:107590000C23F7A21D2100900E20FEF7D0FDF3482A
:1075A000406A58B101200090F048406A0C2302461E
:1075B0001D2102902620FEF7C2FD07E001200C23CA
:1075C000ECA21D2100902C20FEF7B9FDE748406B8E
:1075D00058B101200090E548406B0C2302461D2164
:1075E00002904420FEF7ABFD07E001200C23E2A24D
:1075F0001D2100904A20FEF7A2FDDC48406C58B1E6
:1076000001200090D948406C0C2302461D210290B5
:107610006220FEF794FD07E001200C23D7A21D2174
:1076200000906820FEF78BFD41F2F0120398811A5A
:10763000904201F09A847ADC40F61172A0EB0201CC
:10764000904275D038DCB0F5887F72D018DCF02815
:1076500070D009DC01286ED00F286DD010286CD0B6
:10766000112842F08483B6E1FF2867D0B0F5807F0F
:107670007DD0A0F2011000287AD00E28F1D15AE274
:1076800040F2FF12811A904273D00ADCA0F211106E
:1076900000286FD00E286ED0DF286DD0E028E0D112
:1076A000CAE3A1F60151002967D0012966D00F294C
:1076B00065D01029D5D1FEE2B1F5877F6FD015DCFA
:1076C000EF296DD008DC0E296BD0DF296AD0E029C4
:1076D00069D0EE29C5D1B4E3F02972D0FE2971D06A
:1076E000FF2970D0B1F5807FBBD1F7E3B1F5F87F0A
:1076F00001F03B820BDCA1F2DF11002977D00129D8
:1077000076D00F2975D01029ABD101F073B9B1F53E
:10771000FF7F01F02B82A1F2FF11002901F02484E8
:10772000012901F01F860F299BD101F01CBE06E044
:1077300084E3BDE2F8E0A8E0A8E0F4E04CE14DF617
:107740000F72881A914276D05DDC40F60162A1EB9F
:107750000200914201F00C8636DC40F61F52A1EB8C
:107760000200914201F004821EDC012908E097E149
:10777000DFE162E35EE35EE39CE292E1DCE1D9E11A
:1077800001F0F2850F2901F0F085B1F5516F01F09C
:107790003381A1F6115100298CD101F0E8B9FDE344
:1077A000FDE34CE385E24BE3012801F0DF8302288F
:1077B00001F0DC85102801F0DA85E1288AD101F09A
:1077C000D6BBEDE3EDE3EDE34DF21F02811A9042EB
:1077D0007DD00FDC0E2801F0CC85A0F550400F388D
:1077E000002875D0012874D00F288DD1F5E3F5E37A
:1077F000F5E3F5E301296DD00F296CD0E0296BD0BA
:10780000E12991D1EDE340F60162811A904201F045
:10781000F2801FDC122801F0AD850DDC012801F09B
:10782000EC80022801F0A581102801F0A381112825
:10783000B2D101F09DBBFDE3202801F09C85F12829
:1078400001F09783F22801F09785B0F5807FA3D1EE
:1078500001F093BD1F2901F092850CDC012901F094
:107860008A810F2901F08881102901F08383112971
:1078700092D101F083BDF02901F07D83F12901F05F
:107880007F85FF2988D101F07CBD00BF01200C233A
:107890003B4A082100900846FEF751FC01200C23CA
:1078A000374A082100902620FEF749FC01200C23CE
:1078B000334A082100904420FEF741FC089880B329
:1078C0000398012818D12F4914231A4605E0FDE337
:1078D000FDE3FDE3FDE3FDE3FDE3CDE9001006215B
:1078E0006420FEF7C1FB012010230B222E21009003
:1078F0006620FEF711FB14E003980F2811D1012038
:10790000214914231A46CDE9001006216420FEF710
:10791000ABFB012010230C222E2100906620FEF7E5
:10792000FBFA02F045BA00BF01200C23144A0821DB
:1079300000900846FEF703FC01200C23104A0821A2
:1079400000902620FEF7FBFB01200C230C4A0821A7
:1079500000906220FEF7F3FB069828B303981028E6
:1079600023D10120074914231A460FE0980700206D
:107970004C3100004C3200004C3300004C3400000D
:10798000F0000020000000203C000020CDE90010A5
:1079900006214620FEF768FB012010230B222E2132
:1079A00000904820FEF7B8FA14E00398F02811D1AF
:1079B0000120FE4914231A46CDE900100621462075
:1079C000FEF752FB012010230C222E2100904820AC
:1079D000FEF7A2FAA5E700BF01200C23F44A082114
:1079E00000900846FEF7ABFB01200C23F04A08216B
:1079F00000902620FEF7A3FB069840B3089830B30A
:107A00000398112824D10120EA4914231A46CDE90C
:107A1000001006214620FEF727FB012010230B2231
:107A20002E2100904820FEF777FA0120E149142327
:107A30001A46CDE9001006216420FEF715FB01204F
:107A400010230B222E2100906620FEF765FA26E017
:107A50000398FF2823D10120D44914231A46CDE9E5
:107A6000001006214620FEF7FFFA012010230C2209
:107A70002E2100904820FEF74FFA0120CB49142315
:107A80001A46CDE9001006216420FEF7EDFA012028
:107A900010230C222E2100906620FEF73DFA40E7CD
:107AA00000BF01200C23C24A082100900846FEF7BF
:107AB00046FB01200C23BE4A082100904420FEF71B
:107AC0003EFB01200C23BA4A082100906220FEF7F9
:107AD00036FB059860B30398B0F5807F12D1012082
:107AE000B44914231A46CDE9001006212820FEF7D8
:107AF000BBFA012010230B222E2100902A20FEF732
:107B00000BFA15E00398B0F5706F11D10120A74969
:107B100014231A46CDE9001006212820FEF7A4FA06
:107B2000012010230C222E2100902A20FEF7F4F9C8
:107B3000F7E600BF00BF00BF01200C239C4A0821CC
:107B400000900846FEF7FBFA01200C23984A082112
:107B500000904420FEF7F3FA059850B3089840B31C
:107B600040F201110398884224D101209149142345
:107B70001A46CDE9001006212820FEF775FA0120EB
:107B800010230B222E2100902A20FEF7C5F9012098
:107B9000884914231A46CDE9001006216420FEF717
:107BA00063FA012010230B222E2100906620FEF79D
:107BB000B3F97CE040F60F710398884224D101208C
:107BC0007A4914231A46CDE9001006212820FEF731
:107BD0004BFA012010230C222E2100902A20FEF7C0
:107BE0009BF90120714914231A46CDE900100621A2
:107BF0006420FEF739FA012010230C222E21009078
:107C00006620FEF789F952E040F20F11039888428E
:107C100024D10120674914231A46CDE9001006211A
:107C20002820FEF721FA012010230B222E2100909C
:107C30002A20FEF771F901205C4914231A46CDE988
:107C4000001006216420FEF70FFA012010230C22F9
:107C50002E2100906620FEF75FF928E040F60171C2
:107C60000398884223D10120504914231A46CDE9B4
:107C7000001006212820FEF7F7F9012010230C221E
:107C80002E2100902A20FEF747F9012049491423AC
:107C90001A46CDE9001006216420FEF7E5F901201F
:107CA00010230B222E2100906620FEF735F938E6CE
:107CB00000BF00BF00BF01200C233D4A08210090F7
:107CC0000846FEF73CFA01200C23394A08210090AF
:107CD0006220FEF734FA059848B3069838B3039843
:107CE000B0F5887F24D10120324914231A46CDE90A
:107CF000001006212820FEF7B7F9012010230B22DF
:107D00002E2100902A20FEF707F90120294914238B
:107D10001A46CDE9001006214620FEF7A5F90120FC
:107D200010230B222E2100904820FEF7F5F880E06A
:107D30000398B0F57F6F24D101201C4914231A4603
:107D4000CDE9001006212820FEF78EF9012010232E
:107D50000C222E2100902A20FEF7DEF80120134984
:107D600014231A46CDE9001006214620FEF77CF9BF
:107D7000012010230C222E2100904820FEF7CCF881
:107D800057E00398B0F5F87F2BD10120094914235F
:107D90001A46CDE9001006212820FEF765F90120DA
:107DA00010230B222E2100902A2005E03C00002009
:107DB000F000002000000020FEF7AEF80120FE4990
:107DC00014231A46CDE9001006214620FEF74CF98F
:107DD000012010230C222E2100904820FEF79CF851
:107DE00027E00398B0F5716F23D10120F2491423E5
:107DF0001A46CDE9001006212820FEF735F90120AA
:107E000010230C222E2100902A20FEF785F8012055
:107E1000EA4914231A46CDE9001006214620FEF750
:107E200023F9012010230B222E2100904820FEF779
:107E300073F876E500BF00BF00BF00BF00BF00BF02
:107E400000BF01200C23DE4A082100900846FEF7FF
:107E500076F90598002840D006980028FBD00898AD
:107E60000028F8D040F211110398884237D1012040
:107E7000D24914231A46CDE9001006212820FEF726
:107E8000F3F8012010230B222E2100902A20FEF768
:107E900043F80120C94914231A46CDE900100621F0
:107EA0004620FEF7E1F8012010230B222E2100903E
:107EB0004820FEF731F80120C04914231A46CDE9C5
:107EC000001006216420FEF7CFF8012010230B22BA
:107ED0002E2100906620FEF71FF8BEE18CE340F2F1
:107EE0001F110398884236D10120B44914231A4641
:107EF000CDE9001006212820FEF7B6F80120102356
:107F00000B222E2100902A20FEF706F80120AB4913
:107F100014231A46CDE9001006214620FEF7A4F8E6
:107F2000012010230B222E2100904820FDF7F4FFA2
:107F30000120A14914231A46CDE90010062164202E
:107F4000FEF792F8012010230C222E2100906620CB
:107F5000FDF7E2FF81E140F2F1110398884241D13F
:107F60000120964914231A46CDE900100621282045
:107F7000FEF77AF8012010230B222E2100902A20F0
:107F8000FDF7CAFF01208C4914231A46CDE90010E1
:107F900006214620FEF768F8012004E02DE35DE1AC
:107FA000A5E1A6E162E210230C222E2100904820D8
:107FB000FDF7B2FF0120814914231A46CDE90010D4
:107FC00006216420FEF750F8012010230B222E21F9
:107FD00000906620FDF7A0FF3FE189E148E20DE354
:107FE0000DE30FE340F2FF110398884238D10120DE
:107FF000724914231A46CDE9001006212820FEF705
:1080000033F8012010230B222E2100902A20FDF7A7
:1080100083FF0120684914231A46CDE90010062188
:108020004620FEF721F8012010230C222E2100907B
:10803000482000E0E7E2FDF76FFF01205E491423CE
:108040001A46CDE9001006216420FEF70DF8012044
:1080500010230C222E2100906620FDF75DFFFCE02E
:1080600040F61171039888423DD1012052491423F2
:108070001A46CDE9001006212820FDF7F5FF012062
:1080800010230C222E2100902A20FDF745FF01200D
:108090004A4914231A46CDE9001006214620FDF76F
:1080A000E3FF012010230B222E2100904820FDF732
:1080B00033FF0120414914231A46CDE9001006215F
:1080C0006420FDF7D1FF0120102305E0D1E1C6E0D7
:1080D00010E195E295E2CAE10B222E210090662084
:1080E000FDF71AFFB9E040F61F710398884236D1B8
:1080F0000120314914231A46CDE900100621282019
:10810000FDF7B2FF012010230C222E2100902A201F
:10811000FDF702FF0120294914231A46CDE900107A
:1081200006214620FDF7A0FF012010230B222E215F
:1081300000904820FDF7F0FE01201F4914231A4645
:10814000CDE9001006216420FDF78EFF01201023E9
:108150000C222E2100906620FDF7DEFE7DE040F629
:10816000F171039888423DD10120134914231A4626
:10817000CDE9001006212820FDF776FF012010230D
:108180000C222E2100902A20FDF7C6FE01200A496C
:1081900014231A46CDE9001006214620FDF764FF9E
:1081A000012010230C222E2100904820FDF7B4FE60
:1081B00001200249142305E03C00002000000020BB
:1081C000F00000201A46CDE9001006216420FDF7DA
:1081D0004BFF012010230B222E2100906620FDF77B
:1081E0009BFE3AE040F6FF710398884235D10120AA
:1081F000FE4914231A46CDE9001006212820FDF778
:1082000033FF012010230C222E2100902A20FDF79D
:1082100083FE0120F54914231A46CDE900100621FA
:108220004620FDF721FF012010230C222E21009073
:108230004820FDF771FE0120EC4914231A46CDE9D0
:10824000001006216420FDF70FFF012010230C22EF
:108250002E2100906620FDF75FFE20E400BF012084
:108260000C23E34A082100902620FDF768FF012037
:108270000C23DF4A082100904420FDF760FF012015
:108280000C23DB4A082100906220FDF758FF049878
:1082900060B30398B0F5805F12D10120D549142353
:1082A0001A46CDE9001006210A20FDF7DDFE012067
:1082B00010230B222E2100900C20FDF72DFE15E03F
:1082C0000398B0F5704F11D10120C84914231A4604
:1082D000CDE9001006210A20FDF7C6FE012010237B
:1082E0000C222E2100901046FDF716FE20E400BF60
:1082F00000BF00BF01200C23BD4A082100902620AA
:10830000FDF71DFF01200C23B94A082100904420ED
:10831000FDF715FF049850B3089840B341F20101EE
:108320000398884224D10120B24914231A46CDE98A
:10833000001006210A20FDF797FE012010230B22D2
:108340002E2100900C20FDF7E7FD0120A949142300
:108350001A46CDE9001006216420FDF785FE0120B4
:1083600010230B222E2100906620FDF7D5FD7CE026
:108370004FF20F010398884224D101209B49142316
:108380001A46CDE9001006210A20FDF76DFE0120F6
:1083900010230C222E2100901046FDF7BDFD012078
:1083A000924914231A46CDE9001006216420FDF7F6
:1083B0005BFE012010230C222E2100906620FDF789
:1083C000ABFD52E041F20F010398884224D1012015
:1083D000884914231A46CDE9001006210A20FDF72A
:1083E00043FE012010230B222E2100900C20FDF7CC
:1083F00093FD01207D4914231A46CDE90010062182
:108400006420FDF731FE012010230C222E21009064
:108410006620FDF781FD28E04FF2010103988842B4
:1084200023D10120714914231A46CDE900100621F9
:108430000A20FDF719FE012010230C222E210090A6
:108440001046FDF769FD01206A4914231A46CDE95B
:10845000001006216420FDF707FE012010230B22E7
:108460002E2100906620FDF757FD20E400BF00BFDD
:1084700000BF01200C235E4A082100902620FDF752
:108480005EFE01200C235A4A082100906220FDF76D
:1084900056FE049850B3069840B341F21001039879
:1084A000884224D10120534914231A46CDE90010F3
:1084B00006210A20FDF7D8FD012010230B222E21D2
:1084C00000900C20FDF728FD01204A4914231A468C
:1084D000CDE9001006214620FDF7C6FD012010233E
:1084E0000B222E2100904820FDF716FD7CE04FF274
:1084F000F0010398884224D101203C4914231A46F4
:10850000CDE9001006210A20FDF7AEFD0120102361
:108510000C222E2100901046FDF7FEFC012033496D
:1085200014231A46CDE9001006214620FDF79CFDD4
:10853000012010230C222E2100904820FDF7ECFC96
:1085400052E041F2F0010398884224D101202949E8
:1085500014231A46CDE9001006210A20FDF784FDF8
:10856000012010230B222E2100900C20FDF7D4FCBB
:1085700001201E4914231A46CDE900100621462089
:10858000FDF772FD012010230C222E2100904820BF
:10859000FDF7C2FC28E04FF210010398884223D176
:1085A0000120124914231A46CDE9001006210A20A1
:1085B000FDF75AFD012010230C222E2100901046B9
:1085C000FDF7AAFC01200B4914231A46CDE900103F
:1085D00006214620FDF748FD012010230B222E2105
:1085E00000904820FDF798FC23E400003C000020A8
:1085F000F00000200000002000BF00BF00BF00BF4F
:1086000000BF00BF00BF01200C23F74A08210090E3
:108610002620FDF794FD0498002840D006980028F5
:10862000FBD008980028F8D041F211010398884245
:1086300036D10120ED4914231A46CDE90010062158
:108640000A20FDF711FD012010230B222E2100909E
:108650000C20FDF761FC0120E44914231A46CDE902
:10866000001006214620FDF7FFFC012010230B22FD
:108670002E2100904820FDF74FFC0120DB491423F8
:108680001A46CDE9001006216420FDF7EDFC01201B
:1086900010230B222E2100906620FDF73DFCA2E165
:1086A00041F21F010398884236D10120CF4914239B
:1086B0001A46CDE9001006210A20FDF7D5FC01205D
:1086C00010230B222E2100900C20FDF725FC012009
:1086D000C64914231A46CDE9001006214620FDF7AD
:1086E000C3FC012010230B222E2100904820FDF70F
:1086F00013FC0120BE4914231A46CDE900100621BF
:108700006420FDF7B1FC012010230C222E210090E3
:108710006620FDF701FC66E141F2F1010398884211
:1087200036D10120B14914231A46CDE900100621A3
:108730000A20FDF799FC012010230B222E21009026
:108740000C20FDF7E9FB0120A94914231A46CDE9C5
:10875000001006214620FDF787FC012010230C2283
:108760002E2100904820FDF7D7FB01209F491423BC
:108770001A46CDE9001006216420FDF775FC0120A2
:1087800010230B222E2100906620FDF7C5FB2AE165
:1087900041F2FF010398884236D101209349142306
:1087A0001A46CDE9001006210A20FDF75DFC0120E4
:1087B00010230B222E2100900C20FDF7ADFB012091
:1087C0008B4914231A46CDE9001006214620FDF7F7
:1087D0004BFC012010230C222E2100904820FDF795
:1087E0009BFB0120824914231A46CDE90010062183
:1087F0006420FDF739FC012010230C222E2100906B
:108800006620FDF789FBEEE04FF2110103988842E4
:1088100036D10120764914231A46CDE900100621ED
:108820000A20FDF721FC012010230C222E210090AC
:108830001046FDF771FB01206C4914231A46CDE95F
:10884000001006214620FDF70FFC012010230B220B
:108850002E2100904820FDF75FFB0120634914237F
:108860001A46CDE9001006216420FDF7FDFB01202A
:1088700010230B222E2100906620FDF74DFBB2E065
:108880004FF21F010398884236D101205849142322
:108890001A46CDE9001006210A20FDF7E5FB01206C
:1088A00010230C222E2100901046FDF735FB0120ED
:1088B0004E4914231A46CDE9001006214620FDF743
:1088C000D3FB012010230B222E2100904820FDF71E
:1088D00023FB0120464914231A46CDE90010062146
:1088E0006420FDF7C1FB012010230C222E210090F3
:1088F0006620FDF711FB76E04FF2F1010398884204
:1089000036D101203A4914231A46CDE90010062138
:108910000A20FDF7A9FB012010230C222E21009034
:108920001046FDF7F9FA0120314914231A46CDE922
:10893000001006214620FDF797FB012010230C2292
:108940002E2100904820FDF7E7FA01202749142343
:108950001A46CDE9001006216420FDF785FB0120B1
:1089600010230B222E2100906620FDF7D5FA3AE065
:108970004FF2FF010398884235D101201C4914238E
:108980001A46CDE9001006210A20FDF76DFB0120F3
:1089900010230C222E2100901046FDF7BDFA012075
:1089A000134914231A46CDE9001006214620FDF78D
:1089B0005BFB012010230C222E2100904820FDF7A4
:1089C000ABFA01200A4914231A46CDE9001006210A
:1089D0006420FDF749FB012010230C222E2100907A
:1089E0006620FDF799FA38E4F0000020000000202E
:1089F0003C00002000BF00BF00BF01200C23FD4A47
:108A0000082100904420FDF79AFB01200C23F94A2D
:108A1000082100906220FDF792FB049848B3059866
:108A200038B30398B0F5885F24D10120F2491423AC
:108A30001A46CDE9001006210A20FDF715FB01209A
:108A400010230B222E2100900C20FDF765FA012047
:108A5000E94914231A46CDE9001006212820FDF724
:108A600003FB012010230B222E2100902A20FDF76A
:108A700053FA79E00398B0F57F4F24D10120DF4904
:108A800014231A46CDE9001006210A20FDF7ECFA5E
:108A9000012010230C222E2100901046FDF73CFAF5
:108AA0000120D64914231A46CDE9001006212820BA
:108AB000FDF7DAFA012010230C222E2100902A2043
:108AC000FDF72AFA50E00398B0F5F85F24D10120B1
:108AD000C94914231A46CDE9001006210A20FDF7E2
:108AE000C3FA012010230B222E2100900C20FDF749
:108AF00013FA0120C14914231A46CDE900100621BA
:108B00002820FDF7B1FA012010230C222E2100901D
:108B10002A20FDF701FA27E00398B0F5714F23D121
:108B20000120B64914231A46CDE9001006210A2077
:108B3000FDF79AFA012010230C222E2100901046F6
:108B4000FDF7EAF90120AC4914231A46CDE90010DB
:108B500006212820FDF788FA012010230B222E2160
:108B600000902A20FDF7D8F97FE400BF00BF00BFC6
:108B700000BF00BF00BF00BF01200C239D4A082199
:108B800000904420FDF7DBFA0498002840D00598B7
:108B90000028FBD008980028F8D041F20111039872
:108BA000884236D10120944914231A46CDE9001099
:108BB00006210A20FDF758FA012010230B222E214E
:108BC00000900C20FDF7A8F901208B4914231A46C8
:108BD000CDE9001006212820FDF746FA01201023D8
:108BE0000B222E2100902A20FDF796F901208249C0
:108BF00014231A46CDE9001006216420FDF734FA4B
:108C0000012010230B222E2100906620FDF784F90D
:108C1000A9E141F20F110398884236D1012076492B
:108C200014231A46CDE9001006210A20FDF71CFA8C
:108C3000012010230B222E2100900C20FDF76CF94F
:108C400001206D4914231A46CDE900100621282081
:108C5000FDF70AFA012010230B222E2100902A2072
:108C6000FDF75AF90120654914231A46CDE9001091
:108C700006216420FDF7F8F9012010230C222E2193
:108C800000906620FDF748F96DE141F60171039807
:108C9000884236D10120584914231A46CDE90010E4
:108CA00006210A20FDF7E0F9012010230B222E21D6
:108CB00000900C20FDF730F90120504914231A468A
:108CC000CDE9001006212820FDF7CEF90120102360
:108CD0000C222E2100902A20FDF71EF90120464982
:108CE00014231A46CDE9001006216420FDF7BCF9D3
:108CF000012010230B222E2100906620FDF70CF995
:108D000031E141F60F710398884236D101203A498A
:108D100014231A46CDE9001006210A20FDF7A4F914
:108D2000012010230B222E2100900C20FDF7F4F8D7
:108D30000120324914231A46CDE9001006212820CB
:108D4000FDF792F9012010230C222E2100902A20F9
:108D5000FDF7E2F80120294914231A46CDE9001055
:108D600006216420FDF780F9012010230C222E211A
:108D700000906620FDF7D0F8F5E04FF2011103985E
:108D800088423DD101201D4914231A46CDE9001027
:108D900006210A20FDF768F9012010230C222E215C
:108DA00000901046FDF7B8F80120134914231A4625
:108DB000CDE9001006212820FDF756F901201023E7
:108DC0000B222E2100902A20FDF7A6F801200A4947
:108DD00014231A46CDE9001006216420FDF744F95A
:108DE000012010230B222E2100906620FDF794F81D
:108DF000B9E00000F0000020000000203C0000204E
:108E00004FF20F110398884236D10120F8491423FC
:108E10001A46CDE9001006210A20FDF725F90120A8
:108E200010230C222E2100901046FDF775F801202A
:108E3000F04914231A46CDE9001006212820FDF739
:108E400013F9012010230B222E2100902A20FDF778
:108E500063F80120E64914231A46CDE900100621E3
:108E60006420FDF701F9012010230C222E2100902F
:108E70006620FDF751F876E04FF6017103988842BD
:108E800036D10120DA4914231A46CDE90010062113
:108E90000A20FDF7E9F8012010230C222E21009072
:108EA0001046FDF739F80120D14914231A46CDE9BF
:108EB000001006212820FDF7D7F8012010230C22EE
:108EC0002E2100902A20FDF727F80120C9491423FC
:108ED0001A46CDE9001006216420FDF7C5F80120EF
:108EE00010230B222E2100906620FDF715F83AE0A2
:108EF0004FF60F710398884235D10120BC491423E5
:108F00001A46CDE9001006210A20FDF7ADF8012030
:108F100010230C222E2100901046FCF7FDFF0120AB
:108F2000B34914231A46CDE9001006212820FDF785
:108F30009BF8012010230C222E2100902A20FCF700
:108F4000EBFF0120AA4914231A46CDE9001006219F
:108F50006420FDF789F8012010230C222E210090B7
:108F60006620FCF7D9FF3EE500BF00BF00BF00BF91
:108F700000BF00BF00BF01200C239F4A08210090C2
:108F80006220FDF7DCF80498002840D005980028FE
:108F9000FBD006980028F8D041F2101103988842BF
:108FA00036D10120934914231A46CDE90010062139
:108FB0000A20FDF759F8012010230B222E210090E2
:108FC0000C20FCF7A9FF01208A4914231A46CDE999
:108FD000001006214620FDF747F8012010230B2240
:108FE0002E2100904820FCF797FF0120814914238F
:108FF0001A46CDE9001006212820FDF735F801209A
:1090000010230B222E2100902A20FCF785FFA8E1D7
:1090100041F2F0110398884236D10120754914239A
:109020001A46CDE9001006210A20FDF71DF801209F
:1090300010230B222E2100900C20FCF76DFF012045
:109040006C4914231A46CDE9001006212820FDF7AB
:109050000BF8012010230B222E2100902A20FCF770
:109060005BFF0120624914231A46CDE90010062156
:109070004620FCF7F9FF012010230C222E2100903E
:109080004820FCF749FF6CE141F6107103988842D3
:1090900036D10120574914231A46CDE90010062184
:1090A0000A20FCF7E1FF012010230B222E21009063
:1090B0000C20FCF731FF01204D4914231A46CDE95D
:1090C000001006212820FCF7CFFF012010230C22DE
:1090D0002E2100902A20FCF71FFF01204549142370
:1090E0001A46CDE9001006214620FCF7BDFF0120FD
:1090F00010230B222E2100904820FCF70DFF30E1B9
:1091000041F6F0710398884236D101203949142381
:109110001A46CDE9001006210A20FCF7A5FF012020
:1091200010230B222E2100900C20FCF7F5FE0120CD
:109130002F4914231A46CDE9001006212820FCF7F8
:1091400093FF012010230C222E2100902A20FCF7EF
:10915000E3FE0120264914231A46CDE9001006211A
:109160004620FCF781FF012010230C222E210090C5
:109170004820FCF7D1FEF4E04FF21011039888422A
:109180003CD101201A4914231A46CDE900100621CA
:109190000A20FCF769FF012010230C222E210090E9
:1091A0001046FCF7B9FE0120124914231A46CDE9F6
:1091B000001006212820FCF757FF012010230B2266
:1091C0002E2100902A20FCF7A7FE01200949142334
:1091D0001A46CDE9001006214620FCF745FF012084
:1091E00010230B222E2100904820FCF795FEB8E0BA
:1091F0003C00002000000020F00000204FF2F011A1
:109200000398884236D10120FE4914231A46CDE93D
:10921000001006210A20FCF727FF012010230C2252
:109220002E2100901046FCF777FE0120F64914230A
:109230001A46CDE9001006212820FCF715FF012071
:1092400010230B222E2100902A20FCF765FE01201E
:10925000EC4914231A46CDE9001006214620FCF7FC
:1092600003FF012010230C222E2100904820FCF740
:1092700053FE76E04FF610710398884236D10120F4
:10928000E04914231A46CDE9001006210A20FCF714
:10929000EBFE012010230C222E2100901046FCF73B
:1092A0003BFE0120D74914231A46CDE900100621C0
:1092B0002820FCF7D9FE012010230C222E2100903B
:1092C0002A20FCF729FE0120CF4914231A46CDE9B4
:1092D000001006214620FCF7C7FE012010230B22B8
:1092E0002E2100904820FCF717FE3AE04FF6F0716F
:1092F0000398884235D10120C24914231A46CDE98A
:10930000001006210A20FCF7AFFE012010230C22DA
:109310002E2100901046FCF7FFFD0120B9491423CF
:109320001A46CDE9001006212820FCF79DFE0120F9
:1093300010230C222E2100902A20FCF7EDFD0120A5
:10934000B04914231A46CDE9001006214620FCF747
:109350008BFE012010230C222E2100904820FCF7C8
:10936000DBFD00E600BF00BF00BF00BF00BF00BFC5
:1093700000BF00BF00BF00BF00BF00BF00BF00BFF5
:1093800000BF0498002855D005980028FBD0069807
:109390000028F8D008980028F5D041F21111039860
:1093A000884248D10120984914231A46CDE900107B
:1093B00006210A20FCF758FE012010230B222E2143
:1093C00000900C20FCF7A8FD01208F4914231A46B9
:1093D000CDE9001006212820FCF746FE01201023CD
:1093E0000B222E2100902A20FCF796FD01208649B1
:1093F00014231A46CDE9001006214620FCF734FE5E
:10940000012010230B222E2100904820FCF784FD20
:1094100001207D4914231A46CDE90010062164205D
:10942000FCF722FE012010230B222E210090662043
:10943000FCF772FD25E241F21F110398884248D1E2
:109440000120714914231A46CDE9001006210A2093
:10945000FCF70AFE012010230B222E2100900C2085
:10946000FCF75AFD0120684914231A46CDE9001083
:1094700006212820FCF7F8FD012010230B222E21C5
:1094800000902A20FCF748FD01205F4914231A466A
:10949000CDE9001006214620FCF7E6FD012010234F
:1094A0000B222E2100904820FCF736FD0120554963
:1094B00014231A46CDE9001006216420FCF7D4FDE0
:1094C000012010230C222E2100906620FCF724FDA1
:1094D000D7E141F2F1110398884248D101204A496D
:1094E00014231A46CDE9001006210A20FCF7BCFD22
:1094F000012010230B222E2100900C20FCF70CFDE4
:109500000120414914231A46CDE9001006212820E4
:10951000FCF7AAFD012010230B222E2100902A2007
:10952000FCF7FAFC0120374914231A46CDE9001054
:1095300006214620FCF798FD012010230C222E2145
:1095400000904820FCF7E8FC01202F4914231A461C
:10955000CDE9001006216420FCF786FD01201023D0
:109560000B222E2100906620FCF7D6FCFEE341F290
:10957000FF11039888424DD10120234914231A4634
:10958000CDE9001006210A20FCF76EFD0120102312
:109590000B222E2100900C20FCF7BEFC01201A4962
:1095A00014231A46CDE9001006212820FCF75CFDA3
:1095B000012010230B222E2100902A20FCF7ACFC66
:1095C0000120104914231A46CDE900100621462037
:1095D000FCF74AFD012010230C222E210090482088
:1095E000FCF79AFC0120074914231A46CDE9001024
:1095F00006216420FCF738FD012010230C222E21C7
:10960000009003E03C000020000000206620FCF7F2
:1096100083FCABE341F611710398884248D10120E5
:10962000FE4914231A46CDE9001006210A20FCF752
:109630001BFD012010230B222E2100900C20FCF793
:109640006BFC0120F64914231A46CDE900100621CF
:109650002820FCF709FD012010230C222E21009068
:109660002A20FCF759FC0120EC4914231A46CDE9C5
:10967000001006214620FCF7F7FC012010230B22E6
:109680002E2100904820FCF747FC0120E3491423D9
:109690001A46CDE9001006216420FCF7E5FC012004
:1096A00010230B222E2100906620FCF735FC5DE391
:1096B00041F61F710398884248D10120D7491423ED
:1096C0001A46CDE9001006210A20FCF7CDFC012046
:1096D00010230B222E2100900C20FCF71DFC0120F2
:1096E000CF4914231A46CDE9001006212820FCF7A3
:1096F000BBFC012010230C222E2100902A20FCF715
:109700000BFC0120C54914231A46CDE9001006219F
:109710004620FCF7A9FC012010230B222E210090EB
:109720004820FCF7F9FB0120BD4914231A46CDE976
:10973000001006216420FCF797FC012010230C2266
:109740002E2100906620FCF7E7FB0FE341F6F17154
:109750000398884248D10120B04914231A46CDE924
:10976000001006210A20FCF77FFC012010230B22A9
:109770002E2100900C20FCF7CFFB0120A8491423D8
:109780001A46CDE9001006212820FCF76DFC0120C7
:1097900010230C222E2100902A20FCF7BDFB012073
:1097A0009F4914231A46CDE9001006214620FCF7F4
:1097B0005BFC012010230C222E2100904820FCF796
:1097C000ABFB0120954914231A46CDE90010062170
:1097D0006420FCF749FC012010230B222E2100906D
:1097E0006620FCF799FBC1E241F6FF7103988842BD
:1097F00048D10120894914231A46CDE900100621D9
:109800000A20FCF731FC012010230B222E210090AE
:109810000C20FCF781FB0120814914231A46CDE975
:10982000001006212820FCF71FFC012010230C2229
:109830002E2100902A20FCF76FFB01207849142389
:109840001A46CDE9001006214620FCF70DFC012048
:1098500010230C222E2100904820FCF75DFB0120F4
:109860006F4914231A46CDE9001006216420FCF745
:10987000FBFB012010230C222E2100906620FCF718
:109880004BFB73E24FF211110398884248D101203B
:10989000634914231A46CDE9001006210A20FCF77B
:1098A000E3FB012010230C222E2100901046FCF730
:1098B00033FB0120594914231A46CDE90010062133
:1098C0002820FCF7D1FB012010230B222E21009031
:1098D0002A20FCF721FB0120504914231A46CDE928
:1098E000001006214620FCF7BFFB012010230B22AD
:1098F0002E2100904820FCF70FFB0120474914233C
:109900001A46CDE9001006216420FCF7ADFB0120CA
:1099100010230B222E2100906620FCF7FDFA25E291
:109920004FF21F110398884248D101203C4914236B
:109930001A46CDE9001006210A20FCF795FB01200C
:1099400010230C222E2100901046FCF7E5FA01208E
:10995000324914231A46CDE9001006212820FCF7CD
:1099600083FB012010230B222E2100902A20FCF7DC
:10997000D3FA0120294914231A46CDE90010062103
:109980004620FCF771FB012010230B222E210090B2
:109990004820FCF7C1FA0120214914231A46CDE9D9
:1099A000001006216420FCF75FFB012010230C222D
:1099B0002E2100906620FCF7AFFAD7E14FF2F111AB
:1099C000039888424DD10120154914231A46CDE948
:1099D000001006210A20FCF747FB012010230C226F
:1099E0002E2100901046FCF797FA01200B49142312
:1099F0001A46CDE9001006212820FCF735FB01208E
:109A000010230B222E2100902A20FCF785FA01203A
:109A1000034914231A46CDE9001003E0000000209A
:109A20003C00002006214620FCF71EFB01201023ED
:109A30000C222E2100904820FCF76EFA0120DE490E
:109A400014231A46CDE9001006216420FCF70CFB14
:109A5000012010230B222E2100906620FCF75CFAD7
:109A600084E14FF2FF110398884248D10120D34985
:109A700014231A46CDE9001006210A20FCF7F4FA57
:109A8000012010230C222E2100901046FCF744FAEE
:109A90000120C94914231A46CDE9001006212820C7
:109AA000FCF7E2FA012010230B222E2100902A203D
:109AB000FCF732FA0120C14914231A46CDE90010FF
:109AC00006214620FCF7D0FA012010230C222E217B
:109AD00000904820FCF720FA0120B84914231A46C8
:109AE000CDE9001006216420FCF7BEFA0120102306
:109AF0000C222E2100906620FCF70EFA36E14FF67C
:109B000011710398884248D10120AC4914231A46A8
:109B1000CDE9001006210A20FCF7A6FA0120102347
:109B20000C222E2100901046FCF7F6F90120A349E3
:109B300014231A46CDE9001006212820FCF794FAD8
:109B4000012010230C222E2100902A20FCF7E4F99A
:109B50000120994914231A46CDE900100621462018
:109B6000FCF782FA012010230B222E2100904820BE
:109B7000FCF7D2F90120904914231A46CDE90010D0
:109B800006216420FCF770FA012010230B222E21FD
:109B900000906620FCF7C0F9E8E04FF61F710398CB
:109BA000884248D10120854914231A46CDE9001086
:109BB00006210A20FCF758FA012010230C222E213E
:109BC00000901046FCF7A8F901207C4914231A469E
:109BD000CDE9001006212820FCF746FA01201023C9
:109BE0000C222E2100902A20FCF796F901207249C0
:109BF00014231A46CDE9001006214620FCF734FA5A
:109C0000012010230B222E2100904820FCF784F91C
:109C100001206A4914231A46CDE900100621642068
:109C2000FCF722FA012010230C222E21009066203E
:109C3000FCF772F99AE04FF6F1710398884248D127
:109C400001205E4914231A46CDE9001006210A209E
:109C5000FCF70AFA012010230C222E210090104656
:109C6000FCF75AF90120554914231A46CDE9001092
:109C700006212820FCF7F8F9012010230C222E21C0
:109C800000902A20FCF748F901204C4914231A4679
:109C9000CDE9001006214620FCF7E6F9012010234B
:109CA0000C222E2100904820FCF736F90120424971
:109CB00014231A46CDE9001006216420FCF7D4F9DC
:109CC000012010230B222E2100906620FCF724F99E
:109CD0004CE04FF6FF710398884247D10120374985
:109CE00014231A46CDE9001006210A20FCF7BCF91E
:109CF000012010230C222E2100901046FCF70CF9B5
:109D000001202E4914231A46CDE9001006212820EF
:109D1000FCF7AAF9012010230C222E2100902A2002
:109D2000FCF7FAF80120254914231A46CDE9001062
:109D300006214620FCF798F9012010230C222E2141
:109D400000904820FCF7E8F801201C4914231A462B
:109D5000CDE9001006216420FCF786F901201023CC
:109D60000C222E2100906620FCF7D6F820E001207E
:109D70000C23134A082100900846FCF7E0F9012063
:109D80000C230F4A082100902620FCF7D8F9012067
:109D90000C230B4A082100904420FCF7D0F9012045
:109DA0000C23074A082100906220FCF7C8F900BF85
:109DB00000BF07B000BD0000000000203C000020F4
:109DC000F000002090B0F7F7DDFDFCF7A3FCFBF7F7
:109DD0005DF8FAF7BDFFFBF79DF9FBF7E1F9FBF73B
:109DE00015FAFBF783FAFBF79DFAFBF7B7FAFBF7D7
:109DF00045FAFBF75FFAFBF7B1F9FAF76FFFFBF7EC
:109E0000D1F82448F8F7E4FE2348F8F7E1FE00BF54
:109E1000FBF732FF0020FBF7CFFE0020FBF7DAFE56
:109E200000BF00BF1D480068C06840F010001B491B
:109E30000968C8604FF4006219491848F9F749FCED
:109E400000BF18480068C06840F020001549096844
:109E5000C86000BF14A0FDF79FF9BB201849087027
:109E60000320184908703C22154910316846F6F75E
:109E7000D9F913480FC8F9F7BBFCFBF789FF00BFFE
:109E800000F086FDFAF7D2FCFAF7C2FF00F060FAA4
:109E900000BFFEE7C023002008240020502C002033
:109EA00050240020942C00204A4C5F4454555F42BB
:109EB0004C30312D73746172742E2E2E0D0A0000F9
:109EC000980700208E02002008B5012010231422DC
:109ED0000D2100900A20FCF71FF801201023152205
:109EE0000D2100901B20FCF717F80120102327A25A
:109EF0000D2100902C20FCF722F9012010231C22B8
:109F00000D2100903F20FCF707F8012010231D22AF
:109F10000D2100905020FBF7FFFF012010230D22A0
:109F2000282100900A20FBF7F7FF012010230E22C2
:109F3000282100902120FBF7EFFF012010230F22A2
:109F4000282100903720FBF7E7FF012010231A4655
:109F5000282100905020FBF7DFFF0D4840780128B2
:109F600008D1002010230BA20D2100906420FCF7E3
:109F7000E6F80AE00648407838B90020102305A228
:109F8000282100906420FCF7DAF808BD534E000049
:109F9000980700203C2D2D0001460020842901D087
:109FA000CA1C10447047000000B54FF480524FF4B3
:109FB00070410C48008800F0BBFF4FF480724FF4F2
:109FC00070610948008800F0B3FF1022F0210748B3
:109FD000008800F0ADFF01220F210548008800F045
:109FE000A7FF00BDBA020020BC020020BE02002074
:109FF000C00200200EB58F48C078042873D18D4868
:10A00000007804280BD08B480078052807D08948B1
:10A010000078062803D0874800780728EED18548C5
:10A020000078042838D184480068401C82490860C0
:10A030000846008881B28148FDF770F87D48407875
:10A04000012813D17C4AD2E904109269CDE90102BA
:10A05000009179480FC8FDF7E9F942F222217848CA
:10A06000FDF75CF83220F7F7DDF915E0714840782C
:10A0700090B9714AD2E904109269CDE901020091C8
:10A080006D480FC800F0F4F841F211116C48FDF76B
:10A0900045F83220F7F7C6F966480078052837D129
:10A0A00065484068401C644948600846808881B221
:10A0B0006448FDF733F85F484078012814D15E49C1
:10A0C000D1E904028969CDE9012100905A480FC8FD
:10A0D000FDF7ACF942F222215B48FDF71FF8322070
:10A0E000F7F7A0F914E0A4E05248407880B9524A4A
:10A0F000103207CA8DE807004F480FC800F0B8F8C3
:10A1000041F211115048FDF709F83220F7F78AF9AA
:10A1100048480078062836D147488068401C4649A0
:10A1200088600846008981B24848FCF7F7FF41483B
:10A130004078012811D1404A103207CA8DE8070043
:10A140003D480FC8FDF772F942F222214048FCF762
:10A15000E5FF3220F7F766F915E03648407890B908
:10A16000354AD2E904109269CDE9010200913248E2
:10A170000FC800F07DF841F211113548FCF7CEFF11
:10A180003220F7F74FF92B480078072834D12A48B6
:10A19000C068401C2849C8600846808981B22D48A3
:10A1A000FCF7BCFF23484078012811D1224A103225
:10A1B00007CA8DE8070020480FC8FDF737F942F2BB
:10A1C00022212548FCF7AAFF3220F7F72BF913E0EC
:10A1D0001848407880B9184A103207CA8DE807003D
:10A1E00015480FC800F044F841F211111A48FCF765
:10A1F00095FF3220F7F716F9114800F06FFC174968
:10A200000880114800F06AFC15490880104800F0E9
:10A2100065FC14490880104800F060FC1249088071
:10A220006420F7F7FFF803200249C87001200F49A6
:10A2300008700EBD98070020640C00200038070845
:10A24000000007080040070800100708004807083A
:10A25000002007080050070800300708BA02002055
:10A26000BC020020BE020020C0020020F500002039
:10A270000FB470B586B02AA00068059029A30FCB53
:10A2800001AC0FC42B480078042800D10A9C29484F
:10A290000078052800D10B9C26480078062800D1BC
:10A2A0000C9C24480078072800D10D9C200E8DF8C6
:10A2B0000600200C8DF80700200A8DF80800E0B297
:10A2C0008DF809000E9E300E8DF80A00300C8DF8C6
:10A2D0000B00300A8DF80C00F0B28DF80D000F9DC8
:10A2E000280E8DF80E00280C8DF80F00280A8DF826
:10A2F0001000E8B28DF811009DF840008DF81200B2
:10A3000001200F2301AA0221009005A800F004FDFE
:10A310001420F6F75DF906B070BC5DF814FB000080
:10A3200066010000020C00000000000000000000B8
:10A33000000000009807002070B5044625460DB1C6
:10A34000294600E00121084600F018FF002070BDFA
:10A3500010B500F041FF002010BD7FB504460D464A
:10A36000606998B1A06988B1B4F90800FFF714FEDC
:10A370000646D4E90510CDE9006102902B4622691A
:10A38000D4E9001001F072F9039013E0B4F9080069
:10A39000FFF702FE064603A8CDE90060238A9AB2C1
:10A3A0002B46D4E9001001F02FF9012802D000203B
:10A3B00004B070BD0398FBE72DE9F04105460E4659
:10A3C0001C4807681C480068001D00F0DBFD50B900
:10A3D0001948006890F82C10012088401749096836
:10A3E000814316480160681C38B936B112480168CB
:10A3F000091D134800F010FE1AE07C190E48006891
:10A400004460BC4207D20C480168091D0D48006831
:10A4100000F0E8FD0CE008480168091D0A480068E2
:10A4200000F0E0FD09480068844201D2074804605A
:10A43000BDE8F08148070020340700204C070020C9
:10A44000CC4100203C070020380700206407002092
:10A4500010B5044600F0ECFD23480068401C22497A
:10A4600008602248006840B9204804600846006837
:10A4700001280DD100F03AF90AE01D48006838B90A
:10A480001A480068C06AE16A884201D81748046027
:10A4900018480068401C1749086094F82C100120E7
:10A4A000884015490968084313490860E16A01EBCF
:10A4B0008101124A02EB8100211D00F0ADFD00F088
:10A4C000E1FD0B48006868B108480068C06AE16AAD
:10A4D000884207D24FF0805009490860BFF34F8F80
:10A4E000BFF36F8F10BD0000440700203407002029
:10A4F00050070020600700204C070020F04000209B
:10A5000004ED00E010B516E000F092FD0C48C068C4
:10A51000C468201D00F036FD0A480068401E094945
:10A52000086009480068401E0749086000F0AAFD5D
:10A53000204600F00BF8044800680028E4D110BD64
:10A54000B8410020440700204007002010B5044611
:10A5500094F8510030B9206B00F0B2FD204600F0B5
:10A56000AFFD1AE094F85100012803D1204600F015
:10A57000A7FD12E094F85100022801D1012000E06B
:10A58000002050B900BF502080F31188BFF34F8FD7
:10A59000BFF36F8F00BF00BFFEE710BD30B54FF4B3
:10A5A0004063174800F007042CB1C01D20F00700DD
:10A5B000134C041B1B1B0246124C22600024114D3D
:10A5C0006C60D018083820F007000F4C2060002481
:10A5D0000D4D2D686C600C4D2D682C601146441A91
:10A5E0004C60094C24680C60084D4C682C60084D88
:10A5F0004C682C604FF00044064D2C6030BD0000CC
:10A60000E04100207007002078070020800700202C
:10A610007C0700208407002000BFFFF773FF064877
:10A6200000680128F9D94FF0805004490860BFF351
:10A630004F8FBFF36F8FF0E7F040002004ED00E094
:10A640002DE9FF5F81460F469246DDE90E6B109CB7
:10A65000AAF10100216B01EB800828F0070808F03F
:10A66000070008B9012000E0002050B900BF5020C9
:10A6700080F31188BFF34F8FBFF36F8F00BF00BF10
:10A68000FEE7002507E0795D04F134004155785D6F
:10A6900000B902E06D1C102DF5D300BF002143204E
:10A6A0000155072E00D30626E66266640020A064EA
:10A6B000201D00F094FC04F1180000F090FC2461CF
:10A6C000C6F10700A06164620020E06484F85000D5
:10A6D00049464046039A00F049F92060BBF1000F5B
:10A6E00001D0CBF80040BDE8FF9F000010B500246A
:10A6F00007E004EB84010F4A02EB810000F062FCEA
:10A70000641C072CF5D30C4800F05CFC0B4800F0EF
:10A7100059FC0B4800F056FC0A4800F053FC0A486C
:10A7200000F050FC044809490860044808490860E2
:10A7300010BD0000F04000207C410020904100202E
:10A74000A4410020B8410020CC410020380700205F
:10A750003C07002010B50146164800E00068036879
:10A760008B42FBD30246436813448B4204D14368B7
:10A770004C682344436001460A464B68134404680E
:10A78000A34211D10C4C03682468A34208D04B6843
:10A790000468646823444B6003681B680B6005E031
:10A7A000054B1B680B6001E003680B60884200D01A
:10A7B000016010BD70070020780700200A49096871
:10A7C000096809B9012100E0002121B14FF0FF31F2
:10A7D000064A116006E004490968C968C868034A66
:10A7E00041681160704700003807002064070020AE
:10A7F0000E480068401C08B9012000E0002050B954
:10A8000000BF502080F31188BFF34F8FBFF36F8FCD
:10A8100000BF00BFFEE700BF502080F31188BFF3E8
:10A820004F8FBFF36F8F00BF00BFFEE78807002088
:10A830002DE9F04104464FF0000800F025FD4648A0
:10A84000006808B9FFF7AAFE4448006820400028C5
:10A850006BD1D4B1083404F00700B0B104F00700A4
:10A86000C0F10800044404F0070008B9012000E02A
:10A87000002050B900BF502080F31188BFF34F8FE4
:10A88000BFF36F8F00BF00BFFEE7002C4DD03448F0
:10A890000068844249D8334E3046056801E02E46B0
:10A8A0002D686868A04202D228680028F7D12A489B
:10A8B0000068854239D0306800F1080828683060A7
:10A8C0006868001B102819D92F1907F0070008B96C
:10A8D000012000E0002050B900BF502080F3118813
:10A8E000BFF34F8FBFF36F8F00BF00BFFEE76868F5
:10A8F000001B78606C603846FFF72CFF18496868C9
:10A900000968081A16490860084600681649096867
:10A91000884203D212480068134908600F496868EA
:10A920000968084368600020286000F09FFF08F075
:10A93000070008B9012000E0002050B900BF5020F6
:10A9400080F31188BFF34F8FBFF36F8F00BF00BF3D
:10A95000FEE74046BDE8F08178070020840700202C
:10A960007C0700207007002080070020001F4FF0A8
:10A9700080730360001F21F001030360001F034B7D
:10A98000036014380260203870470000F1A7000807
:10A990002DE9F05F00F0A8F83A4800F09FF88046F3
:10A9A000394800F09BF88146384800F097F8824615
:10A9B000374800F093F88346364800F092F8044692
:10A9C000354800F08EF80546344800F08AF806460F
:10A9D000334800F086F807464FF6FF70804502D0F6
:10A9E0000120304908704FF6FF70814502D00120E8
:10A9F0002D4908704FF6FF70824502D001202B4987
:10AA000008704FF6FF70834502D001202849087076
:10AA1000601C18B901202749086001E0254804603E
:10AA2000681C18B901202349486001E021484560AD
:10AA3000701C18B901201F49886001E01D4886601C
:10AA4000781C18B901201B49C86001E01948C7608B
:10AA5000194800F043F819490880194800F03EF8F9
:10AA600018490880184800F039F818490880184833
:10AA700000F034F817490880012017490870BDE834
:10AA8000F09F0000006007080068070800770708CB
:10AA90000078070800380708004007080048070842
:10AAA00000500708F6000020F7000020F800002002
:10AAB000F9000020640C002000000708BA02002002
:10AAC00000100708BC02002000200708BE0200207A
:10AAD00000300708C0020020F50000200146088869
:10AAE00070470146086870472DE9F0414448FFF778
:10AAF000F5FF04464348FFF7F1FF05464248FFF7DC
:10AB0000EDFF06464148FFF7E9FF0746002018E041
:10AB100081B2491CA14213D13D4901EB00114968A2
:10AB20003C4A51613A4901EB00118968916038490A
:10AB300001EB0011C968D1600121374A117002E0B0
:10AB4000401C1F28E4D300BF002018E081B2491C3C
:10AB5000A94213D12E4901EB001149682D4A5162D7
:10AB60002B4901EB001189689161294901EB001122
:10AB7000C968D1610121294A117002E0401C1F28D7
:10AB8000E4D300BF002018E081B2491CB14213D1C8
:10AB90001F4901EB001149681E4A51631C4901EB32
:10ABA0000011896891621A4901EB0011C968D162EC
:10ABB00001211B4A117002E0401C1F28E4D300BF92
:10ABC000002018E081B2491CB94213D1104901EBB1
:10ABD000001149680F4A51640D4901EB0011896861
:10ABE00091630B4901EB0011C968D16301210D4A42
:10ABF000117002E0401C1F28E4D300BFBDE8F081C3
:10AC00000060070800680708007707080078070851
:10AC1000B804002098070020F6000020F70000206C
:10AC2000F8000020F90000202DE9F047044689468D
:10AC300015461E46002700BF21E005EB85004FEAC0
:10AC4000400821461048FCF75DF93220F6F7EAFB90
:10AC50000E490FA0FCF7A0FA0AE049460B48F5F7A9
:10AC600005FB10B10120BDE8F0876420F6F7DAFBA0
:10AC7000B8F10000A8F10108EFD1781CC7B2B742C3
:10AC8000DBDB0020EFE70000502C0020CC38002058
:10AC90002D2D2D2D2D2D2D3E257300002DE9F04756
:10ACA0000446894615461E46002700BF25E005EBF1
:10ACB00085004FEA400821461248FCF723F91E2080
:10ACC000F6F7B0FB104911A0FCF766FA0EE0494612
:10ACD0000D48F5F7CBFA30B132210B48F5F7BBFA46
:10ACE0000120BDE8F0876420F6F79CFBB8F1000076
:10ACF000A8F10108EBD1781CC7B2B742D7DB00201E
:10AD0000EFE70000942C0020801400202D2D2D2D25
:10AD10002D2D2D3E257300002DE9F0478AB0054604
:10AD2000884616461C46DDF84890142105A8F5F71C
:10AD300092FA28788DF8140068788DF8150021466D
:10AD4000304600F015FE82460020019002900390EC
:10AD5000049000BF03E0315C01AA1154401CA042E2
:10AD6000F9D301A800F804A0B9F1000F09D0144AE2
:10AD700014491548F5F709FB102201A91248F5F707
:10AD8000E6FA002006E001A9095C00EB080205AB29
:10AD90009954401C1028F6DB122105A8FCF7A6FBED
:10ADA0000746F8B28DF82600380A8DF827001422DD
:10ADB00005A90648FCF790F80AB0BDE8F087000046
:10ADC000F4060020E4060020C42F0020942C00206C
:10ADD00008B50120102350A2022100901420FBF797
:10ADE000AEF901200E231422022100903220FBF73D
:10ADF00093F801200E231522022100904620FBF734
:10AE00008BF80120102345A2112100901420FBF79C
:10AE100096F901200E231422112100903220FBF715
:10AE20007BF801200E231522112100904620FBF70C
:10AE300073F8012010233AA2202100901420FBF780
:10AE40007EF901200E231422202100903220FBF7EE
:10AE500063F801200E231522202100904620FBF7E5
:10AE60005BF8012010232FA22F2100901420FBF764
:10AE700066F901200E2314222F2100903220FBF7C7
:10AE80004BF801200E2315222F2100904620FBF7BE
:10AE900043F82548407803280BD12348807840B9EF
:10AEA0000020102321A2022100906420FBF747F923
:10AEB00030E01D48407802280CD11B4880780128DA
:10AEC00008D10020102319A2112100906420FBF763
:10AED00036F91FE01448407801280CD112488078D8
:10AEE000022808D10020102310A220210090642005
:10AEF000FBF725F90EE00C48407858B90A488078ED
:10AF0000032807D10020102308A22F2100906420DD
:10AF1000FBF715F908BD00004C2031004C20320031
:10AF20004C2033004C203400980700203C2D2D008D
:10AF300010B541F2111398420DD10C4B5B680B40D8
:10AF40008B4202D1094B5A600EE0084B5B681343F9
:10AF5000064C636008E042F22223984204D1034B7E
:10AF60005B680B43014C636010BD00009807002034
:10AF700010B5F8F71DFDF8F721FEF8F721FFF9F7F6
:10AF8000E7F910BD01460A69D1E901309860D1E9BD
:10AF9000010358605068884201D1886850600020E1
:10AFA00008611068401E106010687047034B036012
:10AFB000034B0B608023136070470000801C00204F
:10AFC000D41C002000F1080141604FF0FF31816086
:10AFD00000F10801C160016100210160704700219A
:10AFE0000161704710B502460B685C1C0CB9106912
:10AFF00007E002F1080000E04068446824689C42D1
:10B00000FAD944684C604C68A160886041600A616C
:10B010001468641C146010BD42684A6093688B60B9
:10B02000936859609160086103685B1C0360704716
:10B0300000BF502080F31188BFF34F8FBFF36F8F95
:10B0400000BF0E480068401C0C49086008460068B4
:10B05000012812D10A480068C0B208B9012000E0F6
:10B06000002050B900BF502080F31188BFF34F8FEC
:10B07000BFF36F8F00BF00BFFEE770478807002057
:10B0800004ED00E00D48006850B900BF502080F387
:10B090001188BFF34F8FBFF36F8F00BF00BFFEE774
:10B0A00006480068401E054908600846006820B947
:10B0B000002080F3118800BF00BF70478807002080
:10B0C00070B506463546002E3FD0083D2C461F4938
:10B0D00060680968084008B1012000E0002050B90C
:10B0E00000BF502080F31188BFF34F8FBFF36F8FE5
:10B0F00000BF00BFFEE7206808B9012000E0002083
:10B1000050B900BF502080F31188BFF34F8FBFF3B9
:10B110006F8F00BF00BFFEE70C49606809680840F8
:10B1200098B1206888B909496068096888436060F7
:10B1300000F0AAF8064960680968084404490860F4
:10B140002046FFF707FB00F091FB70BD840700204D
:10B150007C07002000204FF0E0210861886106484C
:10B1600000684FF47A71B0FBF1F0401E4FF0E0211F
:10B1700048610720086170473007002070B5044619
:10B180000025D4B11248006808B9012000E0002071
:10B1900050B900BF502080F31188BFF34F8FBFF329
:10B1A0006F8F00BF00BFFEE700F06EF80021204661
:10B1B000FFF702F900F05AFB05463DB94FF0805009
:10B1C00004490860BFF34F8FBFF36F8F70BD00005D
:10B1D0006C07002004ED00E010B586B0002005905B
:10B1E000049003AA04A905A8FFF7E0FE0022DDE908
:10B1F00004101346CDE9002102901CA11D48039ABA
:10B2000000F034FA1C4908600846006808B10124BF
:10B2100000E00024012C15D100BF502080F31188DC
:10B22000BFF34F8FBFF36F8F00BF4FF0FF30134955
:10B23000086001201249086000201249086000F0EF
:10B2400067F910E0601C08B1012000E0002050B94F
:10B2500000BF502080F31188BFF34F8FBFF36F8F73
:10B2600000BF00BFFEE706B010BD000049444C45DA
:10B270000000000019A600086807002064070020ED
:10B28000500700204807002002480068401C014980
:10B29000086070476C0700201D48006818B1012045
:10B2A0001C49086032E000201A4908601A4800680A
:10B2B000B0FA80F0C0F11F0101EB8100174A52F88B
:10B2C000200008B1012000E0002050B900BF50204C
:10B2D00080F31188BFF34F8FBFF36F8F00BF00BFA4
:10B2E000FEE701EB81020D4B03EB820042685268DE
:10B2F000426000F108024368934202D142685268FA
:10B3000042604268D268064B1A6000BF7047000076
:10B310006C070020580700204C070020F040002058
:10B32000340700200FB408B50120102338A20821EB
:10B3300000900420FAF703FF01200C2335A2082116
:10B3400000900020FAF7FBFE0120122300220C21BE
:10B3500000903720FAF7E0FD0120122302460C216D
:10B3600000904B20FAF7D8FD012012230222282159
:10B3700000903720FAF7D0FD012012230322282164
:10B3800000904B20FAF7C8FD9DF80800042806D16C
:10B390000020009010231E21079AFAF7D0FE9DF896
:10B3A0000800052806D10020009010231E210B9ACA
:10B3B000FAF7C5FE9DF80800062806D10020009087
:10B3C00010231E210F9AFAF7BAFE9DF808000728ED
:10B3D00006D10020009010231E21139AFAF7AFFE29
:10B3E0009DF80900012808D1002010230CA20C218F
:10B3F00000905D20FAF7A3FE07E00020102308A2CA
:10B40000282100905D20FAF79AFE01B05DF814FB48
:10B41000534E3A004C4F434B4E414D453A000000CD
:10B420003C2D2D003048007800B970472E48007838
:10B43000662857D12C484078012853D12A48807873
:10B4400001284FD12848C07828490880264800792B
:10B4500027490870244840792649096841EA006074
:10B460002449086020488079096841EA0040214960
:10B4700008601D48C079096841EA00201D4908603C
:10B480001948007A096808431A4908601648407A42
:10B49000194908701448807A184908701248C07A0F
:10B4A000174908701048007B164908700E48407B09
:10B4B0001549098841EA0020134908800A48807B21
:10B4C00009880843104908800748C07B0F4909884C
:10B4D00041EA00200D4908800348007C09880843A0
:10B4E0000A49088000BFA0E780140020D40600208D
:10B4F000D6060020D8060020DC060020DD0600204D
:10B50000DE060020DF060020E0060020E206002024
:10B510001CB53849084600780190FF200A46107093
:10B520000846007800909DF8000000F0F0009DF8BB
:10B530000020904201D1012000E0002050B900BF5E
:10B54000502080F31188BFF34F8FBFF36F8F00BF80
:10B5500000BFFEE79DF8000000F05000264A107082
:10B560000720264A106009E024480068401E234A4C
:10B5700010609DF800004006000E00909DF800004D
:10B5800000F080008028EFD01C480068C0F1070060
:10B59000042801D1012000E0002050B900BF502054
:10B5A00080F31188BFF34F8FBFF36F8F00BF00BFD1
:10B5B000FEE7124800680002104A1060104600883A
:10B5C00000F4E06010600B4A019810700C480068AD
:10B5D00040F470000A4908600846006840F0704076
:10B5E0000860FFF7B7FD002006490860F4F7BEFDCC
:10B5F00000201CBD00E400E08C0700209007002024
:10B6000020ED00E0880700202DE9FF4F85B080463F
:10B6100089461746DDE912ABB800FFF709F906467F
:10B6200056B15420FFF704F904460CB1266304E038
:10B630003046FFF745FD00E000248CB1002084F87F
:10B640005100CDE900ABCDE902403A4649464046BB
:10B65000089BFEF7F5FF2046FEF7FAFE012501E004
:10B660004FF0FF35284609B0BDE8F08F2DE9F04FC7
:10B6700085B00746884691469A46DDE90EB6109C8D
:10B680000EB1012000E0002050B900BF502080F32F
:10B690001188BFF34F8FBFF36F8F00BF00BFFEE76E
:10B6A0000CB1012000E0002050B900BF502080F311
:10B6B0001188BFF34F8FBFF36F8F00BF00BFFEE74E
:10B6C000542003900398542801D1012000E0002069
:10B6D00050B900BF502080F31188BFF34F8FBFF3E4
:10B6E0006F8F00BF00BFFEE7B4B1AEB125462C4658
:10B6F0002E63022085F85100002004A953464A46D3
:10B70000CDE900B1CDE9025041463846FEF798FF39
:10B710002846FEF79DFE01E000200490049805B045
:10B72000BDE8F08F2DE9F0414FF000084448006873
:10B73000002877D143480068451C4248056015BB86
:10B7400041480068006808B9012000E0002050B9B5
:10B7500000BF502080F31188BFF34F8FBFF36F8F6E
:10B7600000BF00BFFEE73848076838480068364920
:10B7700008603648076036480068401C3449086055
:10B78000FFF71CF800BF3348006885423CD300BF78
:10B790002D480068006808B9012000E0002020B1B1
:10B7A0004FF0FF302B4908602DE027480068C06843
:10B7B000C4686668B54202D22648066023E0201DB0
:10B7C000FFF7E0FBA06A18B104F11800FFF7DAFBFD
:10B7D00094F82C10012088401F49096808431E492D
:10B7E0000860E16A01EB81011C4A02EB8100211D26
:10B7F000FFF712FC1A49E06A0968C96A8842C7D390
:10B800004FF00108C4E700BF15480068C06A00EBAC
:10B810008000124951F82000012801D94FF0010899
:10B8200005E0FFE70F480068401C0E4908600E481D
:10B83000006808B14FF001084046BDE8F081000003
:10B840006C07002048070020380700203C07002034
:10B850005C070020640700204C070020F040002017
:10B8600034070020540700205807002070B500243A
:10B8700000263648006850B900BF502080F3118878
:10B88000BFF34F8FBFF36F8F00BF00BFFEE7FFF71F
:10B89000CFFB2E480068401E2C490860084600680F
:10B8A00000284FD12A48006800284BD024E02948BE
:10B8B000C068C46804F11800FFF764FB201DFFF79F
:10B8C00061FB94F82C100120884023490968084343
:10B8D00021490860E16A01EB8101204A02EB810005
:10B8E000211DFFF799FB1E49E06A0968C96A884271
:10B8F00002D301201B4908601648006808B90120DE
:10B9000000E000200028D2D00CB1FEF757FF164807
:10B91000056865B100BFFFF705FF10B101201149AF
:10B9200008606D1E002DF6D100200F4908600D48FB
:10B93000006838B1012630070C490860BFF34F8F0B
:10B94000BFF36F8FFFF79EFB304670BD6C07002082
:10B9500044070020A44100204C070020F0400020B4
:10B9600034070020580700205407002004ED00E0B1
:10B9700010B502461378012002E0145C6340401CBD
:10B980008842FADB184610BD0146C80900EBC0002A
:10B9900000EB400080EA4100C0B2704700000000A8
:10B9A00000000000002F0000000007000700001446
:10B9B0007F147F1400242A7F2A1200626408132354
:10B9C00000364955225000000503000000001C22EB
:10B9D0004100000041221C000014083E0814000829
:10B9E000083E0808000000A06000000808080808D9
:10B9F000000060600000002010080402003E514971
:10BA0000453E0000427F400000426151494600210E
:10BA100041454B31001814127F1000274545453928
:10BA2000003C4A4949300001710905030036494983
:10BA3000493600064949291E00003636000000003C
:10BA40005636000000081422410000141414141487
:10BA50000000412214080002015109060032495930
:10BA6000513E007C1211127C007F49494936003E4C
:10BA700041414122007F4141221C007F4949494107
:10BA8000007F09090901003E4149497A007F080801
:10BA9000087F0000417F4100002040413F01007FBE
:10BAA00008142241007F40404040007F020C027F8A
:10BAB000007F0408107F003E4141413E007F09099C
:10BAC0000906003E4151215E007F091929460046C2
:10BAD000494949310001017F0101003F4040403F99
:10BAE000001F2040201F003F4038403F00631408E3
:10BAF00014630007087008070061514945430000BE
:10BB00007F41410000552A552A55000041417F00E0
:10BB100000040201020400404040404000000102D5
:10BB20000400002054545478007F484444380038BE
:10BB30004444442000384444487F00385454541846
:10BB400000087E0901020018A4A4A47C007F080458
:10BB500004780000447D4000004080847D00007F28
:10BB6000102844000000417F4000007C0418047845
:10BB7000007C0804047800384444443800FC242441
:10BB800024180018242418FC007C08040408004829
:10BB90005454542000043F444020003C4040207C4A
:10BBA000001C2040201C003C4030403C0044281039
:10BBB0002844001CA0A0A07C004464544C441414ED
:10BBC0001414141400000000000000000000000025
:10BBD0000000FC000000000002000000000C020C4D
:10BBE000020000000000000090D0BCD0BC90000318
:10BBF000000300001824FE448C0003020702010029
:10BC00001824D8B04C80000300010201C038E43889
:10BC1000E00001020201020208060000000000002C
:10BC200000000000000000F804020000000102040F
:10BC3000000204F800000004020100009060F860B7
:10BC400090000000010000002020FC2020000000E7
:10BC500001000000000000000000080600000000D5
:10BC60002020202020000000000000000000000034
:10BC700000000002000000000080601C02000403BD
:10BC800000000000F8040404F800010202020100B0
:10BC90000008FC0000000002030200001884442495
:10BCA000180003020202020008042424D800010242
:10BCB0000202010040B088FC800000000003020086
:10BCC0003C242424C400010202020100F824242C94
:10BCD000C0000102020201000C04E41C0400000088
:10BCE00003000000D8242424D8000102020201002D
:10BCF00038444444F8000003020201000000100030
:10BD00000000000002000000000020000000000011
:10BD1000060000000020508804020000000001021C
:10BD200090909090900000000000000000020488B5
:10BD300050200002010000001804C4241800000074
:10BD400002000000F804E494F8000102020202007C
:10BD500000E09CF0800002030000030204FC2424A5
:10BD6000D800020302020100F80404040C000102DE
:10BD70000202010004FC0404F800020302020100B4
:10BD800004FC24740C0002030202030004FC24746B
:10BD90000C00020302000000F0080444CC40000143
:10BDA0000202010004FC2020FC0402030000030244
:10BDB0000404FC040400020203020200000404FC68
:10BDC000040406040403000004FC24D00C04020351
:10BDD0000200030204FC040000000203020202034A
:10BDE000FC3CC03CFC0003000300030004FC30C426
:10BDF000FC04020302000300F8040404F80001023A
:10BE00000202010004FC24241800020302000000C6
:10BE1000F8848404F80001020207050004FC24648D
:10BE20009800020302000302182424448C00030239
:10BE3000020201000C04FC040C00000203020000DA
:10BE400004FC0000FC04000102020100047C80E00C
:10BE50001C040000030000001CE03CE01C00000388
:10BE600000030000049C609C040002030003020025
:10BE7000041CE01C04000002030200000C84641C8B
:10BE800004000203020203000000FE0202000000A0
:10BE900007040400000E30C0000000000001020092
:10BEA000000202FE00000004040700000004020477
:10BEB0000000000000000000000000000000080872
:10BEC0000808080800000200000000000000000050
:10BED0000040A0A0C00000010202030204FC2020D8
:10BEE000C00000030202010000C020206000000129
:10BEF0000202020000C02024FC0000010202030232
:10BF000000C0A0A0C0000001020202000020F8242E
:10BF100024040002030202000040A0A060200007E9
:10BF20000A0A0A0404FC2020C000020302000302E3
:10BF30000020E4000000000203020000000020E4F2
:10BF4000000008080807000004FC80E0202002032D
:10BF5000020003020404FC000000020203020200CB
:10BF6000E020E020C00003000300030020E02020C8
:10BF7000C00002030200030200C02020C000000134
:10BF80000202010020E02020C000080F0A02010088
:10BF900000C02020E0000001020A0F0820E040203D
:10BFA00020000203020000000060A0A020000002A8
:10BFB000020203000020F82000000000010202003D
:10BFC00020E00020E00000010202030220E02080C7
:10BFD00060200000030100006080E080600000033A
:10BFE00000030000206080602000020300030200C4
:10BFF00020E0208060200808070100000020A060E9
:10C000002000000203020200000020DE0200000007
:10C0100000070400000000FF00000000000F000007
:10C020000002DE20000000040700000002010204FC
:10C0300004020000000000000000000000000000FA
:10C040000000000000000000000000F800000000F8
:10C05000000000333000000000100C06100C060039
:10C06000000000000000000040C07840C0784000A0
:10C07000043F04043F040400007088FC0830000002
:10C08000001820FF211E0000F008F000E01800005A
:10C0900000211C031E211E0000F008887000000013
:10C0A0001E2123241927211010160E000000000065
:10C0B0000000000000000000000000E01804020082
:10C0C000000000071820400000020418E0000000F3
:10C0D0000040201807000000404080F080404000F1
:10C0E0000202010F01020200000000F00000000047
:10C0F0000101011F0101010000000000000000001B
:10C1000080B070000000000000000000000000008F
:10C110000001010101010101000000000000000018
:10C1200000303000000000000000000080601804B3
:10C13000006018060100000000E010080810E00090
:10C14000000F102020100F00001010F80000000059
:10C150000020203F202000000070080808887000A0
:10C160000030282422213000003008888848300020
:10C170000018202020110E000000C02010F8000040
:10C1800000070424243F240000F8088888080800D9
:10C190000019212020110E0000E0108888180000EE
:10C1A000000F112020110E0000380808C8380800C0
:10C1B0000000003F00000000007088080888700040
:10C1C000001C222121221C0000E010080810E000C1
:10C1D0000000312222110F00000000C0C00000004A
:10C1E000000000303000000000000080000000006F
:10C1F0000000806000000000000080402010080067
:10C20000000102040810200040404040404040002F
:10C21000040404040404040000081020408000000A
:10C220000020100804020100007048080808F0000F
:10C230000000003036010000C030C828E810E000DF
:10C240000718272423140B000000C038E00000006A
:10C25000203C23020227382008F8888888700000D4
:10C26000203F202020110E00C030080808083800A8
:10C27000071820202010080008F808080810E0001F
:10C28000203F202020100F0008F88888E8081000C0
:10C29000203F20202320180008F88888E808100094
:10C2A000203F200003000000C030080808380000CC
:10C2B00007182020221E020008F808000008F808CD
:10C2C000203F210101213F20000808F80808000054
:10C2D0000020203F2020000000000808F808080087
:10C2E000C08080807F00000008F888C028180800FF
:10C2F000203F20012638200008F808000000000038
:10C30000203F20202020300008F8F800F8F808002E
:10C31000203F003F003F200008F830C00008F80828
:10C32000203F200007183F00E01008080810E00038
:10C330000F10202020100F0008F808080808F0004F
:10C34000203F210101010000E01008080810E00072
:10C350000F18242438504F0008F888888888700007
:10C36000203F2000030C30200070880808083800A7
:10C370000038202121221C00180808F8080818009D
:10C380000000203F2000000008F808000008F8081E
:10C39000001F202020201F000878880000C83808CF
:10C3A000000007380E010000F80800F80008F80047
:10C3B000033C0700073C03000818688080681808E1
:10C3C00020302C03032C30200838C800C83808005F
:10C3D0000000203F2000000010080808C8380800AE
:10C3E0002038262120201800000000FE0202020052
:10C3F0000000007F40404000000C30C00000000002
:10C40000000000010638C00000020202FE00000029
:10C41000004040407F0000000000040202020400CF
:10C42000000000000000000000000000000000000C
:10C4300080808080808080800002020400000000F4
:10C4400000000000000000000000808080800000EC
:10C450000019242222223F2008F8008080000000DA
:10C46000003F112020110E0000000080808000009D
:10C47000000E112020201100000000808088F800AC
:10C48000000E112020103F200000808080800000DE
:10C49000001F222222221300008080F08888881842
:10C4A0000020203F2020000000008080808080004D
:10C4B000006B94949493600008F8008080800000E2
:10C4C000203F210000203F200080989800000000BD
:10C4D0000020203F202000000000008098980000ED
:10C4E00000C08080807F000008F80000808080000D
:10C4F000203F24022D302000000808F80000000032
:10C500000020203F202000008080808080808000EC
:10C51000203F20003F20003F80800080808000007E
:10C52000203F210000203F2000008080808000000C
:10C53000001F202020201F0080800080800000003D
:10C5400080FFA12020110E0000000080808080006C
:10C55000000E112020A0FF8080808000808080005D
:10C5600020203F212000010000008080808080008A
:10C570000033242424241900008080E080800000FF
:10C580000000001F2020000080800000008080004C
:10C59000001F202020103F208080800000808080AD
:10C5A00000010E300806010080800080008080803D
:10C5B0000F300C030C300F00008080008080800062
:10C5C0000020312E0E31200080808000008080808D
:10C5D00080818E701806010000808080808080003D
:10C5E0000021302C2221300000000000807C02025B
:10C5F00000000000003F404000000000FF0000007D
:10C6000000000000FF0000000002027C800000002B
:10C610000040403F00000000000601010202040447
:10C62000000000000000000000000000000000000A
:10C6300000000000000000000000000000000000FA
:10C6400000000000000000000000000000000000EA
:10C6500000F0F0F0000000000000000000017F0189
:10C660000000000000000000001C1C1C0000000076
:10C6700000008060301C8C60301C0C00000000004A
:10C6800000000000000000000000000000000000AA
:10C6900000000000000000E00000000000E00000DA
:10C6A0000086E69F86868686E69F860000011F013B
:10C6B000010101011F010100000080C06020F8207D
:10C6C000E0C00000000003070C18FF70E1810000CB
:10C6D0000000070F10107F100F070000806020601F
:10C6E00080000000E02000000F3020309F70DC3719
:10C6F0001030C0000000100E0300071810180700CB
:10C700000000C02020E0C0000000000080E01F38D2
:10C71000E88703C43C040000070F1810100B070D36
:10C720001010080000808C4C380000000000000051
:10C7300000000000000000000000000000000000F9
:10C74000000000000000000000000000000080E089
:10C75000300804000000000000FEFF01000000009F
:10C76000000000000000030F182040000004083003
:10C77000E0800000000000000000000001FFFE005B
:10C7800000000000004020180F030000000000001F
:10C79000000000000000C0000000000000426666CB
:10C7A0003C18FF183C6666420000000000000300D1
:10C7B00000000000000000000000800000000000F9
:10C7C000001010101010FF101010101000000000CA
:10C7D0000000030000000000000000000000000056
:10C7E0000000000000000000000000000000000049
:10C7F00000808C4C380000000000000000000000A9
:10C8000000000000000000000010101010101010B8
:10C8100010101000000000000000000000000000E8
:10C820000000000000000000000000000000000008
:10C83000000000000000000000001C1C1C000000A4
:10C84000000000000000000000000000E0380C00C4
:10C850000000000080701C03000000000060380E23
:10C860000100000000000000000080C06020206087
:10C87000C080000000FEFF010000000001FFFE007C
:10C880000001070E181010180E070100000080802C
:10C8900080C0E000000000000000000000FFFF007A
:10C8A0000000000000001010101F1F1010100000EA
:10C8B0000080402020202060C08000000003030092
:10C8C000804020381F070000001C1A19181818187B
:10C8D000181F00000080C020202060C080000000E1
:10C8E000000303001010182FE780000000070F104E
:10C8F000101010180F070000000000000000C0E03A
:10C90000F000000000C0B088868180FFFF808000BA
:10C91000000000000010101F1F1010000000E06059
:10C92000606060606060000000003F100808081848
:10C93000F0E0000000070B101010101C0F030000A7
:10C94000000080C040202020E0C0000000FCFF214B
:10C950001008080818F0E0000001070C181010106B
:10C96000080F03000000C0E06060606060E06000ED
:10C97000000003000000E0180700000000000000B5
:10C98000001F1F00000000000080C0602020202049
:10C9900060C080000087EF2C1818303068CF83000B
:10C9A00000070F0810101010180F07000000C0C07B
:10C9B00020202020C0800000001F3F604040402019
:10C9C00010FFFE0000000C1C101010080F030000E8
:10C9D0000000000000000000000000000000000057
:10C9E000000E0E0E0000000000000000001C1C1CC9
:10C9F0000000000000000000000000000000000037
:10CA000000000000000C0C0000000000000000000E
:10CA10000058380000000000000000000000008006
:10CA20004020100000001028448201000000000097
:10CA300000000000000001020408100000000000D7
:10CA4000000000000000000000848484848484844A
:10CA5000848484000000000000000000000000004A
:10CA600000001020408000000000000000000000D6
:10CA70000000018244281000000010080402010098
:10CA80000000000000C020201010101030E0C00096
:10CA90000003030000F010080C0703000000000072
:10CAA0001C1C1C0000000000000000C04060202092
:10CAB0002040C00000FCFF01F00E03C1FE03807F98
:10CAC0000001070E081111101109040200000000F6
:10CAD00080E0E000000000000000807C4340477FD1
:10CAE000F880000010181F1000000000131F1C1019
:10CAF00020E0E02020202060C080000000FFFF1028
:10CB0000101010182FE78000101F1F1010101010A9
:10CB1000180F0700000080C0402020202060E000A7
:10CB200000FCFF0100000000000001000001070EF2
:10CB3000181010100804030020E0E02020202040FE
:10CB4000C080000000FFFF000000000001FFFE00A9
:10CB5000101F1F10101018080E07010020E0E02021
:10CB6000202020202060800000FFFF101010107C8B
:10CB700000000000101F1F101010101010180600E9
:10CB800020E0E020202020206060800000FFFF10D7
:10CB90001010107C00000100101F1F10000000008A
:10CBA00000000000000080C06020202040E0000065
:10CBB00000FCFF0100004040C0C140400001070EE2
:10CBC000181010100F0F000020E0E02000000000FF
:10CBD00020E0E02000FFFF101010101010FFFF00F9
:10CBE000101F1F1000000000101F1F100000202049
:10CBF00020E0E020202000000000000000FFFF00F7
:10CC00000000000000001010101F1F101010000086
:10CC100000000000202020E0E02020200000000094
:10CC2000000000FFFF0000000060E0808080C07F07
:10CC30003F00000020E0E020000020A06020200055
:10CC400000FFFF30187CE3C000000000101F1F1021
:10CC5000000001131F1C181020E0E020000000005D
:10CC60000000000000FFFF000000000000000000C6
:10CC7000101F1F10101010101018060020E0E0E028
:10CC800000000000E0E0E02000FF013FFEC0E01EE9
:10CC900001FFFF00101F1000031F0300101F1F10D3
:10CCA00020E0E0C0000000000020E02000FF0003C2
:10CCB000071C78E08000FF00101F1000000000003B
:10CCC000030F1F00000080C060202060C0800000B3
:10CCD00000FEFF010000000000FFFE000001070E43
:10CCE000181010180C07010020E0E0202020202060
:10CCF00060C0800000FFFF2020202020301F0F0098
:10CD0000101F1F100000000000000000000080C085
:10CD100060202060C080000000FEFF0100000000D5
:10CD200000FFFE000001070E1111133C7C6721007B
:10CD300020E0E0202020202060C0800000FFFF10C5
:10CD40001030F0D0080F0700101F1F100000000364
:10CD50000F1C10100080C060202020204040E00008
:10CD600000070F0C1818303060E08100001F0C081D
:10CD700010101010180F07008060202020E0E02025
:10CD8000202060800100000000FFFF000000000183
:10CD900000000000101F1F100000000020E0E02035
:10CDA000000000000020E02000FFFF000000000065
:10CDB0000000FF0000070F181010101010080700E7
:10CDC0002060E0E02000000020E060200000077FFD
:10CDD000F88000807C03000000000000071F1C0793
:10CDE0000000000020E0E02000E0E0200020E02043
:10CDF0000007FFF8E01FFFFCE01F00000000031F1A
:10CE00000300011F03000000002060E0A0000020DC
:10CE1000E0602000000000038F7CF8C601000000E5
:10CE20000010181E130001171F1810002060E0E00A
:10CE30002000000020E06020000001073EF8E0181C
:10CE40000700000000000010101F1F10100000005D
:10CE500000806020202020A0E0E0200000000000F2
:10CE6000C0F03E0F0300000000101C1F1710101030
:10CE7000101806000000000000FC04040404040074
:10CE80000000000000FF00000000000000000000A3
:10CE9000007F404040404000000010E000000000E3
:10CEA0000000000000000000031C60800000000083
:10CEB00000000000000000030C708000000004046B
:10CEC000040404FC0000000000000000000000FF5B
:10CED00000000000000040404040407F0000000093
:10CEE00000000010080C040C0810000000000000F6
:10CEF0000000000000000000000000000000000032
:10CF00000000000000000000000000000000000021
:10CF10000000000000000000000000008080808011
:10CF200080808080808080800000000404080800E9
:10CF300000000000000000000000000000000000F1
:10CF400000000000000000000000000000000000E1
:10CF50000000000000000000000098D84464242471
:10CF6000FCF80000000F1F18101010081F1F1018E9
:10CF70000020E0F000000000000000000000FFFFC3
:10CF8000180804040CF8F00000001F0F181010100F
:10CF9000180F030000000000000000000000000067
:10CFA00000E0F8180404043C3800000000030F0CF3
:10CFB0001010101008060000000000000000002003
:10CFC000E0F0000000E0F81C04040408FFFF00008B
:10CFD00000030F18101010081F0F080000000000B9
:10CFE00000000000000000000000E0F84844444455
:10CFF0004C7870000000030F0C181010100804008B
:10D000000000000080C0602020E0C0000004040494
:10D01000FFFF040404040000000010101F1F101084
:10D0200010000000000000000000000000000000F0
:10D03000000070F88C04048CF874040C007076CF37
:10D040008D8D8D89C87870000020E0F00000000010
:10D05000000000000000FFFF08040404FCF80000CA
:10D0600000101F1F100000101F1F10000000000004
:10D0700000606000000000000000040404FCFC00EC
:10D080000000000000001010101F1F101010000002
:10D0900000000000000000606000000000000000D0
:10D0A000040404FCFC0000000000C0C08080C07FBD
:10D0B0003F0000000020E0F0000000000000000041
:10D0C0000000FFFF80C0F41C0404000000101F1FBC
:10D0D0001100031F1C1010000000202020E0F000B1
:10D0E000000000000000000000FFFF000000000042
:10D0F00000001010101F1F10101000000000000092
:10D10000000000000000000004FCFC0804FCFC0817
:10D1100004FCFC00101F1F10001F1F10001F1F1019
:10D120000000000000000000000000000004FCFC03
:10D1300008080404FCF8000000101F1F1000001075
:10D140001F1F100000000000000000000000000091
:10D1500000E0F0180C04040C18F0E00000030F0CC1
:10D16000101010100C0F0300000000000000000061
:10D17000000000000004FCFC080404040CF8F000AB
:10D180000080FFFF889010101C0F030000000000BB
:10D19000000000000000000000E0F81C0404040887
:10D1A000F8FC000000030F1810109088FFFF8000AB
:10D1B000000000000000000000000000040404FC67
:10D1C000FC100804040C0C001010101F1F1010108D
:10D1D000000000000000000000000000000000004F
:10D1E00000003078CCC48484840C1C0000001E181D
:10D1F00010101011190F06000000000000C0000000
:10D200000000000000040404FFFF04040400000008
:10D21000000000000F1F1010100C000000000000A4
:10D2200000000000000000000004FCFE00000004FC
:10D23000FCFE000000000F1F181010081F0F080050
:10D2400000000000000000000000000000040C3C92
:10D25000FCC40000C43C0C0400000000010F1E0EC2
:10D2600001000000000000000000000000000000BD
:10D27000043CFCC400E47CFC84807C040000071FA8
:10D28000070000071F07000000000000000000006A
:10D29000000000000004041C7CE4C0341C040400F2
:10D2A0000010101C1601131F1C18100000000000B5
:10D2B000000000000000000000040C3CFCC400C49E
:10D2C0003C0404000000C080C1370E0100000000D3
:10D2D00000000000000000000000000000001C042E
:10D2E00004C4F47C1C0400000000101C1F17111063
:10D2F00010180E0000000000000000F80C040000F0
:10D3000000000000001028EF0000000000000000F6
:10D310000000003F60400000000000000000FF002F
:10D3200000000000000000000000FF0000000000FE
:10D33000000000000000FF00000000000000040CDE
:10D34000F80000000000000000000000EF281000BE
:10D3500000000000000040603F00000000000000EE
:10D360000018060202040810202030080000000007
:10D3700000000000000000000000000000000000AD
:10D38000000000000000F010101010FF101010102E
:10D39000F000000000000F04040404FF040404046F
:10D3A0000F0000004040405F555555755555555F7D
:10D3B000404040000040200F094989790909090FC0
:10D3C0002040000000FE02424ACA4A4ACA4A4A4273
:10D3D00002FE000000FF40504C4340404F50505C64
:10D3E00040FF00000000F888888888FF88888888C7
:10D3F000F800000000001F080808087F8888888857
:10D400009F80F00080828282828282E2A2928A865B
:10D4100082808000000000000040807F000000004B
:10D4200000000000101010FF109008888888FF8806
:10D43000888808000444827F01808040432C1028A3
:10D44000468180000010101010D030FF30D0121C28
:10D450001010000010080402010000FF000001028B
:10D460000408100004040484E43C2724242424E455
:10D470000404040004020100FF0909090949897F25
:10D480000000000000FE225A8600FE9292929292C4
:10D49000FE00000000FF04080700FF4020030C14FA
:10D4A00022414000008040201806800007182040DC
:10D4B00080000000010020702826212020243860F0
:10D4C00000010100001012929292929292121202A6
:10D4D000FE0000000000003F101010103F004080D0
:10D4E0007F00000080828282FE8282828282FE82AF
:10D4F00082828000008040300F0000000000FF00AA
:10D500000000000000001011161010F0101014138D
:10D51000100000008181414121110D030D112141B5
:10D52000418181000008488808C83800901010FF29
:10D53000101010000020100C030418000043807F1E
:10D540000000000020102CE7242400E22C20BF2043
:10D5500028E600000101017F2111804F20100F10EB
:10D56000204F8000008060F80740300FF8888888DE
:10D5700088080800010000FF00000000FF080808FC
:10D58000080800000010608000FF000000FF00009D
:10D59000C030000040404043407F4040407F424117
:10D5A000404040001010F196909010E80784FC84F1
:10D5B00044C4040080601F40807F013F41405F44BD
:10D5C000484778002010EC27F42CE00022920ED27D
:10D5D000221E000080601F093F89FF000A0909FF21
:10D5E00009090800404848487F4848480090101002
:10D5F000FF10100040C444443F2424240000438012
:10D600007F000000404042CC0040A09E8282829E6B
:10D61000A02020000000003F908840432C102846A6
:10D6200041808000809090484C57242424544C44DE
:10D6300080808000000000FF4949497F494949FF37
:10D64000000000001010FF1090E02F29E909E929DF
:10D650002FE0000042827F414425150D05FE0D1587
:10D6600025454400008060F80740300FF88888881E
:10D6700088080800010000FF00000000FF080808FB
:10D6800008080000404424A4948C84FF848C94A453
:10D69000244440004040405F4A4A4A4A4A4A4A5F5E
:10D6A0004040400020222A2AAA6A3A2E2929292904
:10D6B0002920200008040201FF555555555555FFF6
:10D6C0000000000000083000FF20202020FF202064
:10D6D000222C200004040201FF8040300E010618B5
:10D6E00020408000000484844424548F1424448403
:10D6F00084040000413900003C4040424C404070EE
:10D70000040931002038E730004848FF484800FE4F
:10D7100042B20E00222712120082621F020200FF94
:10D7200008100F00100C4444444445C6444444448B
:10D7300044140C008040201E2040407F4444444458
:10D7400044404000000000FC4444444546444444F6
:10D75000447C00004020180700FC444444444444F6
:10D7600044FC00004044C4444444401010FF1010E6
:10D7700010F00000103C131014B840300E0140802F
:10D78000403F000080808888888888FF8888888853
:10D790008880800020201008040201FF0102040894
:10D7A000102020002038E730004848FF484800FE9D
:10D7B00042B20E00222712120082621F020200FFF4
:10D7C00008100F00100C4444444445C644444444EB
:10D7D00044140C008040201E2040407F44444444B8
:10D7E000444040001060028C00445454547F545410
:10D7F0005444400004047E010000FF1515155595A2
:10D800007F000000100C44241404050604041424B2
:10D8100044140C00004040414141417F414141419D
:10D82000404000002038E730004848FF484800FEEC
:10D8300042B20E00222712120082621F020200FF73
:10D8400008100F00100C4444444445C6444444446A
:10D8500044140C008040201E2040407F4444444437
:10D8600044404000008060F807000424242526245A
:10D8700024240400010000FF000000F9494949493F
:10D8800049F90000000000FC54545655545454FC0F
:10D8900000000000403000033941414559414173C7
:10D8A00000083000000000C080808080808080FC04
:10D8B00084808080808080C0C0000000000000FF65
:10D8C0007F404040404040FF40404040404040FF9B
:10D8D0007F00000000000000000000000000007F4A
:10D8E00070000000000000000000000000000000C8
:10D8F0000000000000000000000000FCF800000034
:10D900000000000000000000000000000000000017
:10D91000FFFE020202020202020202FFFF020202F4
:10D92000020202020202FF030000000000000000E9
:10D930001F1F040404040404040404FFFF0404047B
:10D940000404040404041F000000000000000000A0
:10D9500000000000000000000000007F3F00000009
:10D9600000000000000000000000000000000000B7
:10D9700000000000000000000000000000000000A7
:10D98000000000000000000000F8F8F0F070200037
:10D990000000000000000000000000000000000087
:10D9A0000000000000000000000000000000000077
:10D9B00000000000800000000000000000000000E7
:10D9C000000000000000000000FFFFFFFF0000005B
:10D9D0000000000000000000000000000000000047
:10D9E0008080000000000000000000000000000037
:10D9F0000000000000FFFFFE0606060606060606FB
:10DA0000060606060606060606FFFFFFFF060606D2
:10DA1000060606060606060606060606060606FFAD
:10DA2000FFFFFF07020000000000000000000000F0
:10DA30000000000000FFFFFF0000000000000000E9
:10DA4000000000000000000000FFFFFFFF000000DA
:10DA5000000000000000000000000000000000FFC7
:10DA6000FFFFFF00000000000000000000000000B9
:10DA70000000000000FFFFFF1818181818181818E9
:10DA8000181818181818181818FFFFFFFF1818187A
:10DA9000181818181818181818181818181818FF1F
:10DAA000FFFFFF0000000000000000000000000079
:10DAB0000000000002010100000000000000000062
:10DAC000000000000000000000FFFFFFFF0000005A
:10DAD0000000000000000000000000000000000145
:10DAE0000100000000000000000000000000000035
:10DAF0000000000000000000000000000000000026
:10DB0000000000000000000000FFFFFFFF00000019
:10DB10000000000000000000000000000000000005
:10DB200000000000000000000000000000000000F5
:10DB300000000000000000000000000000000000E5
:10DB40000000000000000000001F1F0F0F00000079
:10DB500000000000000000000000000000000000C5
:10DB600000000000000000000000000042F22EE271
:10DB700000F453F25A56F0000007020708070107A5
:10DB800001090F001011F2000000C03FC0000000AA
:10DB90000000070209060100010608001011F2004A
:10DBA000FE0A2A4A894939000804030609080A09B5
:10DBB00008090A0000FE0202F29292F20202FE003E
:10DBC000000F04040404040404040F0094F39200FE
:10DBD000F21410DF1014F200000F0408090402010F
:10DBE0000204090000001010F8000000000040408E
:10DBF0007F400000000000000000000000700808E6
:10DC00000810E0000060584442417000000000002D
:10DC1000000000000030080808F0600000304041BB
:10DC200041221C00000000000000000000008040B5
:10DC300030F8000000060948487F4000000000005E
:10DC40000000000004FD26E444F342FE2212F2002C
:10DC50000807080F0007080B08090D00202424BF3F
:10DC60002424488808FF0800080909070505000959
:10DC7000080F000008F453FA56F0896741E94F0095
:10DC800008070107090F0002020F02000202020248
:10DC9000FE02122242820200000000000F0000007B
:10DCA00000010000404040404040404040404000B3
:10DCB00000000000000000000000000010FC03084D
:10DCC0006888090A08E80800000F0008080B080C1B
:10DCD0000B080800DCB30880FE2AEA2BEA2AEE00D3
:10DCE000040402000F01070107090F00645CF744F8
:10DCF00010F7555555F7100002020F0104070505EE
:10DD0000050F0200FC242424FF242424FC0000002E
:10DD1000030101010709090909080E008868FF28A5
:10DD200040FE0202FE00000000000F080403000095
:10DD300007080E00001F25E525252525E5273000CD
:10DD400001090503010101010F0101000C047556D1
:10DD500054D7545675040C0000070101010F01014E
:10DD60000507000021E20004342C27F424240400D9
:10DD7000080708090909090F090909008888FF48E7
:10DD8000A4ACB5E6B4ACA40000080F00080A0B046C
:10DD9000040B080000FC2424E404FF04856604004E
:10DDA000080700020B04020102040F000404FC0433
:10DDB0000408FF080808F800020201090503000032
:10DDC0000808070000244484641C00488808FF08F1
:10DDD000080010080601030C000021203F0000008D
:10DDE0001028E7242400F21410DF1014F2000101BF
:10DDF0003F11092027100807081027004020F807C6
:10DE0000201807FC44444444040000003F00000084
:10DE1000003F0404040404000830C000FF000000B8
:10DE2000FF00C0380000202021203F2020203F217B
:10DE3000202020002021E60040A09E8282829EA019
:10DE4000200000001F0824201314081412212000B1
:10DE5000002FA9A9AFA9F9A9AFA9A92F00002020D7
:10DE60003F2020203C2020203F2020004444A49438
:10DE70008C84BF848C94A444440020202F2A2A2A16
:10DE80002A2A2A2A2F20200020222AAAEABAAEAA69
:10DE9000A9A9A92120000402013F2A2A2A2A2A2A04
:10DEA0003F000000041880FF001010907F901214B3
:10DEB00010000201003F20100C0300030C10200092
:10DEC0008484444424548F142444448484002018BB
:10DED000001C2020222C2030000418004042CC00DE
:10DEE0008888FF888888FF88880020100F102028E5
:10DEF000272020202F2020008844E2190020222201
:10DF000022E22222200000003F0000000020203FEB
:10DF10000000000008F8494AC81008E784FC44E4FF
:10DF20000400201F00203F00011F202F242738005D
:10DF300008F493FA96F000D28EE2929E0000201F21
:10DF4000041F243F0504043F04040400202424BFCC
:10DF5000242400488808FF0808001011110F09093F
:10DF6000000021203F0000004048C4A6AB929292DE
:10DF7000AAA6C240400000003F2424243F242424B9
:10DF80003F00000090DCB3980424FF2400FE0262EE
:10DF90009E000808040421110F01003F0808070033
:10DFA0000C0424242425E624242424040C0020101A
:10DFB0000F1020203F22222222202000404141FF3A
:10DFC0004141414141FF4141400020100C0300000C
:10DFD0000000003F00000000808888898E88F88853
:10DFE0008C8B88888000202010080403000304081C
:10DFF000102020000808FF880070577505755770BD
:10E00000000021213F0012120A063F060A121200E8
:10E010004020F807201807FC444444440400000052
:10E020003F000000003F040404040400000008F165
:10E030008E88884828D80FF02888888808000080B3
:10E04000704F80807F0202FF81BF81889C83E00047
:10E0500000000000000000000000000000000000C0
:10E0600000000000888888FF888880A0202020FF8A
:10E070002020200000C04444447F44242420018EFA
:10E0800080FF000000000000000000000000000011
:10E0900000000001000000000040F02C27F42CE0FC
:10E0A0006040E29CC262223E000000807F05057F46
:10E0B00005FF080A0909FF09090908000000000016
:10E0C000000000010000000001000000000000004E
:10E0D000888888FF888880A0202020FF20202000BA
:10E0E00000C04444447F44242420018E80FF00006B
:10E0F000000000000000000000000000000000011F
:10E1000000000000000010FF1090E0203EEA0A0A24
:10E11000F22E20E00000008282FF01804745351B7F
:10E12000FE0A172545C74400000000010100000059
:10E130000000010000000000000000008060FC03FF
:10E1400040201C0FF08888888888000000010000AB
:10E15000FF0000000000FF08080808080000000099
:10E1600000000100000000000100000000000000AD
:10E17000000000F010101010101EFA10121CD090A9
:10E1800000000080601F2121413F8080433C3866B1
:10E19000C180E0000001000000000001000000005C
:10E1A0000000000001000000080808F0080808202E
:10E1B00020FF202020E0000000003010100F088811
:10E1C00040201C038080807F0000000000000001D0
:10E1D000010000000000000101000000000000F844
:10E1E00088888888FF88888888F8080000000000F0
:10E1F000000F04040404FF848484848F80E0800082
:10E20000000000000000000000000000000000000E
:10E210000000000010D0FF90100000FC020202FE7F
:10E220000000000000180601FF0081631C030000CD
:10E2300000FF8080E00000000000010100000000FD
:10E24000000000000000000000000000FE9292921A
:10E2500092929292929EE080000000000888886866
:10E260001E08080808FE0A0808080000000001004F
:10E27000000000000000000100000000000000207D
:10E28000300809EA2C282F29282CEA082818000031
:10E290000000000078070505FE050505457C040023
:10E2A000000000000000000000000100000000006D
:10E2B0000000000000000000F888888C8B888888A7
:10E2C00088F80800000000000000FF48484848485F
:10E2D000484848FF00000000000000000100000066
:10E2E00000000000000100000000000010E0FF90AE
:10E2F00090502098878688902060000000080601D2
:10E30000FF000384B8808698C0B986808000000032
:10E3100000000100000000000000000000000000FC
:10E3200004F0000839640008030000000000000049
:10E33000800000000000000000000000E0EF000886
:10E340002F640008030000000000000080000000AF
:10E350000000000000000000F8EF000871640008F1
:10E36000030000000000000080000000000000002A
:10E3700000000000ECEF0008A166000803000000A8
:10E38000000000008000000000000000000000000D
:10E39000637C777BF26B6FC53001672BFED7AB7662
:10E3A000CA82C97DFA5947F0ADD4A2AF9CA472C00D
:10E3B000B7FD9326363FF7CC34A5E5F171D831157A
:10E3C00004C723C31896059A071280E2EB27B2759B
:10E3D00009832C1A1B6E5AA0523BD6B329E32F8413
:10E3E00053D100ED20FCB15B6ACBBE394A4C58CF0B
:10E3F000D0EFAAFB434D338545F9027F503C9FA8DF
:10E4000051A3408F929D38F5BCB6DA2110FFF3D2AC
:10E41000CD0C13EC5F974417C4A77E3D645D197360
:10E4200060814FDC222A908846EEB814DE5E0BDB5A
:10E43000E0323A0A4906245CC2D3AC629195E47991
:10E44000E7C8376D8DD54EA96C56F4EA657AAE08EB
:10E45000BA78252E1CA6B4C6E8DD741F4BBD8B8A86
:10E46000703EB5664803F60E613557B986C11D9EEC
:10E47000E1F8981169D98E949B1E87E9CE5528DF63
:10E480008CA1890DBFE6426841992D0FB054BB168F
:10E4900052096AD53036A538BF40A39E81F3D7FB19
:10E4A0007CE339829B2FFF87348E4344C4DEE9CB63
:10E4B000547B9432A6C2233DEE4C950B42FAC34ED8
:10E4C000082EA16628D924B2765BA2496D8BD1258E
:10E4D00072F8F66486689816D4A45CCC5D65B69232
:10E4E0006C704850FDEDB9DA5E154657A78D9D84D6
:10E4F00090D8AB008CBCD30AF7E45805B8B34506F6
:10E50000D02C1E8FCA3F0F02C1AFBD0301138A6B0F
:10E510003A9111414F67DCEA97F2CFCEF0B4E6733F
:10E5200096AC7422E7AD3585E2F937E81C75DF6EED
:10E5300047F11A711D29C5896FB7620EAA18BE1B53
:10E54000FC563E4BC6D279209ADBC0FE78CD5AF4F9
:10E550001FDDA8338807C731B11210592780EC5F3F
:10E5600060517FA919B54A0D2DE57A9F93C99CEF9B
:10E57000A0E03B4DAE2AF5B0C8EBBB3C835399619C
:10E58000172B047EBA77D626E169146355210C7DDA
:10E590008D01020408102040801B3600000000009E
:10E5A0000000000102030406070809000000000142
:10E5B0000203040041542B434F4E4E3D3130313065
:10E5C00030303030303031300D0A000041542B43B0
:10E5D0004F4E4E3D313031303030303030303031D0
:10E5E0000D0A000041542B434F4E4E3D3130313027
:10E5F00030303030303031310D0A000041542B437F
:10E600004F4E4E3D3130313030303030303030329E
:10E610000D0A000041542B434F4E4E3D31303130F6
:10E6200030303030303031320D0A000041542B434D
:10E630004F4E4E3D3130313030303030303030336D
:10E640000D0A000041542B434F4E4E3D31303130C6
:10E6500030303030303031330D0A000041542B431C
:10E660004F4E4E3D3130313030303030303030343C
:10E670000D0A000041542B434F4E4E3D3130313096
:10E6800030303030303031340D0A000041542B43EB
:10E690004F4E4E3D3130313030303030303030350B
:10E6A0000D0A000041542B434F4E4E3D3130313066
:10E6B00030303030303031350D0A000041542B43BA
:10E6C0004F4E4E3D313031303030303030303036DA
:10E6D0000D0A000041542B434F4E4E3D3130313036
:10E6E00030303030303031360D0A000041542B4389
:10E6F0004F4E4E3D313031303030303030303037A9
:10E700000D0A000041542B434F4E4E3D3130313005
:10E7100030303030303031370D0A000041542B4357
:10E720004F4E4E3D31303130303030303030303877
:10E730000D0A000041542B434F4E4E3D31303130D5
:10E7400030303030303031380D0A000041542B4326
:10E750004F4E4E3D31303130303030303030303946
:10E760000D0A000041542B434F4E4E3D31303130A5
:10E7700030303030303031390D0A000041542B43F5
:10E780004F4E4E3D3130313030303030303030410E
:10E790000D0A000041542B434F4E4E3D3130313075
:10E7A00030303030303031410D0A000041542B43BD
:10E7B0004F4E4E3D313031303030303030303042DD
:10E7C0000D0A000041542B434F4E4E3D3130313045
:10E7D00030303030303031420D0A000041542B438C
:10E7E0004F4E4E3D313031303030303030303043AC
:10E7F0000D0A000041542B434F4E4E3D3130313015
:10E8000030303030303031430D0A000041542B435A
:10E810004F4E4E3D3130313030303030303030447A
:10E820000D0A000041542B434F4E4E3D31303130E4
:10E8300030303030303031440D0A000041542B4329
:10E840004F4E4E3D31303130303030303030304549
:10E850000D0A000041542B434F4E4E3D31303130B4
:10E8600030303030303031450D0A000041542B43F8
:10E870004F4E4E3D31303130303030303030304618
:10E880000D0A000041542B434F4E4E3D3130313084
:10E8900030303030303031460D0A00002B434F4EBF
:10E8A0004E45435445443A302C31303130303030CD
:10E8B00030303031300000002B444953434F4E4E2E
:10E8C0003A302C313031303030303030303130006F
:10E8D00030303130000000002B434F4E4E45435442
:10E8E00045443A302C3130313030303030303030F7
:10E8F000310000002B444953434F4E4E3A302C31E7
:10E900003031303030303030303031003030303134
:10E91000000000002B434F4E4E45435445443A30CF
:10E920002C31303130303030303030313100000077
:10E930002B444953434F4E4E3A302C313031303016
:10E9400030303030303131003030313100000000B3
:10E950002B434F4E4E45435445443A302C313031D1
:10E960003030303030303030320000002B444953EA
:10E97000434F4E4E3A302C31303130303030303021
:10E980003030320030303032000000002B434F4E28
:10E990004E45435445443A302C31303130303030DC
:10E9A00030303031320000002B444953434F4E4E3B
:10E9B0003A302C313031303030303030303132007C
:10E9C00030303132000000002B434F4E4E4543544F
:10E9D00045443A302C313031303030303030303006
:10E9E000330000002B444953434F4E4E3A302C31F4
:10E9F0003031303030303030303033003030303340
:10EA0000000000002B434F4E4E45435445443A30DE
:10EA10002C31303130303030303030313300000084
:10EA20002B444953434F4E4E3A302C313031303025
:10EA300030303030303133003030313300000000BE
:10EA40002B434F4E4E45435445443A302C313031E0
:10EA50003030303030303030340000002B444953F7
:10EA6000434F4E4E3A302C31303130303030303030
:10EA70003030340030303034000000002B434F4E33
:10EA80004E45435445443A302C31303130303030EB
:10EA900030303031340000002B444953434F4E4E48
:10EAA0003A302C3130313030303030303031340089
:10EAB00030303134000000002B434F4E4E4543545C
:10EAC00045443A302C313031303030303030303015
:10EAD000350000002B444953434F4E4E3A302C3101
:10EAE000303130303030303030303500303030354B
:10EAF000000000002B434F4E4E45435445443A30EE
:10EB00002C31303130303030303030313500000091
:10EB10002B444953434F4E4E3A302C313031303034
:10EB200030303030303135003030313500000000C9
:10EB30002B434F4E4E45435445443A302C313031EF
:10EB40003030303030303030360000002B44495304
:10EB5000434F4E4E3A302C3130313030303030303F
:10EB60003030360030303036000000002B434F4E3E
:10EB70004E45435445443A302C31303130303030FA
:10EB800030303031360000002B444953434F4E4E55
:10EB90003A302C3130313030303030303031360096
:10EBA00030303136000000002B434F4E4E45435469
:10EBB00045443A302C313031303030303030303024
:10EBC000370000002B444953434F4E4E3A302C310E
:10EBD0003031303030303030303037003030303756
:10EBE000000000002B434F4E4E45435445443A30FD
:10EBF0002C3130313030303030303031370000009F
:10EC00002B444953434F4E4E3A302C313031303043
:10EC100030303030303137003030313700000000D4
:10EC20002B434F4E4E45435445443A302C313031FE
:10EC30003030303030303030380000002B44495311
:10EC4000434F4E4E3A302C3130313030303030304E
:10EC50003030380030303038000000002B434F4E49
:10EC60004E45435445443A302C3130313030303009
:10EC700030303031380000002B444953434F4E4E62
:10EC80003A302C31303130303030303030313800A3
:10EC900030303138000000002B434F4E4E45435476
:10ECA00045443A302C313031303030303030303033
:10ECB000390000002B444953434F4E4E3A302C311B
:10ECC0003031303030303030303039003030303961
:10ECD000000000002B434F4E4E45435445443A300C
:10ECE0002C313031303030303030303139000000AC
:10ECF0002B444953434F4E4E3A302C313031303053
:10ED000030303030303139003030313900000000DF
:10ED10002B434F4E4E45435445443A302C3130310D
:10ED20003030303030303030410000002B44495317
:10ED3000434F4E4E3A302C3130313030303030305D
:10ED40003030410030303041000000002B434F4E46
:10ED50004E45435445443A302C3130313030303018
:10ED600030303031410000002B444953434F4E4E68
:10ED70003A302C31303130303030303030314100A9
:10ED800030303141000000002B434F4E4E4543547C
:10ED900045443A302C313031303030303030303042
:10EDA000420000002B444953434F4E4E3A302C3121
:10EDB000303130303030303030304200303030425E
:10EDC000000000002B434F4E4E45435445443A301B
:10EDD0002C313031303030303030303142000000B2
:10EDE0002B444953434F4E4E3A302C313031303062
:10EDF00030303030303142003030314200000000DD
:10EE00002B434F4E4E45435445443A302C3130311C
:10EE10003030303030303030430000002B44495324
:10EE2000434F4E4E3A302C3130313030303030306C
:10EE30003030430030303043000000002B434F4E51
:10EE40004E45435445443A302C3130313030303027
:10EE500030303031430000002B444953434F4E4E75
:10EE60003A302C31303130303030303030314300B6
:10EE700030303143000000002B434F4E4E45435489
:10EE800045443A302C313031303030303030303051
:10EE9000440000002B444953434F4E4E3A302C312E
:10EEA0003031303030303030303044003030304469
:10EEB000000000002B434F4E4E45435445443A302A
:10EEC0002C313031303030303030303144000000BF
:10EED0002B444953434F4E4E3A302C313031303071
:10EEE00030303030303144003030314400000000E8
:10EEF0002B434F4E4E45435445443A302C3130312C
:10EF00003030303030303030450000002B44495331
:10EF1000434F4E4E3A302C3130313030303030307B
:10EF20003030450030303045000000002B434F4E5C
:10EF30004E45435445443A302C3130313030303036
:10EF400030303031450000002B444953434F4E4E82
:10EF50003A302C31303130303030303030314500C3
:10EF600030303145000000002B434F4E4E45435496
:10EF700045443A302C313031303030303030303060
:10EF8000460000002B444953434F4E4E3A302C313B
:10EF90003031303030303030303046003030304674
:10EFA000000000002B434F4E4E45435445443A3039
:10EFB0002C313031303030303030303146000000CC
:10EFC0002B444953434F4E4E3A302C313031303080
:10EFD00030303030303146003030314600000000F3
:10EFE000425434475461736B000000006C6F6769D2
:10EFF0006E666F5461736B00746573745461736BE8
:10F00000000000005363616E4B65795461736B00BF
:10F0100030F000080000002098070000F00200080F
:10F02000CCF3000898070020484A0000007200084E
:10F030004280012005FCFEFF8701100807071F1E04
:10F040001CFF0001100718E42222F40809310E30D9
:10F05000040007080133090907320F143200384150
:10F0600039500887FFFFFEFC80802E40080038E4FE
:10F070004040E43C2652FF3C113D513F000419083A
:10F08000080778E0080222F4C8E0E0E078220F01E7
:10F0900081784004FEFF8F78A2FE78223C783338D6
:10F0A000C001C178313F40070F076E756C6CA350EB
:10F0B00006003130313001A2310DA2320DA2330DE4
:10F0C000A2340DA2350DA2360DA2370DA2380DA225
:10F0D000390DA2410DA2420DA2430DA2440DA2453D
:10F0E0000D92460DA331300DA1D0A231D0A231D066
:10F0F000A231D0A231D0A231D0A231D0A231D0A23F
:10F1000031D0A231D0A231D0A231D0A231D0A2319F
:10F11000D0801531460000205741524E494E4720BD
:10F12000003C3C003E3E0001C0122B434F4E4E457A
:10F1300043542054494D454F55540001100ACCE525
:10F140000008D8E80008F4041A01B612FC101006F2
:10F1500050E900086C041602ED10062CE60008C801
:10F160001012E4141A0343125C10100640EA00085F
:10F170005C04120440128C2012B81012D414120530
:10F180005012BC20100630EB00084C04120650123E
:10F19000EC2012A81012C41412078F100A1CE700EA
:10F1A0000820EC00083C042D2603124C1012981085
:10F1B00012B4141A09A3127C20100610ED00082CBA
:10F1C00004120A5012AC2012881012A414120B5010
:10F1D00012DC20100600EE00081C041A0CF7120CBA
:10F1E000BC1278101294142A0DC911CC22F01C10F4
:10F1F00005EF00080E50126C2012680C1284042DCA
:10F200007E0312B4F0129C2412B8181210A012E45B
:10F21000F01214F01230041E1147031214B0128CB5
:10F22000F012A8141212A01244D01204F0122004FA
:10F230001213A0127420127CF01298141214A0164B
:10F24000A42012F41C1210F41215A012D420126C77
:10F25000F01688041E1600041204E016E40C1200D6
:10F26000F41E17E1031234D0125CF0167804121861
:10F27000A012642016D40016F01412195012942013
:10F28000124CF0166804161AA012C42016C40016F8
:10F29000E014161BA012F420123CF026580415DFCF
:10F2A0001224CC16B40012D014161DA01254F01261
:10F2B0002CF0124804161EA012842016A40012C0BE
:10F2C00014121F9025E4160CD065F825E41684E08E
:10F2D00065F825E416FC1065F825E42674F055F869
:10F2E00025E416EC0065F825E41664E065F825E4ED
:10F2F00016DCF065F82D0A051654F065F825E416BD
:10F30000CC0065F825E41644E065F825E412BCF06D
:10F3100065F825E41234E065F825E426ACE055F8FC
:10F3200025E41224F065F825E4169CF065F825E440
:10F3300026D02455F825E42A48D055F825E412C0F3
:10F34000F065F825E41238F065F825E412B0F065B0
:10F35000F825E41228F065F825E412A0F065F825F8
:10F36000E41A18DC65F825E41A90F065F825E4162F
:10F3700008E065F825E41A80E065F825E416F8F061
:10F3800065F825E416700065F825E41AE80065F8CC
:10F3900025E41260F065F825E42AD8F055F8023922
:10F3A0000001D0124A49414C4F4E475F324038214C
:10F3B0003523393231010122445A107400055200BC
:0CF3C00024F4000112AA01A15900000071
:0400000508000131BD
:00000001FF
